:10000000D8910120FD090000F9090000F90900005C
:10001000F9090000F9090000F909000000000000DA
:10002000000000000000000000000000F9090000CE
:10003000F909000000000000F9090000F9090000BA
:10004000F9090000F9090000F9090000F9090000A8
:10005000F9090000F9090000F9090000F909000098
:10006000F9090000F9090000F9090000F909000088
:10007000F9090000F9090000F9090000F909000078
:10008000F9090000F9090000F9090000F909000068
:10009000F9090000F9090000F9090000F909000058
:1000A000F9090000F9090000F9090000F909000048
:1000B000F9090000F9090000F9090000F909000038
:1000C000F9090000F9090000F9090000F909000028
:1000D000F9090000F9090000F9090000F909000018
:1000E000F9090000F909000000000000000000000C
:1000F000000000001D06000055090000C1090000B5
:10010000C9090000D1090000F9090000F90900003F
:10011000F9090000F9090000F9090000F9090000D7
:10012000F9090000F9090000F9090000F9090000C7
:10013000F9090000F9090000F9090000F9090000B7
:10014000F9090000F9090000F9090000F9090000A7
:10015000F9090000F9090000F9090000F909000097
:10016000F9090000F9090000F9090000F909000087
:10017000F9090000F9090000F9090000F909000077
:10018000F9090000F9090000F9090000F909000067
:10019000F9090000F9090000F9090000F909000057
:1001A000F9090000F9090000F9090000F909000047
:1001B000F9090000F9090000F9090000F909000037
:1001C000F9090000F9090000F9090000F909000027
:1001D000F9090000F9090000F9090000F909000017
:1001E000F9090000F9090000F909000031100000C8
:1001F000F9090000F9090000F9090000F9090000F7
:10020000F9090000F9090000F9090000F9090000E6
:10021000F9090000F9090000F9090000F9090000D6
:10022000F9090000F9090000F9090000F9090000C6
:10023000F9090000F9090000F9090000F9090000B6
:10024000F9090000F9090000F9090000F9090000A6
:10025000F9090000F9090000F9090000F909000096
:10026000F90900000348044B834202D0034B03B159
:100270001847704790C4020090C4020000000000BC
:100280000548064B1B1AD90F01EBA301491002D0F8
:10029000034B03B11847704790C4020090C402009A
:1002A0000000000010B5064C237843B9FFF7DAFFD1
:1002B000044B13B10448AFF300800123237010BD39
:1002C000080A00200000000090C4020008B5044B9A
:1002D0001BB104490448AFF30080BDE80840CFE7F4
:1002E000000000000C0A002090C4020070B50D460A
:1002F0001646044610B1081E18BF01200549064BDA
:10030000342298472368324629462046BDE870408B
:10031000184700BF54DC0100A5060000430904494A
:1003200000F01F0001224033824041F82320704733
:1003300000E100E07723584302300323B0FBF3F0E1
:1003400070477723584302300323B0FBF3F04FF498
:100350007A735843704770470139FDD8704700BF22
:10036000044A1168034609B903491160106803443F
:1003700013607047240A0020D89101204FF0FF300D
:1003800070474FF400534B600020704701207047C6
:100390000020704708B50146014B02489847FEE728
:1003A0009D6F010068DC010070474FF0FF3070471F
:1003B000F0B505681DB90F4BBDE8F0401847D1F8FE
:1003C00008C02C460026C2F1010ED4E90137934241
:1003D00095BFDB1973449B1ADB199C4507D9236829
:1003E000264613B9044B3046E6E71C46EDE7A54226
:1003F000E1D0F7E765060000910600002DE9F0471F
:10040000D0E90465037E0136DA07044606611FD48D
:10041000037E9B071CD4DFF84480DFF8449000F192
:100420001407CDB16B68AA68F31A934214D3384607
:10043000C0472B7C012B04D16E60324629463846DA
:10044000C847D4F814A0EB68284698475546E8E713
:10045000237E43F002032376BDE8F087990600006F
:10046000B103000038B50D46044610B1081E18BF90
:1004700001203B220549064B9847064B294620465A
:100480009847054B23600020206138BD81DC0100C6
:10049000A5060000850E0000FD03000038B50546E6
:1004A000003818BF01200849084B53229847084BD1
:1004B00028469847044620B92846064B98472046C8
:1004C00038BD6FF01000FBE781DC0100A5060000DD
:1004D000D50F0000C10F00002DE9F3410D46044681
:1004E00010B1081E18BF01201E49DFF890807A2243
:1004F000C047237E04F1140743F001032376294605
:10050000194B38469847064660B1237E154903F0DB
:10051000FE03002023767F22C0476FF0110002B057
:10052000BDE8F0812269114B6A6029463846984738
:10053000237E03F0FE032376237E13F002030ED006
:100540000B4B01A89847237E03F0FD03237620463A
:10055000084B984701A8084B98473046DFE71846F4
:10056000DDE700BF81DC010055060000B10300009B
:100570004D100000F10F00005B100000A506000008
:10058000014B1860014B1847280A00205703000050
:10059000054B10B51C68054B9847054B0146204696
:1005A000BDE81040184700BF280A002035030000AE
:1005B00059030000054B10B51C68054B9847054BC7
:1005C00001462046BDE81040184700BF280A002019
:1005D00043030000590300000A4A13889BB210B578
:1005E00043F4A0631380084B9847084B9847084B87
:1005F0009847084B9847BDE81040074B40F6FF70FE
:10060000184700BF00400041E10A0000AB060000AF
:10061000E9060000AD060000D90900000B4A9378F6
:1006200082B0DBB20193019B990705D5084B1B688B
:1006300013B1506802B01847019BDB0704D5044B87
:100640005B680BB1014AF4E702B070470000024159
:100650002C0A0020006800B970478842FAD10120B6
:100660007047000038B5074B0446984780F00100FA
:100670000D46054B05493922C0B2984723682B60C7
:10068000256038BD55060000A506000098DC010075
:1006900003680B600160704703680BB11A68026061
:1006A0001846704700B900BE704770470C4B0D4AA2
:1006B0005A63DA6B12F0060FFBD14FF402629A63B1
:1006C000022283F83020064AD36B9807FCD4044BEF
:1006D0001A6CD10702D41A6C9207F9D5704700BF83
:1006E000001000404D0E0100014B01225A7170476D
:1006F00000080040C3690B42FCD170470268034BFD
:1007000042F0020202600321184700BFF506000014
:100710000268034B22F0020202600321184700BF67
:10072000F50600000160014B03211847F5060000A3
:1007300070B50C4D06460FCD88B06C460FC495E8D9
:100740000F0084E80F006A46002352F8041BB142F0
:1007500002D1D8B208B070BD0133082BF5D100200A
:10076000F8E700BFD4DC010008B5034B98478000D0
:100770002E3000F0FE0008BD310700004109044A98
:1007800000F01F000123834042F82130704700BF72
:1007900000E100E04309064900F01F002033012278
:1007A000824041F82320BFF34F8FBFF36F8F704714
:1007B00000E100E04309044900F01F00012260331A
:1007C000824041F82320704700E100E070B5194BEA
:1007D0000446984728B11849184B40F26B22002074
:1007E0009847E369164D174E13F0010F0DD1164BC4
:1007F00003212046984723689B0703D5134B98474E
:100800000221A84705212046B04720460121A847DC
:100810000F49B0474FF4403363601F21A8470D4B89
:10082000A3604FF61143A3810023A373184684F8F5
:10083000303070BD31070000B6DC0100A5060000B5
:10084000F506000025070000F5060000110700006E
:1008500004001040020070002DE9F74305460038FF
:1008600018BF0120144B0C46CB2214499847144B57
:10087000204698470646D8B9124BAC619C4208BF47
:10088000114BDFF8509008BF1D6020460F4BDFF87A
:1008900048800F4F9847002405462B19D8B2019085
:1008A000C8470198C04701340198B847042CF4D1D7
:1008B000304603B0BDE8F083A5060000B6DC0100B9
:1008C000CD070000003000403C0A0020690700000E
:1008D0007D07000095070000B50700008069014B07
:1008E000184700BFFD06000083699962704783695D
:1008F00001229A757047836902229A757047000039
:1009000070B5044600380E4618BF01200F49104B41
:10091000154640F22B22984716F0FD0F09D1A36926
:100920000121022215B919751A7570BD99759A754C
:10093000FBE7012E04D1A3690422002DF7D1F3E7D0
:10094000032EF2D1A3698022F7E700BFB6DC0100D5
:10095000A5060000194B186810B58469237EDA07D4
:1009600008D5A37DDB0705D5012323750368BDE802
:1009700010401847237E990706D5A37D9A0703D513
:10098000022323758368F2E7237E5B070CD5638B14
:1009900003F0370313B1FF23638310BDA16A4368DB
:1009A000BDE81040C9B21847237EDB09F5D080238B
:1009B0002376C3689847638B9BB2EDE73C0A00201F
:1009C000004B184755090000004B18475509000017
:1009D000004B184755090000C30707D5044B054ACB
:1009E0001A6243F6FD7259681142FCD1704700BF8C
:1009F000001C004007010100FEE7000018491948EB
:100A0000814210B50AD0184BDA1C121A22F00302E8
:100A1000C41EA34238BF0022144B9847144B1548FC
:100A2000DA1C121AC11E22F00302994288BF00226A
:100A3000114B00219847114A114B22F07F029A6016
:100A4000D3F8882042F47002C3F88820BFF34F8F98
:100A5000BFF36F8F0B4B98470B4B9847FEE700BFD8
:100A600090C4020000000020040A0020CD6C0100A8
:100A7000D4D10020080A0020F96E01000000000017
:100A800000ED00E0216C01008D0A000008B5024B6A
:100A9000024C9847A047FDE7A10A0000D90A0000D0
:100AA00010B5074B9847074B9847074B9847074B9C
:100AB0009847074B9847BDE81040064B184700BFC2
:100AC000D90500004114000085130000B112000098
:100AD000AD130000D1150000004B18477D16000033
:100AE000064B42F28E329A8200229A75DA75DA69E2
:100AF00002F47C52DA6101221A747047001400403B
:100B000000238362C3690BB108381847704700237C
:100B10008362436A0BB108381847704770B50446C2
:100B2000054BA0F108052C309847236A1BB12846D5
:100B3000BDE87040184770BDCD0D000070B50E4681
:100B40001546044618B1D9B1101E18BF01200F4B2D
:100B50000F4940F23B129847B4F84420B4F84C30A7
:100B60009A420FD10023A4F844300123236304F1F7
:100B70000800084BA664A4F84C509847284670BD5E
:100B80000846E4E76FF01B00F9E700BFA506000088
:100B90001DDD0100EF080000838FB0F844209A4269
:100BA00010B504460AD0026C591C8187D15C044BF5
:100BB0009847044B2046BDE810401847024BFAE71F
:100BC000E9080000EF080000F70800002DE9F743EE
:100BD0000E461746044618B1E9B1101E18BF012091
:100BE0001049114BDFF850904FF4AC7298473434F1
:100BF0000E4B01A898470E4B204698470D4B804658
:100C000001A898470025A84501D0BD4205D1284636
:100C100003B0BDE8F0830846E2E771192046C847F3
:100C20000135F0E71DDD0100A50600004D100000B4
:100C30000D0E00005B1000008D0D0000F8B50D4694
:100C400016461F46044620B109B312B3181E18BF3A
:100C500001201249124B3A229847124B3A4631462C
:100C600004F134009847B0B90F4B294604F108004D
:100C7000984758B90D4B63600D4B23600D4BA36033
:100C80000D4BE3600D4B23610D4B6361F8BD0846CE
:100C9000DFE71046DDE76FF00C00F7E71DDD010030
:100CA000A5060000510D000059080000CD0B000002
:100CB0003D0B0000990B00001D0B0000010B000014
:100CC0000F0B000010B50446003818BF012005497D
:100CD000054B6122984704F10800044B9847002017
:100CE00010BD00BF1DDD0100A5060000DD080000ED
:100CF00070B5054600380C4618BF01201149124B4B
:100D0000164683229847012C0DD0022C11D0B4B97D
:100D1000321EAE6218BF0122012105F108000B4B03
:100D20009847002070BD321E6E6218BF012202215A
:100D3000F3E7321EEE6218BF01220321EDE76FF0E8
:100D40000C00EFE71DDD0100A50600000109000011
:100D500070B50E461446054618B189B1101E18BF6D
:100D600001200849084B28229847631E13EA040013
:100D700003BFC5E90130E8602E606FF00C0070BD64
:100D80000846EEE73ADD0100A506000038B50D463D
:100D9000044610B1081E18BF01200A4B0A49402220
:100DA0009847D4E902329A4209D062681340226817
:100DB000D35C2B70A3680133A360002038BD6FF0B3
:100DC0000900FBE7A50600003ADD010038B504463E
:100DD0000D460C4B0C49512201209847E36862688C
:100DE00013402268D554D4E90121E368591A91428D
:100DF00088BF9A1A03F1010388BFA260E360002054
:100E000038BD00BFA50600003ADD010010B5054958
:100E1000054B0446672201209847D4E90230C01AE6
:100E200010BD00BF3ADD0100A506000003690B42BA
:100E3000FCD1704770B5104D06460FCD88B06C469A
:100E40000FC495E80F0084E80F006A46002052F8AE
:100E5000041BB14202D130B908B070BD013008287E
:100E6000F5D10020F8E700200449054B4FF49E72AD
:100E700098474FF0FF30EFE774DD01005EDD0100C1
:100E8000A50600002DE9F843454B814608460C466F
:100E90009847444B4449C9F80C408D2280460120B4
:100EA00098472369414A13F0010F11D103212046CD
:100EB000904723689B0706D5236823F0020323602D
:100EC0009047022190470123236003212046904749
:100ED000374F142505FB08750121204690476E6A9F
:100EE00026600321904795F82A30E37306F00C063C
:100EF0002B8DE380082E4FF0010323733AD1EB6A68
:100F0000E361C0219047002323629047012363726D
:100F1000284B9C4204BF284BC3F80090142303FBCA
:100F20000873B3F92230002B0DDB5A09012103F0BD
:100F30001F03994002F12003204A42F82310BFF317
:100F40004F8FBFF36F8F142303FB0870B0F922306B
:100F5000002B0CDB03F01F015B099B0003F16043D6
:100F600003F5614301228A40C3F880211A60002002
:100F7000BDE8F8832EB9AB8DA383C0219047E683EB
:100F8000C3E7042EC2D195F82C302377C0219047B7
:100F900000236377904795F82B30E3762021B4E760
:100FA000350E0000A50600005EDD01002D0E0000DC
:100FB00074DD010000380040400A002000E100E03C
:100FC000C068036843F0020303600321004B184725
:100FD0002D0E000008B5C068034B03219847006838
:100FE000C0F3400008BD00BF2D0E00000020704778
:100FF00010B50A4BC0689847094B0A49044640F2AD
:101000000F12012098470848084B142202FB0400E5
:10101000BDE8104090F82200184700BF350E0000D0
:10102000A50600005EDD010074DD01001D03000067
:10103000054B1868C3689A7AD20703D501229A72C1
:1010400003681847704700BF400A0020EFF3108381
:10105000036072B6BFF35F8F7047BFF35F8F0368A3
:1010600083F31088704700004309012200F01F003D
:10107000012902FA00F210D002291FD029BBDB019E
:1010800003F1824303F500435A6091B241F080417D
:10109000120C996242F040420EE0DB0191B203F182
:1010A000824303F5004341F0804141F400315A602E
:1010B0009962084941EA12429A627047DB0103F1E2
:1010C000824303F500439A60DFE70349034B46225E
:1010D00000201847000002C0A8DD0100A50600009E
:1010E00030B54B1CC5B2184B00F01F044FEA50102E
:1010F0004FEAC010034407D1234493F8402002F084
:10110000FE0283F8402030BD181903EB540390F819
:10111000402002F0FE0242F0010280F8402093F8E5
:10112000302015F0010FC9B219BF02F00F0242EAD8
:10113000011202F0F00201F00F0114BFD2B20A4313
:1011400083F83020DFE700BF0080004101294FEA2B
:10115000501300F01F000FD002291DD069BB00EB17
:10116000C31000F1824000F5004090F8403003F0D9
:10117000FB0380F840307047DB0103F1824303F545
:10118000004381401844596090F8402042F0040226
:1011900080F8402099617047DB0103F1824303F539
:1011A00000430122824018445A6090F8401041F0F8
:1011B000040180F840105A6170470249024B8922AD
:1011C00000201847A8DD0100A5060000530010B557
:1011D000540104F4703403F47C73234302F00704D5
:1011E000520302F0E0522343134303EA010221EACF
:1011F00003018261416110BD38B5074C074B4FF4C4
:101200008075656198474FF08073C4F89430C4F8D6
:101210009830A56138BD00BF00800041CD110000AD
:101220002DE9F041074F884616461D460024A54289
:1012300001DCBDE8F08136F814204146B84701349E
:10124000F5E700BFF91100002DE9F84F4701154BF4
:10125000DFF858A0884616465FFA87FB002528FA73
:1012600005F2D20719D5EC19E4B2204671789847F7
:101270000BEB05090C4B31782046984771684846BE
:10128000D04704F01F016409E40104F18244012203
:1012900004F500448A40034B62610135202DDED104
:1012A000BDE8F88F691000004D110000E11000004A
:1012B0002DE9F7434FF000096A462D4BCDF8009019
:1012C00002254FF0FF346FF07F410120DFF8B0803E
:1012D0008DF801500194984729460820254F264E45
:1012E000C04749460820B84721460820B04729464C
:1012F0005C20C04749465C20B84721465C20B04787
:1013000029463720C04749463720B847214637206D
:10131000B04729460920C04749460920B847214619
:101320000920B04729463820C04749463820B847E9
:1013300021463820B04701210320C0472946032019
:10134000B84721460320B0470C4B4FF480729A6196
:101350004FF08052C3F818214FF40002C3F89820D0
:101360004FF08072C3F8982003B0BDE8F08300BF4F
:10137000491200004D110000E11000000080004102
:10138000691000007047000010B4064CD4E9002337
:10139000501C43F10001C4E90001034B5DF8044B0C
:1013A00001201847480A002061DC000070B512488F
:1013B000124B134C9847134A536943F480435361CB
:1013C000114B4022C3F8A420104B984704F11C0590
:1013D00002460F490F4B2846984701232361237685
:1013E0000D4A0E4B626104F10801284698472846D1
:1013F0000B4BBDE87040184710E000E0810500008D
:10140000480A002000080040001C0040ED0F0000CA
:10141000003800406504000089130000D904000072
:101420009D040000014B01221A707047000000204B
:10143000014B01221A607047800A002070470000AB
:10144000274B402273B5C3F89C204322C3F88C205D
:10145000244A25495369254E43F480535361244A55
:10146000002502F114040095102304322046B047F1
:10147000204B214E93F8452002F0FE0242F001027B
:1014800083F8452093F8322002F00F0242F0300238
:1014900083F8322093F8442002F0FE0242F0010269
:1014A00083F8442093F8322002F0F00242F0030265
:1014B00083F832200121114A2046B0472946104ABC
:1014C0002046B0470F4A02212046B0470E4B204627
:1014D00098470E480E4B02B0BDE87040184700BF59
:1014E000001C004000080040003000403D0C00009F
:1014F000800A002000800041F10C0000251400004B
:10150000311400003D140000C50C000099150000C6
:1015100015EB000010B5044C00232370034B9847D3
:101520002378002BFCD010BD00000020ED0200004D
:101530000FB430B5C5B0134C489D2846A047FF28CE
:101540001CD8114B4FF48072002104A8984749AB76
:101550004FF4807200210393009304A82B460B4D97
:10156000A84704A8A0470A4B82B204A90948984793
:10157000002045B0BDE8304004B070474FF0FF3068
:10158000F7E700BF81730100F96E0100898801004F
:1015900015150000940A002013B5C0B2032896BFA9
:1015A000064C074854F82000064CCDE900230B46B2
:1015B000024605490548A04702B010BD0CDE0100F7
:1015C000C4DD010031150000C9DD0100D6DD0100D8
:1015D00030B51A4B1A4C1B4D8DB098471A4B984793
:1015E00000221A4920464FF47F53A84701A8184B00
:1015F0009847184B049301A8174B02949847174B30
:1016000000209847164B002104469847154B164971
:1016100005469847002211462846144DA847144B0A
:10162000002120469847232204465A21A847114901
:10163000114B204698470DB030BD00BF591F000028
:10164000E40A0020C9D9000005170000080B00209B
:1016500089D90000B1180000E9D900009D1A0000E6
:1016600051490100FD46010028DE0100CD2A00009D
:10167000695B01001CDE01006D580100004B18473A
:1016800035FC00000B4908B54FF480734B610A4BE1
:101690000246187820B94FF4007048610121197092
:1016A000064B07486FF07F419847024B4FF480721A
:1016B0009A6108BD0080004101000020F91100007E
:1016C000808000410B4908B54FF480734B610A4B91
:1016D0000246187820B14FF400708861002119701B
:1016E000064B07486FF07F419847024B4FF48072DA
:1016F0009A6108BD0080004101000020F91100003E
:10170000808000412DE9F84300BF614F614E4FF0EA
:101710008054C7F818413220B047C7F8144100BFC1
:101720003220B047C7F818413220B04700BF4FF40D
:1017300080780A20C7F81480B0470520C7F81880C1
:10174000554D564CDFF86091B0470120A847142052
:10175000B0470120A8471420B0470120A847142013
:10176000B047E220C7F81480A8472F20A0470320E5
:10177000A0475420A047E020A8470120A047484B9D
:1017800064209847E020A8470320A0470120B047E5
:101790000120A8470120B047E620A8470120A04724
:1017A000CC20A047CC20A047B020A8472820A047A5
:1017B0003C4E8020A047B047C8470138C0F30720FF
:1017C000A047B047C8470138C0B2A047DFF8DC9057
:1017D000B047C8470138C0F30720A047B047C84703
:1017E0000138C0B2A0470020A047F020A84703203E
:1017F000A0473A20A8475520A047B420A847022078
:10180000A0470D20A0470020A0472B20A04728205C
:10181000A0470020A0470020A0470020A047B620F6
:10182000A8470120A0471D20A0470020A0470C206A
:10183000A0470920A0470020A0470020A0472A2059
:10184000A8470020A0470020A0470120A047DF2094
:10185000A0472B20A8470020A0470020A047012038
:10186000A0470F20A0472920A847BE20A847062050
:10187000A047FF20A0470120A047FF20A04700204D
:10188000A0470120A047C7F81880BDE8F88300BF33
:1018900000800041B505000085160000C516000057
:1018A0009105000029DB000035DB000059DB00005A
:1018B0002DE9F04FB1F904302DED028B002B08EE2D
:1018C000100A81B00D469046C0F28680B1F906300C
:1018D000002BC0F28180434FDFF818A1B847D047F2
:1018E000B5F90030834277DAB847DFF80CB1D84752
:1018F000B5F90260B0426FDDB5F90040B847D04796
:10190000B5F90430984224EAE47426EAE67655DC18
:10191000B847D04700F1FF3AB847D847B5F9063085
:1019200098424DDCB847D847471EDFF8D090DFF823
:10193000D0B02A20C847C4F30720D847E0B2D84720
:10194000CAF30720D8475FFA8AF0D8472B20C84748
:10195000C6F30720D847F0B2D847C7F30720D847C7
:10196000F8B2D8472C20C847AB882A8801339D1A83
:101970001D4A1E4B1178ADB221B14FF4007199612F
:1019800000211170C4F101044FF480725A61DFF834
:1019900074B004EB0A03DFF870A09CB26D00BE4285
:1019A00010DD124B4FF480729A6118EE100A104B42
:1019B00001B0BDEC028BBDE8F04F18479A46ABE78B
:1019C0001F46B2E7424623466FF07F41504601363C
:1019D000D847A84436B2E2E701B0BDEC028BBDE8BF
:1019E000F08F00BF29DB00000100002000800041D3
:1019F000E5DB000035DB000059DB00008516000048
:101A0000C51600002112000080800041003818BF78
:101A100001207047F0B51B4BC3B0074616469847E8
:101A2000E528044629D802AD0246174B3946284618
:101A300098472B1920222A5528225A7030229A7052
:101A4000124C7822DA70181D1C2226FA02F101F0DD
:101A50000F012144043AC97C00F8011B111DF4D187
:101A600029221A7300225A73094B0095BC22094996
:101A7000094C0320A04743B0F0BD054B0097BF229F
:101A8000F5E700BF8173010069EE00009964020070
:101A9000BD6402008F63020021EB000037B50446ED
:101AA00070B9084B9847044650B9074B0093074953
:101AB000074B084D2E220220A847204603B030BD18
:101AC000E46BFAE729DB000000650200D064020045
:101AD0007066020021EB000037B5044670B9084B70
:101AE0009847044650B9074B00930749074B084DE8
:101AF0004B220220A847204603B030BD246CFAE7F1
:101B000029DB000039650200D0640200846602000F
:101B100021EB000037B5044670B9084B98470446DE
:101B200050B9074B00930749074B084D5C22022030
:101B3000A847204603B030BD646CFAE729DB0000FB
:101B400072650200D06402009A66020021EB000078
:101B500070B5094D002428B964B12046074BBDE893
:101B60007040184790F8343013F0200F18BF044627
:101B7000A847F0E770BD00BF512300003D2A0000D8
:101B80002DE9F347067D16F00106054688461746FF
:101B90005CD1C468DFF8C8A04FF00109002C4CD11B
:101BA0002B7DDB0601D4002E50D1B9F1000F4DD0B2
:101BB0002846C0470446002E3AD1002846D00646A3
:101BC0004FF000092068D04702460028E6D1EB68B4
:101BD000A3423BD01F4E7BB118680192C369172105
:101BE0009847EB68019A18680E21B04701282DD15B
:101BF000EB681868184B98472068EC60C3690022AE
:101C000016219847EB68002218680D21B04701287B
:101C10001CD1EB681868114B9847EB6818680E4B9D
:101C200098472B6993B1284602B0BDE8F0471847A2
:101C30004FF00009002CC5D1B2E721462846B8472D
:101C4000002E08BF2646B0420446F3D102B0BDE8DC
:101C5000F08700BFA5210000B1290000511B000042
:101C6000492800000148024B18211847E48F002042
:101C700031E80000014A0249024B1847E1E8000040
:101C8000D5E80000811B0000014A0249024B1847B9
:101C900001E90000DBE80000811B000038B5037D8E
:101CA000C3F3001543F01003037504461B0754BF2C
:101CB000034B044B9847237D65F30413237538BD0C
:101CC000751C0000891C00002DE9F3410D460446F7
:101CD000002836D0DFF8C480244EC04730BBAB6B41
:101CE00073B1234B2846984750B1A86B214B224E25
:101CF0009847224B00932249224B7F220120B04774
:101D0000214BAC6320469847204B06469847074630
:101D1000F0B91C4B1A49009385220320164CA047AA
:101D20001B481C4932463B468847FEE70368AB42E6
:101D30000AD1194B00931249124B0F4C7522012006
:101D4000A04702B0BDE8F08101462046B047C5E794
:101D5000002EF6D035602046C0478642F1D1054BB3
:101D6000204602B0BDE8F041184700BFE1E800009E
:101D7000254400009D1C000021EB00008867020044
:101D80000D670200CA6702008DE800000D1A00000E
:101D90003E670200151A00004C670200D5E80000FB
:101DA000F8B5846B0646002C33D0E368002B30D0A6
:101DB0001B681C4D83421BD1237DDA0744BF6FF3A0
:101DC000000323752046A847E368834222D1164BBF
:101DD00020469847E36898421CD100680022C369F6
:101DE00017219847E3681B68B34204BF0023E360F0
:101DF0002046A8470D4F05465DB12B68B3422946E2
:101E000020460BD10A4B98470A4B28469847002397
:101E1000B363F8BD084B20469847E3E7B84705464B
:101E2000EAE700BFD5E80000DBE80000E1E80000D9
:101E300099E900001DED00009D1C000010B1C06874
:101E400000B10068704710B1007DC0F340007047DA
:101E5000F8B50C4D0C4E04460020A847002700B9E9
:101E6000F8BD90F8503043F0020380F850307368AA
:101E7000984208BF376014B1C36B9C4200D1C7635E
:101E8000A847ECE745DC0000888A0020014B0020D1
:101E9000184700BF511E0000014B5868704700BF33
:101EA000888A0020034690B190F8502042F0020248
:101EB00080F85020084A5068984204BF0020106003
:101EC00011B1DA6B8A4205D10022DA637047034B05
:101ED00008461847704700BF888A0020511E00003E
:101EE000014B1868704700BF888A00202DE9F04731
:101EF000051D124BDFF8489028460E4617469847B6
:101F00001FFA86F804461FFA87FA0CB9BDE8F08775
:101F1000238A43442382638A53446382A38A4344CB
:101F2000A382E38A5344E38220463A463146FFF7D0
:101F3000DDFF21462846C8470446E6E7D5E800000D
:101F4000E1E80000013900F1080311F8012F00F861
:101F5000012B9842F9D17047F0B5204E204D3378CF
:101F600085B043B11F4B00931F49204B78220220BC
:101F7000A84705B0F0BD1E4B1E4C1F4F98471F4B86
:101F800098471F4B98471F4B98471F4B98471F4830
:101F90001021A0471E4B009302224FF01F01CDE9F4
:101FA00001334FF60000B8471A4B98471A4B984731
:101FB0001A484FF4B871A04760211948A047194B3F
:101FC0009847194B9847194B01209847184B009395
:101FD0000120064B04493070A222C9E7908A0020F4
:101FE00021EB00000A680200DB670200E2690200E0
:101FF0004DEC000031E800004127010069FA0000C3
:1020000005E600005DDE0000651C0000FC8F00207E
:10201000040000200505010035510000A88F0020B4
:10202000B48F00208D1E000001D30000D5C8000031
:102030002268020073B50E4B04460E4698470546CB
:1020400068B90C4B0C49009340F2945203200B4E9C
:10205000B0470B480B4922462B468847FEE794F8C9
:10206000343066F3C71384F8343002B070BD00BF5B
:102070000D1A0000376A0200DB67020021EB000046
:102080003F680200151A000073B50E4B04460E4659
:102090009847054668B90C4B0C4900934FF4B4625D
:1020A00003200B4EB0470B480B4922462B4688476E
:1020B000FEE794F8343066F3000384F8343002B05D
:1020C00070BD00BF0D1A00004E6A0200DB670200FF
:1020D00021EB00003F680200151A00002DE9F043D3
:1020E000804687B016461F460C4691B1244B0846E1
:1020F0009847054668B9234B234900934FF4DB62A8
:102100000320224EB0472248224922462B468847C8
:10211000FEE7214D039400238DF810306B68059382
:1021200003AB6B601D4BD5F80890AF60984718B1B2
:1021300083680BB131469847B8F1000F02D03146A1
:102140002046C0476B68C5F808909B686B609DF897
:10215000103083B98CB194F834305A060DD520680C
:1021600058B10F4B3A4631469847431E58425841A2
:1021700007B0BDE8F0830020FAE70120F8E700BFD0
:102180000D1A0000136B0200DB67020021EB000058
:102190003F680200151A0000908A0020991E000076
:1021A000A52100007FB50E4603920446D8B10F4A20
:1021B0009047039B054668B90D4B0E49009340F2CA
:1021C000C46203200C4EB0470C480D4922462B46F2
:1021D0008847FEE7A06921460A4C3246A44604B06F
:1021E000BDE870406047012004B070BD0D1A0000CA
:1021F000266B0200DB67020021EB00003F68020053
:10220000151A0000DD20000073B50B4B04460E4686
:102210009847054668B9094B0949009340F21B727B
:102220000320084EB0470848084922462B468847F5
:10223000FEE7E66102B070BD0D1A0000346B0200CB
:10224000DB67020021EB00003F680200151A000066
:1022500010B1C36903B118470120704773B50B4B28
:1022600004460E469847054668B9094B094900934C
:1022700040F237720320084EB0470848084922460A
:102280002B468847FEE7266202B070BD0D1A00009B
:10229000496B0200DB67020021EB00003F6802008F
:1022A000151A00007FB50E4B039104469847039919
:1022B000054668B90B4B0C49009340F24972032064
:1022C0000A4EB0470A480B4922462B468847FEE78C
:1022D000606A094B984700B1606204B070BD00BFEE
:1022E0000D1A00005E6B0200DB67020021EB0000AC
:1022F0003F680200151A00004DF0000073B50E4B48
:1023000004469847054668B90C4B0D49009340F2C6
:10231000597203200B4EB0470B480C4922462B46FE
:102320008847FEE7E369002206212046628602B064
:10233000BDE87040184700BF0D1A0000776B02001F
:10234000DB67020021EB00003F680200151A000065
:1023500073B50B4B04469847054668B9094B0A49C3
:10236000009340F29F720320084EB0470848094985
:1023700022462B468847FEE7206802B070BD00BFAA
:102380000D1A0000936B0200DB67020021EB0000D6
:102390003F680200151A000073B50E4B04469847BB
:1023A000054648B10C4E2046B04725460446002855
:1023B000F9D1284602B070BD084B0949009340F29C
:1023C0006B720320074EB0470748084922462B4648
:1023D0008847FEE70D1A000051230000A56B02009C
:1023E000DB67020021EB00003F680200151A0000C5
:1023F0002DE9F7431E4B05469847044668B91D4B27
:102400001D49009340F27F7203201C4EB0471C48C8
:102410001C492A4623468847FEE72B681BB12846FD
:10242000194B984705461948194E1A4FDFF85C803A
:10243000B047044664B9184B00930F490D4B0F4D3C
:102440004FF4F2620220A847204603B0BDE8F083B3
:1024500004F130094846B04720B921464046B84704
:102460000446E7E78542EFD001464846B847F3E720
:102470000D1A0000B76B0200DB67020021EB0000C1
:102480003F680200151A000099230000A88F002061
:10249000D5E80000E1E800004C68020073B5104B7D
:1024A00004460D469847064668B90E4B0E49009300
:1024B00040F2AD7203200D4DA8470D480D4922464C
:1024C00033468847FEE7201D25B90B4B02B0BDE817
:1024D00070401847094B294602B0BDE870401847C4
:1024E0000D1A0000C76B0200DB67020021EB000041
:1024F0003F680200151A0000D5E80000E1E800007E
:1025000073B50E4B04460E469847054668B90C4B0A
:102510000C49009340F6010203200B4EB0470B48D4
:102520000B4922462B468847FEE70A4B04F110016F
:10253000304602B0BDE87040184700BF0D1A0000D9
:10254000386C0200DB67020021EB00003F680200EC
:10255000151A0000451F000073B5104B044698473C
:10256000054668B90E4B0F49009340F6220203203E
:102570000D4EB0470D480E4922462B468847FEE7D0
:102580000C4B2046984728B1238A028A981A00B239
:1025900002B070BDB4F91000FAE700BF0D1A0000D8
:1025A0004A6C0200DB67020021EB00003F6802007A
:1025B000151A00005123000073B5104B04469847CC
:1025C000054668B90E4B0F49009340F636020320CA
:1025D0000D4EB0470D480E4922462B468847FEE770
:1025E0000C4B2046984728B1638A428A981A00B259
:1025F00002B070BDB4F91200FAE700BF0D1A000076
:10260000576C0200DB67020021EB00003F6802000C
:10261000151A00005123000073B50D4B044698476E
:10262000054668B90B4B0C49009340F64A0203205B
:102630000A4EB0470A480B4922462B468847FEE718
:10264000A38A228A0133981A00B202B070BD00BF7B
:102650000D1A0000646C0200DB67020021EB000031
:102660003F680200151A000073B50D4B04469847E9
:10267000054668B90B4B0C49009340F656020320FF
:102680000A4EB0470A480B4922462B468847FEE7C8
:10269000E38A628A0133981A00B202B070BD00BFAB
:1026A0000D1A0000756C0200DB67020021EB0000D0
:1026B0003F680200151A000013B511B9283002B0A6
:1026C00010BD8DF800100024044B01946A460821C7
:1026D000984701280CBF01982046F0E751220000DE
:1026E0002DE9F84F0746984619481A4BDFF86090D5
:1026F000DFF87CB00D461646984704460CB9BDE895
:10270000F88F4445FBD0144B2146484698478246F3
:102710002068B8421AD1A179A94201D0FF2D15D164
:10272000A288B24201D0FF2E10D1D8470B4A904761
:10273000A1880B4A90470B4A0021204690470A4A3D
:10274000484621469047094A204690475446D5E7D7
:10275000FC8F0020DBE8000001E90000E55E0000DE
:102760003D5A0000DDDE000099E900001DED00008B
:10277000B926000037B50E4B04460D46984750B9B0
:102780000C4B00930C490D4B0D4C40F29242022031
:10279000A04703B030BD0B4B984720460A4C00239E
:1027A000FF222946A44603B0BDE83040604700BF81
:1027B000B926000094680200DB670200316D020058
:1027C00021EB0000F55E0000E12600002DE9F0415C
:1027D000154B04681548154E154F9847002590B9BC
:1027E00045B9A179134B20689847134B9847A188A6
:1027F000124B98470D48124B214698472046114BE3
:10280000BDE8F0411847A0420AD0026823689A4206
:1028100006D143686268534033F07F4308BF012507
:1028200001463046B847DAE7D5E80000FC8F0020C3
:10283000E1E80000B9260000E55E00003D5A000016
:1028400099E900001DED000073B50C4B0446984754
:10285000054668B90A4B0B49009340F64122032014
:10286000094EB04709480A4922462B468847FEE7E9
:1028700094F83400C0F3001002B070BD0D1A0000CF
:102880007F6D0200DB67020021EB00003F68020061
:10289000151A00002DE9F041354B86B004468846F4
:1028A0009847054668B9334B334900934FF4F072AB
:1028B0000320324EB0473248324922462B468847E1
:1028C000FEE7314F2046B847002841D12F4B204624
:1028D00098472F4B054698472E4B0646984785420A
:1028E0002CD1B4F932502C4B04F1100102A89847B6
:1028F000BDF80820ABB2D21AADF80820BDF80A2006
:10290000264DD21AADF80A20BDF80C201A44ADF8B5
:102910000C20BDF80E204146134404A802AAADF8CD
:102920000E30A847A0B1DFF884802046C047044697
:1029300088B91B4B04A93046984709E0194B30462B
:1029400098478542CDD0184B304698478542C8D02D
:1029500006B0BDE8F08104A904F110020846A847BA
:102960000028F5D02046B8470028F1D12046DDE701
:102970000D1A0000916D0200DB67020021EB0000E0
:102980003F680200151A0000492800009923000042
:10299000F12300009D1A0000451F0000B9E000006F
:1029A00039510000D91A0000151B00005123000006
:1029B0007FB51A4B05469847044668B9184B194924
:1029C000009340F20D220320174EB04717481849D4
:1029D0002A4623468847FEE7B5F93240154B05F1F4
:1029E000100102A89847BDF80820A3B2D21AADF88A
:1029F0000820BDF80A20D21AADF80A20BDF80C2034
:102A00001A44ADF80C20BDF80E201344ADF80E307A
:102A100002A9094B2846984704B070BD0D1A000062
:102A2000A86D0200DB67020021EB00003F68020096
:102A3000151A0000451F000095280000F7B5194B36
:102A400005469847044668B9174B1849009340F269
:102A500062220320164EB047164817492A462346DD
:102A60008847FEE7154B28469847071D144B044638
:102A700038469847854213D0124E2046B0472A4622
:102A8000394638460123104FB847E3692A460121E9
:102A9000204698472046334603B0BDE8F04018472B
:102AA00003B0F0BD0D1A0000BA6D0200DB67020032
:102AB00021EB00003F680200151A000051230000BE
:102AC000D5E80000B129000019EA00002DE9F04323
:102AD0002E4B87B00446884617469847054668B986
:102AE0002B4B2C49009340F2962203202A4EB047EC
:102AF0002A482B4922462B468847FEE726685EB9BE
:102B0000284B00932349224B234C4FF42772022079
:102B1000A04707B0BDE8F083228A338A9B1A03EBF3
:102B20000801628A738A9B1ADA1997B21FFA81F830
:102B300012B258EA07030DB20392EAD02046DFF83A
:102B40007090C84704A92046174B9847238A039AD8
:102B500043442382638A3B446382A38A9844E38A82
:102B6000A4F814801F4429462046104BE78298475A
:102B7000E36904AA022120469847F369224601210D
:102B8000304698472046C847C3E700BF0D1A0000EB
:102B9000E86D0200DB67020021EB00003F680200E5
:102BA000151A0000CA68020001250000ED1E000091
:102BB000B129000073B50F4B04460E4698470546F1
:102BC00068B90D4B0D4900934FF4337203200C4E3E
:102BD000B0470C480C4922462B468847FEE70B4B72
:102BE000204698470A4B02463146204602B0BDE8CF
:102BF000704018470D1A0000F76D0200DB670200F5
:102C000021EB00003F680200151A0000B925000002
:102C1000CD2A000073B50F4B04460E469847054673
:102C200068B90D4B0D4900934FF4367203200C4EDA
:102C3000B0470C480C4922462B468847FEE70B4B11
:102C4000204698470A4B01463246204602B0BDE86E
:102C5000704018470D1A0000046E0200DB67020086
:102C600021EB00003F680200151A00005925000002
:102C7000CD2A00002DE9FF47DFF8D8A0BDF930804C
:102C800004460D4617461E46D047814668B92A4B72
:102C90002A49009340F26D320320294DA847294864
:102CA000294922464B468847FEE71DB9274B204657
:102CB000984705462846D047814668B91E4B1F49AC
:102CC000009340F2713203201D4CA0471D481E495D
:102CD0002A464B468847FEE73A4604F1100103AB0B
:102CE00005F11000DFF87090C847184B2046984750
:102CF000BDF80E20BDF80C10B0F91230008A424425
:102D00003144091AD21A09B212B2114BADF80C10A3
:102D10002046ADF80E20984794F8493084F8487062
:102D20006FF34103A4F84460A4F84680256484F856
:102D3000493004B0BDE8F087116E0200DB67020085
:102D400021EB00003F680200151A0000512300002B
:102D5000CD2A00000D1A00005DE300002DE9F04FC0
:102D600087B0CDE90323DFF8A4B1BDF94030059366
:102D700080460E46D847044668B95A4B5A490093D4
:102D800040F295320320594DA847594859494246C7
:102D900023468847FEE7584BDFF874914046984732
:102DA000564B044640469847554A8246404690470F
:102DB00005464046C84707461EB95249404688471F
:102DC00006463046D8474E4A834668B9454B464981
:102DD000009340F2A1320320444CA04744484549A7
:102DE00032465B468847FEE7039B05EBD57507EB4C
:102DF000D77745F34F0547F34F07142B24D8DFE867
:102E000003F00B5819615E4B6B5B665819615E4BA2
:102E10006B585B5E61666B003046904700EBD0708C
:102E2000C5EB600424B23046C84700EBD070C7EB56
:102E3000600307E03046904700EBD070C5EB6004BC
:102E400024B27B420FFA83FA2E4A40469047049BF5
:102E5000318A028A19442144059B891A728A1A44CC
:102E6000438A5244D21A12B2274B09B240469847BD
:102E7000039B88F84830049BA8F84430059BA8F8C9
:102E8000463098F84930C8F8406043F0020388F8AB
:102E9000493007B0BDE8F08F3046904700EBD07066
:102EA000C5EB600424B23046C847C01B0FFA80FA55
:102EB000CAE76D422CB2C4E76D422CB2B3E76D4253
:102EC0002CB2F0E730469047401B04B2B9E73046D9
:102ED0009047401B04B2A6E730469047401B04B21F
:102EE000E1E700BF1E6E0200DB67020021EB00007D
:102EF0003F680200151A000059250000B92500009E
:102F00001926000051230000CD2A00000D1A0000F0
:102F10006926000073B5124B04469847054668B908
:102F2000104B1149009340F22A4203200F4EB04744
:102F30000F48104922462B468847FEE794F849502F
:102F4000B4F94600216C94F84820B4F9443000905C
:102F50002046AC074CBF084C084CA04702B070BDDF
:102F60000D1A0000316E0200DB67020021EB000049
:102F70003F680200151A00005D2D0000752C00004E
:102F8000F8B500210B4E0C4F0546B047044604B976
:102F9000F8BD2046B847E36900220421204698473F
:102FA0002046B8472046FFF7EBFF21462846B047AA
:102FB0000446ECE79D240000B129000073B5364BB0
:102FC00005460C469847064668B9344B3449009389
:102FD00040F21D520320334CA047334833492A4660
:102FE00033468847FEE7902C314E38D8722C19D8DA
:102FF000532C2ED83F2C22D8072C25D8012C18D999
:103000002846B047EB690022042128469847182C2F
:1030100034D8142C34D9286890B3C3690022012114
:1030200098472DE0A4F17302224B92B2D340DA0705
:10303000E6D42846334602B0BDE870401847A4F1F4
:1030400040021D4B92B2F1E7A4F11003082BF0D817
:10305000D6E75C2CD4D0A4F17003012BF7E748F23B
:1030600081039C4206D848F27F039C42C8D8FF2CBB
:10307000DFD1C5E748F28E039C42F9E7FF2CCAD0A6
:103080002846B047FF2C01D0230402D50B4B28461D
:10309000D1E702B070BD00BF0D1A0000406E020003
:1030A000DB67020021EB00003F680200151A0000F8
:1030B000B1290000071A002003100F00812F000023
:1030C00010B5044B044698472046034BBDE810401A
:1030D000FF21184775270000BD2F0000F8B51E4CD2
:1030E00006460D460027F9B22846A0470246F8B129
:1030F00001794FF0000C5FFA8CF3994215D95079A1
:1031000000F00600062823D10133DBB2994216D91C
:10311000106850F823309E4203D00CF1010C002EB1
:10312000E9D10E4BFF21284698470137402FDAD1CD
:103130000B4F00212846B847044610B9F8BD0023BC
:10314000E9E721463046FFF7C9FF21462846F2E766
:103150000029DDD10B46DEE7B9260000BD2F0000B7
:103160009D2400002DE9F84F0F4FDFF84090DFF865
:1031700040A006460020B84704460CB9BDE8F88FC9
:1031800004F130084046C847DFF828B005461DB9AD
:103190002046B8470446F0E729463046D04729463E
:1031A0004046D8470546F2E7F1DB0000D5E80000CD
:1031B000DD300000E1E800002DE9F0413B4B044622
:1031C0000D46817900689847394B9847A18801F0EE
:1031D0000F03082B16D84DB9B4F90820354B984782
:1031E000A1882068344BBDE8F0411847FF2DB4F9A1
:1031F0000C20F3D0B4F90830D21A6A4303EB22232F
:103200001AB2EBE70B2B38D8002D03DC22892B4BAD
:103210009847E5E7FE2D01DDA289F8E72389A28919
:1032200094F808C0C5F1FF07C3F345137B43C2F30D
:10323000451215FB0232237B0CF01F0C07FB0CFC24
:1032400003F01F0348F2810615FB03C37243734367
:10325000C3F3C45394F809C0C2F3C55243EA4212FF
:10326000637B4FEADC0CDB0807FB0CF715FB0373F1
:103270007343DB0D42EAC322C9E70D2B0FD8002DA3
:1032800003DC227A0E4B9847AAE7FE2D227BF9DC5D
:10329000237AD21A6A4303EB2223DAB2F2E77F2DB4
:1032A000D4BFA268E268074B984799E7B9260000A7
:1032B000E55E0000A55A0000BD2F0000755B000010
:1032C000455C0000195D000073B50B4B054698473F
:1032D000044668B9094B0A49009340F6B12203201D
:1032E000084EB047084809492A4623468847FEE762
:1032F000002002B070BD00BF0D1A0000016F020077
:10330000DB67020021EB00003F680200151A000095
:103310002DE9FF470D460646002877D1894B98478F
:10332000044640B9884B00938849894BCF2202203C
:10333000884DA84716E0884B30309847874B0446A5
:103340009847074660B9824B80490093D4220320F6
:10335000804DA8478248834922463B468847FEE77E
:1033600024B90024204604B0BDE8F0874C217E4BF0
:103370002046984794F83530A66166F3051384F823
:1033800035307A4BE3617A4B23622661794B3046C4
:1033900098470138A082784B304698470138E08240
:1033A000764B4C21201D9847B4F8483023F4FF7326
:1033B00023F00103A4F84830A38E23F47F6323F0A5
:1033C0000F0343F4E063002243F0010304F12800FB
:1033D000A386C4E910226A4B2263A263A2876262B9
:1033E000039098470398002D40F0D880654B002E3D
:1033F00000F09D80022120469847F3692246012172
:1034000030469847604B2046984793E0534FB84763
:10341000044660B94E4B4D490093ED2203204D4DBB
:10342000A8475A484F49324623468847FEE74A4B49
:10343000301D98470446B847074660B9444B434996
:103440000093F0220320434DA847454845492246B2
:103450003B468847FEE7002C83D0434BDFF838918A
:103460004C212046984794F8353026606FF30513B9
:1034700084F835303D4BE3613D4B23624FF000084B
:10348000B6F912306382C4F818804046778AC8477C
:103490004FF0320A00FB0AF0EF282CDD4046C84707
:1034A000502300FB0A30A02390FBF3F080B20744C6
:1034B000E782374B20469847012807461DD1B6F9C9
:1034C0001480A4F814800020C8474FF0640A00FB61
:1034D0000AF0EF281FFA88F808DD0020C8475027B7
:1034E00000FB0A77A02397FBF3F7BFB2A8EB07080E
:1034F000A4F8108054E70120D9E7B6F910702782AC
:103500000020C8474FF0640800FB08F0EF28BFB266
:103510000BDD0020C847502300FB0830A02390FBA0
:10352000F3F080B20744A7823AE70120FAE70121CD
:1035300020469847174B00930449054B40F28712E9
:103540000120F5E629DB000030690200DB6702009C
:10355000156F020021EB000045E800000D1A000085
:103560003E670200151A000051F20000594D00009C
:10357000C947000035DB000059DB000031E80000DE
:10358000695700001D050100B12900003F680200D5
:10359000C9320000806902007DDB0000544B05F158
:1035A00028019847534B04F1100005F1100198478A
:1035B000B5F93230638695F8303084F8303095F8BC
:1035C000313084F8313095F8483084F84830B5F916
:1035D0004430A4F84430B5F94630A4F846302B6C9A
:1035E00095F84920236494F8493062F3000384F885
:1035F0004930AB69A36195F8343094F83420DB0985
:1036000063F3C71284F8342095F8342094F83430EA
:1036100062F3000384F8343095F8343094F83420A1
:10362000C3F3400363F3410284F8342095F8353046
:1036300094F83520C3F3420363F3430284F8352042
:1036400095F8343094F83420C3F3800363F3820296
:1036500084F8342095F83430D2B2C3F3C00363F356
:10366000C30284F8342095F83430D2B2C3F3001387
:1036700063F3041284F8342095F83430D2B2C3F3E3
:10368000401363F3451284F8342095F83430D2B2F5
:10369000C3F3801363F3861284F8342095F83C302A
:1036A00084F83C3095F8352094F8353062F3000307
:1036B00084F83530A86B10B10F4B214698470F4B5B
:1036C0002846984778B1002E3FF434AF0C4B28467B
:1036D00098470C4B03902846984703990A4B02469B
:1036E0002046984789E6002E7FF487AE22E700BF88
:1036F000595F0000451F0000C91C00005123000055
:1037000059250000B9250000CD2A00002DE9FF4110
:10371000334B04460D4617469847064668B9314B69
:103720003149009340F2E5220320304DA84730484C
:103730003049224633468847FEE72F4B20469847BC
:10374000854204D12D4B2046984787423AD02046E7
:103750002B4EB04702A92B4B20469847638A013F66
:103760001F44E782284B204698470128ADB20BBF83
:10377000A38A238AC5F1010505F1FF350ABFED18BB
:10378000ED182582E36918BFA58202AA022120460E
:1037900098471E4B2046984718B1C369224601211D
:1037A0009847271D1A4BDFF8708038469847054622
:1037B0005DB92046B04794F84930DB0702D5154B78
:1037C0002046984704B0BDE8F081EB6902AA0321C6
:1037D0002846984729463846C0470546E8E700BFCF
:1037E0000D1A0000356F0200DB67020021EB0000BC
:1037F0003F680200151A0000192600006926000023
:10380000B129000001250000C93200005123000049
:10381000D5E80000152F0000E1E8000073B50F4B5C
:1038200004460E469847054668B90D4B0D4900936E
:1038300040F2273203200C4EB0470C480C49224678
:103840002B468847FEE70B4B204698470A4B01461C
:103850003246204602B0BDE8704018470D1A0000FD
:10386000566F0200DB67020021EB00003F68020098
:10387000151A0000192600000D37000073B50E4B15
:1038800004460E469847054668B90C4B0C49009310
:1038900040F6D72203200B4EB0470B480B49224677
:1038A0002B468847FEE794F83C301E4214BF0120A7
:1038B000002002B070BD00BF0D1A00007B6F020037
:1038C000DB67020021EB00003F680200151A0000D0
:1038D0007FB5134B04460D469847064668B9114B11
:1038E0001149009340F6DE220320104DA8471048EE
:1038F0001049224633468847FEE73F2D03D894F807
:103900003D0004B070BD00238DF80D3003AA0A4BB2
:103910008DF80C500921204698479DF80D00F0E7DE
:103920000D1A00008F6F0200DB67020021EB000020
:103930003F680200151A0000512200002DE9F74FE0
:10394000DFF894A0DFF894B005460E4617464FEA1C
:103950001228144665B924F4FE44222CA0B230D0BB
:1039600027D803282FD0C21F50425041000213E035
:10397000174B314628469847314681462846D0475E
:1039800007EB002084B20DF1060221464846D847D5
:10399000012804D1BDF9060003B0BDE8F08F18F08E
:1039A000800FD8D01EB928460A4B984705460026F6
:1039B000D0E7312809D0A0F1C00358425841000196
:1039C000EAE7FF20E8E70620E6E70F20E4E700BF8C
:1039D000B926000051230000D1380000B960000072
:1039E0002DE9F74FDFF874A0DFF874B005460E46F6
:1039F00017464FEA122814464DB924F4FE44293CD8
:103A0000012C96BF124B0020B3F8020612E0114BB6
:103A1000314628469847314681462846D04707EB2D
:103A2000002084B201AA21464846D847012804D183
:103A3000BDF8040003B0BDE8F08F18F0800FDCD0B3
:103A40001EB92846044B984705460026D4E700BF18
:103A5000E2690200B926000051230000D1380000BD
:103A6000416100002DE9F74FDFF880A0DFF880B05A
:103A700005460E4617464FEA1228144675B924F437
:103A8000FE446D2CA0B22AD048F2AD03984226D055
:103A90002C3818BF4FF0FF30C0B213E0114B314645
:103AA00028469847314681462846D04707EB0020F4
:103AB00084B20DF1070221464846D847012804D1B7
:103AC0009DF8070003B0BDE8F08F18F0800FD6D046
:103AD0001EB92846044B984705460026CEE700202D
:103AE000F0E700BFB926000051230000D1380000E4
:103AF000C96100002DE9F74FDFF884A0DFF884B03A
:103B000005460E4617464FEA122814466DB924F4AE
:103B1000FE44BE2CA3B227D048F28E02934201D0BD
:103B20007E2B23D1124B984711E0124B3146284689
:103B30009847314681462846D04707EB002084B29B
:103B400001AA21464846D847012803D1019803B06D
:103B5000BDE8F08F18F0800FD9D01EB92846064B6B
:103B6000984705460026D1E70448F0E70020EEE735
:103B700011050100B926000051230000A4B802007D
:103B8000D13800005162000070B50468A588206833
:103B9000A17905F00F03082B2A460CD80D4B984746
:103BA00020810023A380A17920680B4E23462A465A
:103BB000B047A58070BD0B2B02D8084B9847EFE7A4
:103BC0000D2B03D8064B98472072EAE7054B984720
:103BD000A060E6E73D390000E1260000E139000081
:103BE000653A0000F53A00002DE9F04F90F83D30BD
:103BF0008B429FB00446884600F04282954B98471E
:103C0000054668B9944B9549009340F2376203200A
:103C1000934EB0479348944922462B468847FEE787
:103C200094F83D300293002384F83D8003939DF87F
:103C30000C608E4B314620469847059040B147793D
:103C400017F008070BD0039B0133402B0393EED1F1
:103C5000874BFF2120461FB0BDE8F04F1847854D28
:103C6000B02231462046A847B1220990314620466D
:103C7000A847814B0890BE22314620469847B22281
:103C8000069031462046A847B322ADF82C003146B5
:103C90002046A847B422ADF82E0031462046A8475A
:103CA000B522ADF8300031462046A847B622ADF81F
:103CB000320031462046A847B722ADF834003146DD
:103CC0002046A8470497ADF83600049A0BAB33F8AA
:103CD0001270002F00F0B680684B05989847634B30
:103CE000314620469847664B0546984707F00F0334
:103CF000082B824600F2DC806B79DFF878B143F064
:103D000004036B71029B84F83D303A4631462046ED
:103D1000D8473A46079084F83D8031462046D84738
:103D20006A79079B6FF38202834281466A7100F0D1
:103D30008980029B84F83D303A4631462046D84778
:103D4000504B84F83D80024683463946504698479A
:103D5000012F22D147F6FF739B4501D099451CD115
:103D6000DFF848A12046D04700EBD07040F34F0564
:103D70002046D04747F6FF7300EBD0709B4540F3D9
:103D80004F002AD185421EDA05F1010B99450FFA41
:103D90008BFB02D101350FFA85F93B4B3B48984725
:103DA0002C4B054698478246E0B9394B2B49009386
:103DB00040F6B26203202A4CA04736482A492A46D8
:103DC00053468847FEE700F1010B99450FFA8BFB3C
:103DD000E3D101300FFA80F9DFE79945DDD1854263
:103DE000F7DAD7E7002D2DD0A5F808B0A5F80C908C
:103DF000294B2C60AF80AE710EA89847274B0F93CC
:103E0000274B1093274B11930022FF23CDE9142356
:103E1000099B1693089B069A0E955B421793069B87
:103E2000D11D013B12AA13F8010F02F8010B9942B0
:103E3000F9D19DF86E306FF300038DF86E300EA847
:103E4000194B9847049B0133062B04937FF43DAF35
:103E5000F9E600BF0D1A0000E66F0200DB67020002
:103E600021EB00003F680200151A0000B92600008F
:103E7000BD2F00003D390000F53A00000D60000044
:103E8000E55E0000A55A000045E80000FC8F002018
:103E9000F76F02003E670200A5DE0000B9310000A6
:103EA000893B0000CD2700004DDF000019260000EF
:103EB0000B2B4BD86B79DFF800B243F004036B7126
:103EC000029B84F83D303A4631462046D8473A4670
:103ED000814684F83D8031462046D8476A79ADF85E
:103EE0001C006FF382026A711FFA89F982B2914550
:103EF000A8D0029B84F83D303A4631462046D84748
:103F000039460246604B84F83D80814650469847CA
:103F10005E4B5F4898475F4B05469847824668B9B5
:103F20005D4B5E49009340F6C66203205C4CA0479F
:103F30005C485D492A4653468847FEE7002D81D0FC
:103F4000BDF81C30A5F80890AB8151E70D2B49D87E
:103F50006B79DFF868B143F004036B71029B84F85E
:103F60003D303A4631462046D8473A46079084F8D5
:103F70003D8031462046D8476A79079B6FF382021D
:103F8000834281466A713FF45DAF029B84F83D3005
:103F90003A4631462046D84739460246434B84F8D4
:103FA0003D80834650469847384B39489847394BAF
:103FB00005469847824668B9374B3849009340F622
:103FC000DB620320364CA047364837492A46534621
:103FD0008847FEE7002D3FF435AF85F808B085F837
:103FE0000C9005E7029B84F83D306B79DFF8D0B088
:103FF00043F004036B713A4631462046D8473A46AF
:104000000A90314684F83D802046D8470E906B795F
:104010006FF3820381466B710422254B0EA90AA817
:10402000984700283FF40EAF029B84F83D303A4693
:1040300031462046D847394602461E4B0A908346F1
:1040400084F83D8050469847104B11489847114BD3
:1040500005469847824668B90F4B1049009340F6D1
:10406000EF6203200E4CA0470E480F492A465346E4
:104070008847FEE7002D3FF4E5AEC5E902B9B7E693
:104080001FB0BDE8F08F00BF755B000045E8000081
:10409000FC8F00200D1A0000F76F0200DB670200A2
:1040A00021EB00003E670200151A0000455C00008D
:1040B000696C0100195D0000E1390000653A0000FB
:1040C000F53A000073B5114B04460D469847064675
:1040D00068B90F4B0F49009340F27E6203200E4DEA
:1040E000A8470E480E49224633468847FEE794F813
:1040F0003D3043EA05019D4305D00A4B204602B0FE
:10410000BDE87040184702B070BD00BF0D1A000036
:1041100004700200DB67020021EB00003F68020030
:10412000151A0000E93B000073B5114B04460D461B
:104130009847064668B90F4B0F49009340F28F62CB
:1041400003200E4DA8470E480E49224633468847A5
:10415000FEE794F83D301D4223EA050105D00A4BE5
:10416000204602B0BDE87040184702B070BD00BFE5
:104170000D1A000015700200DB67020021EB000041
:104180003F680200151A0000E93B000073B50B4BB5
:1041900004469847054668B9094B0A49009340F61A
:1041A000F5220320084EB0470848094922462B460D
:1041B0008847FEE7E06902B070BD00BF0D1A00003D
:1041C00028700200DB67020021EB00003F6802005C
:1041D000151A000073B50B4B04469847054668B99D
:1041E000094B0A49009340F61E320320084EB0479F
:1041F0000848094922462B468847FEE7606A02B014
:1042000070BD00BF0D1A000066700200DB6702007F
:1042100021EB00003F680200151A000073B50B4B3C
:1042200004469847054668B9094B0A49009340F689
:104230006F320320084EB0470848094922462B46F2
:104240008847FEE7A06B02B070BD00BF0D1A0000EA
:104250008A700200DB67020021EB00003F68020069
:10426000151A00002DE9F047394B044600221521AC
:104270009847384B20469847074610B1364B2046A2
:104280009847364B364DDFF8F4900021204698478A
:10429000FF2200231146204604F10408A847314BB1
:1042A0004046984705463DBB2F4B5E68012366BBE1
:1042B000DFF8CC80DFF8CC90DFF8CCA03046C047E8
:1042C000054645BB2A462946E369284D20469847BE
:1042D000274B20469847002837D1264B2046984741
:1042E00021463030A847606A234D00B1A8472046D8
:1042F0002B46BDE8F047184729464046C8470646C2
:104300002846FFF7AFFF3546CDE73268944208BF35
:104310003371B668CBE76B6BA34202D0AB6BA342A1
:1043200002D121462846C847EB6BA342AB6D08BFBC
:10433000EE63BB4205D1D047844202D121462846D4
:10434000C8472846C0470546BBE721460430C9E7B1
:10435000A52100001D420000A11D0000DDDE0000BF
:10436000E1260000D5E80000908A002099E90000CD
:1043700051230000F12300001DED0000E1E80000E2
:1043800045DC0000A51E0000E11E0000F7B51B4B38
:1043900004469847054668B9194B1A49009340F2FC
:1043A00093120320184EB0471848194922462B464D
:1043B0008847FEE7174B20469847174B20469847FB
:1043C0000646B8B9154B20469847054678B1C76BE5
:1043D0003B1B5F425F41124B2046984726B1F36971
:1043E00000220121304698470FB10023EB630020E3
:1043F00003B0F0BD00273D46EDE700BF0D1A0000F9
:104400009B700200DB67020021EB00003F680200A6
:10441000151A0000B129000051230000F12300000B
:104420006542000073B50E4B04469847054668B9CF
:104430000C4B0D4900934FF4386203200B4EB047EC
:104440000B480C4922462B468847FEE7A06B20B15B
:10445000094B9847231A5842584102B070BD00BF1B
:104460000D1A0000C7700200DB67020021EB00009C
:104470003F680200151A00003D1E000007B5028AC1
:1044800090F83030D21AADF80020828A1344ADF88B
:104490000430428A90F83130D21AADF80220C28A34
:1044A0001344ADF806300022024B6846984703B02B
:1044B0005DF804FB51E1000010B5002350F82340E3
:1044C000DAB21CB10133072BF8D11A4640F822109A
:1044D000012010BD2DE9F0471446B64FDFF8E08209
:1044E000012205460E46B84748F20C0220803146AC
:1044F0002846C047052881460AD800232373237520
:1045000084F8283084F8363084F84430BDE8F087E9
:10451000237B43B32C2231462846C047052820730D
:1045200021D929223146DFF890A22846D0472322FC
:10453000608031462846B847C0B2A07170B12A22C7
:1045400031462846D0472122A08031462846B84728
:104550002222208131462846B847608120223146F8
:104560002846B8476073237DEBB130223146284698
:10457000B8472082B8B13C2231462846C0470528BA
:1045800020750BD9312231462846B847C0B2608227
:10459000894B3922314628469847E08132223146FC
:1045A0002846B8476075237FE3B14022314628464C
:1045B000B8472083B0B14C2231462846C047052871
:1045C00020770AD9412231462846B8477A4B608382
:1045D0004922314628469847E08242223146284601
:1045E000B847607794F83630002B3BD0DFF8D4A181
:1045F0006E2231462846D047E062002832D06C2235
:1046000031462846C047052884F836002AD96D224D
:1046100031462846C047612284F837003146284693
:10462000B84794F83830003818BF012060F3000311
:1046300084F83830E06A614B9847022840F0AD803A
:104640005D4B692231462846984748F28E02A08683
:1046500031462846D0472063602231462846B84775
:1046600084F8390094F82830052B28D95022314697
:104670002846B847208410B35C2231462846C047FC
:10468000052884F828001AD9512231462846B8470F
:104690005222608431462846B8475322A0843146CE
:1046A0002846B847444BE08459223146284698476B
:1046B0005422E08331462846B84784F8290094F80C
:1046C0004430052B40D9DFF8FCA07F223146284634
:1046D000D047E063002837D07C2231462846C047C7
:1046E000052884F844002FD9732231462846B8475C
:1046F0007422A4F8480031462846B8472E4BA4F847
:104700004A0079223146284698477E22A4F846007E
:1047100031462846D0477022206431462846B847A3
:104720007122A4F84C0031462846B8477522A4F8F7
:104730004E0031462846B847722284F85000314670
:104740002846B84784F85100B9F1F90F3FF6DEAEBC
:10475000237B1FFA89F013FB00F3C3F307232373B2
:10476000237D13FB00F3C3F30723237594F828304C
:1047700013FB00F3C3F3072384F8283094F8363092
:1047800013FB00F3C3F3072384F8363094F8443066
:1047900013FB00F3C3F30723B6E694F83730052B79
:1047A0007FF65AAF044B6922314628469847A086C7
:1047B00052E700BF3D390000E1390000317A0000C6
:1047C000653A0000F53A00002DE9F04F022A99B051
:1047D00004460F46154659D1DFF830920021C847EC
:1047E0000646002850D1014601222046C84704222F
:1047F000824631462046C847052283463146204638
:10480000C847774B804604F1100103A89847BDF8CC
:104810000C30BDF80E201FFA8BF01B1AADF80C30CF
:10482000BDF8103018441FFA88F3D21AADF80E20E4
:10483000BDF81220ADF810001344ADF81230524606
:10484000684B03A938469847D0B1674F2C223146B0
:104850002046B847F92813D9314620222046C847B8
:1048600010F0FF010CD132222046C84710F0FF01A2
:1048700006D148F20C022046B847F92888BF012526
:10488000284619B0BDE8F08F0325F9E7002A56D174
:1048900003A8564BDFF874819847332229462046F7
:1048A000C04708B18DF82050514B03AA0021204683
:1048B0009847042200212046C047052206460021D1
:1048C0002046C04704F11009454B8246494601A8DD
:1048D0009847BDF80420B3B2D21AADF80420BDF851
:1048E00008201344ADF80830BDF806301FFA8AF0EE
:1048F0001B1AADF80630BDF80A301844ADF80A00AE
:1049000003AA394601A83B4B9847022200212046C2
:10491000C0470028B4D0384B384F1C20984701229C
:10492000064600212046C04749460246002330463D
:10493000B847334B04F5187130469847A0E7012A71
:1049400001D000259CE7DFF8C48002220021C04787
:1049500028B12C4B04F5187098472B4B98473322FD
:1049600000212046C0470028EBD0002503A81F4B9C
:1049700098471F4B8DF8185003AA294620468DF8FA
:1049800042508DF834509847294604222046C047AB
:104990000522064629462046C04704F110018046FC
:1049A0000F4B01A89847BDF80420B3B2D21AADF856
:1049B0000420BDF808201344ADF80830BDF80630D7
:1049C0001FFA88F01B1AADF80630BDF80A301844FB
:1049D000ADF80A00074B03AA394601A898474FE7EC
:1049E000451F0000BDE20000653A0000CD9D0000BB
:1049F000D5440000199E0000EDF00000419B00002E
:104A00003D990000F5990000A1ED00003D3900003E
:104A10002DE9F0411446284F48F28C0205460E4617
:104A2000B8470528207245D948F20C02314628467D
:104A3000B847F9289FBF237A13FB00F0C0F3072083
:104A40002072237A052B35D948F289023146DFF8E6
:104A500074801A4F2846C04748F2800220803146B1
:104A60002846B84748F28102A08131462846B84717
:104A700048F28202608131462846B84748F28302F4
:104A8000207631462846B8470D4B607648F28E02B4
:104A9000314628469847E28960604FF6FF739A4294
:104AA00008D0228A9A4205D048F28A023146284626
:104AB000C0472080BDE8F081653A00003D39000024
:104AC000F53A0000E1390000F8B51446234F48F2EA
:104AD000AC0205460E46B847052820703CD948F27E
:104AE0000C0231462846B847F9289FBF237813FBAC
:104AF00000F0C0F3072020702378052B2CD9002369
:104B000063804FF480732381AB8A2A8A01339B1A16
:104B1000C3F3C03202FA83F35B10A380EB8A6A8A84
:104B200001339B1AC3F3C03202FA83F35B10E380B4
:104B300048F2AD0231462846B847094BA07248F208
:104B4000A902314628469847064BA08148F2A002A8
:104B5000314628469847A073F8BD00BF653A00006B
:104B6000E13900003D3900002DE9F0475022754F32
:104B70008AB004460E46B8470546002840F0B48087
:104B80000025DFF8C8A17F2231462046D047804665
:104B900000287ED06C4B7C22314620469847052861
:104BA00077D9702231462046B847702205903146A9
:104BB0002046B8477E22814631462046D0474FF0F6
:104BC000000A47F61841CDE9011A02464146059B05
:104BD000DFF87C81CDF8009006A8C047BDF81830FA
:104BE000CDF820A0013BADF82430BDF81A30752275
:104BF000013B31462046ADF82630B8477322824645
:104C000031462046B8477422814631462046B8478F
:104C10005FFA8AF2804607AB08A904F11000DFF8BA
:104C200034A1D047BDF81E20BDF81C30B4F91010D7
:104C300008EB0200BDF820204B4412FA83F212B2B6
:104C4000891AA942B8BF2946BDF82250B4F91220EA
:104C500015FA80F52DB2521B09B28A42B8BF0A4636
:104C6000BDF8241011FA83F3B4F914101BB25B1AC7
:104C700012B29342B8BF1346BDF8262012FA80F054
:104C8000B4F9162000B2801A1BB29842B8BF184679
:104C900005B2402231462046B847804678B12A4BBB
:104CA0004C22314620469847052808D941223146F2
:104CB0002046B8474044A842B8BF284605B231460E
:104CC00004222046B8470522804631462046B84790
:104CD0004045B8BF404600B20028C4BF401905B2E5
:104CE00028460AB0BDE8F087174B5C2231462046C3
:104CF000984705287FF644AF532231462046B847EF
:104D000005EBD57500EB6505512231462046B847C5
:104D10005222804631462046B8470028B8BF40425C
:104D2000B8F1000FB8BFC8F100080135ADB280B2CC
:104D30001FFA88F840452CBF2D1845442DB225EAAE
:104D4000E5751EE73D390000653A0000F53A0000C0
:104D5000D50301005DE3000070B505461046172934
:104D600011D8DFE801F0551A102E371023150C105A
:104D7000103B1040401010101010101044531378C6
:104D80001BB92835556001240EE000235360FAE773
:104D9000BDE870402049214B1847214B012128468E
:104DA000984780F00100C4B2204670BD1D4B002121
:104DB00028469847B5F932309842B8BF18466886F9
:104DC000E1E795F8494014F00104DCD0164B284681
:104DD0009847E9E7154B28469847D4E7144B10212C
:104DE00028469847CFE71021124B2846F9E7124B87
:104DF00028469847114B98470D4B10B1062128467D
:104E0000EFE70221284698470421EDE70621EBE76A
:104E10000B4B00212846E4E7DB690200B94400009F
:104E20007D380000694B0000152F0000FD220000B6
:104E3000C5400000294100001D420000471E00003F
:104E40007527000038B5174D174B28689847174B42
:104E500004462868984758B9286801234268A36126
:104E6000116AC90709D400230AE0C3690BB1984746
:104E70002868A369002BF8D1EEE7126A9207F2D5F1
:104E8000E361C3681BB1A26804F11001984722686E
:104E900032B1636823B1A1688A4218BF1346A36088
:104EA00038BD00BF9C8A00200DDC000011DC000032
:104EB0002DE9F84300220C46174B1031074698475E
:104EC00010B90020BDE8F88394F83430DB06F8D43C
:104ED000236A9BB10222394620469847032806469A
:104EE000EFD004F104080D4BDFF8349040469847AA
:104EF00005462DB9012EE4D12046E3E70226F0E76E
:104F000029463846FFF7D4FF0028DBD12946404622
:104F1000C8470546EDE700BFBDE20000D5E8000048
:104F2000E1E800002DE9F04390F8348018F0100813
:104F30008BB004460F463CD1B0F93250314EDFF809
:104F4000CC9004A9B047BDF81020ABB2D21AADF88E
:104F50001020BDF81220D21AADF81220BDF814208E
:104F60001A44ADF81420BDF816203946134402A89F
:104F700004AAADF81630C847D8B1236A1BB142461F
:104F800002A92046984704A92046B04704AA3946FA
:104F90006846C84738B1271D1B4BDFF87480384678
:104FA0009847054645B9236A1BB1012202A920464C
:104FB00098470BB0BDE8F08308A92846B0476B8E30
:104FC000BDF82020D21AADF82020BDF82220D21A38
:104FD000ADF82220BDF824201A44ADF82420BDF8F5
:104FE00026206946134406A808AAADF82630C8470B
:104FF00018B106A92846FFF795FF29463846C0474D
:105000000546CFE701250000DBE80000B9E000001D
:1050100001E900002DE9F0470E46044628B9154B7A
:105020001868154B9847044658B131462046134F2F
:10503000DFF84C80DFF84C90B8472046C047054663
:105040000DB9BDE8F08705F1040A21465046C8476E
:10505000044650B92B6A1BB10122314628469847B5
:105060002846C0472C460546EAE731462046B84761
:10507000EBE700BF9C8A00209D1A0000254F00002E
:105080005123000001E9000073B51A4C1A4B064683
:1050900020689847194B05462068984720B305F1CA
:1050A00010023146164B174D68469847164B20683C
:1050B0009847164B0146684698476946A847144BDF
:1050C000206898476946A847124B20689847694668
:1050D000A8472068104B984708B9104B984702B072
:1050E00070BDC3690BB198472068AB69002BF8D13C
:1050F000D5E700BF9C8A00200DDC000011DC000019
:10510000B9E00000155000009D1A0000B14E0000EB
:10511000D91A0000151B000021DC0000454E0000DC
:10512000013900F1080311F8012F00F8012B984212
:10513000F9D17047704700002DE9FF410D46044644
:1051400018B92D4B9847044630B145B9B4F86831C9
:1051500065F30903A4F8683104B0BDE8F0810023C9
:1051600000932046254B98470138254BADF80400A5
:10517000204698470138ADF80600224B6A4629467A
:1051800002A898470028E7D0236913B102A9204656
:10519000984704F14805DFF8788000262F46B4F8D8
:1051A0006831B2B2C3F3090090421CD81F289BBFDC
:1051B0000930C0F309006FF3090302A991BF04EBA2
:1051C000C000A4F86831694638460F4A9047B4F8E1
:1051D0006831E06A5A1C62F30903A4F868310321BC
:1051E0000A4B9847B8E72946002202A8C047013673
:1051F00008350028D3D0AFE729DB000035DB0000FD
:1052000059DB0000B9E0000021510000A5FD0000BD
:10521000BDE20000014B1868704700BF9C8A002067
:105220002DE9F04F2DED028B824B834C8BB0054660
:105230009847EB6823600021804B08EE900A2846CF
:1052400098472368D96B002940F08B80B3F8682118
:1052500061F30902A3F868210BB0BDEC028BBDE835
:10526000F08F334493F84851002D3CD00136236829
:10527000B3F86821C2F309018E42F2D300206060C6
:10528000002971D16C4F3868B0F86831C3F3090355
:1052900003B36B4B9847002840F0A1812068694D0B
:1052A0004FF480714830A8472068202100F5A47091
:1052B000A8472368B3F868216FF30902A3F86821AF
:1052C00018EE900A604B9847014620688369002BCE
:1052D00040F0DD815D4B98475D4B0BB0BDEC028B20
:1052E000BDE8F04F18474FEAC609DFF884A109F17D
:1052F00048092068B0F86831C3F309039D42B5D26C
:10530000431993F8483153BBAE4228D04FEAC50B3E
:105310000BF1480B00EB0B014844B847F8B121688A
:105320004C4B01EB0B0208A84944984708A8D0470A
:10533000804620684844D047039020685844D047AE
:10534000039B184480450AD2D4F800B0424B0BEBC3
:10535000090008A9AB44984701238BF8483101356F
:10536000C7E73E4F002682E74F1E03F5A472791C63
:105370005BD100275B68DFF8C08093F820206FF3D3
:10538000000283F8202093F820206FF3410283F875
:1053900020204FF0000BD8F80050B5F86831C3F367
:1053A00009039B45BFF66EAF05EB0B0393F848313D
:1053B000002B40F0C6806B68BB4502BF93F82020ED
:1053C00042F0010283F8202093F820204FEACB0915
:1053D0006FF3410283F8202009F148030493EB188E
:1053E00008EE103A2846164B98471D4B002841D02E
:1053F00020689847002605461A4B06822068984781
:105400000138194BA8826E822068984723680138BA
:105410005A68E88292F8203043F0020382F8203084
:1054200018EE100A114B98477EE0D15D0029A1D0FB
:10543000013F9CE775DC00009C8A0020A5FD000070
:1054400021DC000051F2000089DC000015EE0000B4
:105450006DD900000DE100002151000081E2000043
:105460000DDC000035DB000059DB00008950000036
:105470009DE000004D4420689847B5F84C90B5F881
:105480004830B5F94E20039209F10109A9EB03094F
:10549000B5F84A3002F1010AAAEB030A06467D4B31
:1054A00020689847039A7B4B82420FFA89F90FFADA
:1054B0008AFA49DB20689847013803B2F268B2FBE8
:1054C000F9F25245A8BF52460392D8F8002012695B
:1054D000002A40D00022BDF90C900892ADF824209B
:1054E000D8F800000593CA4609F1FF390FFA89F987
:1054F0000269ADF8269008A99047BDF92610BDF8BD
:105500002220039B01318A1A12B29342059B1EDAB4
:10551000B9F1000FE4DC604B00936049604B614DD2
:105520004FF4CF720220A847D8F80000836943B136
:10553000049B18445C4B9847D8F804301844C8F8CA
:1055400004000BF1010B26E7B5F94E30B6E7BAF1CE
:10555000000FE0DD0391BDF80C10B5F94A20481E9C
:105560004FF00009059003981018013898420CDD9F
:105570004B45D9D0B5F9480021683082B5F94C00C7
:10558000B0827282F3824A6844E7B5F948003082FB
:10559000B5F94C00B082059872821FFA82FA10FAAF
:1055A00082F212B293429946A8BF91469342A6F85E
:1055B000169008DCD8F80020506890F8202042F0BF
:1055C000020280F82020394A18EE100ACDE906318F
:1055D00090470799069B8A440FFA8AF2C3E7386816
:1055E0004369002B7FF45AAE314B9847314B054647
:1055F0009847AB69002BFCD1D5F80090D5F808B0DE
:105600002D4B3868D94508BFD5F804909847002538
:10561000804643003A68B2F86811A8B2C1F30901A4
:1056200081427FF63BAE511991F8481109B101351D
:10563000F0E702EBC502B2F94800B2F94A60B2F8ED
:105640004C20013208FB0601121A05F1090012B2C2
:10565000C0000BEB410A4FEA420C09EB41010390F9
:105660003868039A1044B0F90600B042DFDB0693B5
:105670006246124B5046CDE9041C9847069B04999C
:10568000DDF814C0013636B29A441944E8E762687E
:1056900098471FE659DB000009710200D97002002B
:1056A0005971020021EB00009DE0000089500000CC
:1056B0000DDC0000454E000035DB000069EE000007
:1056C000437903F00603062B08BF0131037908BFB5
:1056D000C9B28B4286BF036853F82100002070478F
:1056E000F0B578B34FF0FF35CFB24FEA112C00235D
:1056F0002E46C1F30621C25CFF2A01D1284609E0EB
:10570000974211D1C41864788CEA040E1EF07F0F02
:1057100001D11846F0BD04F07F0434EA010E03D134
:10572000B442C4BF26B21DB202F00F02082A02D84A
:1057300002330233DFE70B2AFAD90D2A94BF013373
:105740000433F6E74FF0FF30E4E70139024411F883
:10575000013F00F8013B9042F9D17047014B042111
:10576000184700BF51F20000014B0821184700BF45
:1057700051F20000F7B5037904460E464BB10068BC
:10578000002250F82210B1423CD00132D1B28B42FB
:10579000F7D803B0F0BD013B9900214B9847214B4E
:1057A00005469847074668B91F4B204900934FF4B8
:1057B000827203201E4CA0471E481F492A463B46C2
:1057C0008847FEE74DB1002321791A46D8B28842B6
:1057D0000DD3013921712560DBE7184B0093134984
:1057E000114B134C4FF483720220A047D1E720687D
:1057F00050F82300B0421EBF45F822000132D2B259
:105800000133E3E7012BC6D10D4B984700232360FA
:10581000A38823F4FF7323F00103A380B9E700BF3B
:105820004DF000000D1A00006F7202006671020058
:1058300021EB00003E670200151A0000977102007C
:105840001DED00002DE9F3410F46054638B3294B05
:1058500098472979A1B9284B04209847274B04463B
:105860009847064690B9264B26490093D02203203C
:10587000254DA84725482649224633468847FEE756
:1058800001312868234B89009847E7E754B9224B38
:1058900000931C491A4B1C4CD2220220A04702B094
:1058A000BDE8F0816B792E79C3F34008DB0748BF70
:1058B00008F10108A6EB0802D2B24645C2F1010088
:1058C00006F180414FEA800001F1FF3138BF04202A
:1058D00000EB810100EB86004FEA82020F4B38BFDC
:1058E0000022214420440136984744F828702E7144
:1058F0002C60D4E77557000065EC00000D1A00001D
:105900008B7202006671020021EB00003E6702000C
:10591000151A00004DF00000D2710200016E010066
:105920004379DB0773B5054605D51A4B002102B054
:10593000BDE870401847184B04209847174B0446A1
:105940009847064668B9164B1649009340F235420F
:105950000320154DA8471548154922463346884768
:10596000FEE75CB9134B00930E490D4B0E4D40F210
:1059700037420220A847204602B070BD0E4B204699
:1059800098470E4B2146284698476B7943F0010310
:105990006B71F0E7C156000065EC00000D1A0000C5
:1059A000A47202006671020021EB00003E67020053
:1059B000151A0000027202005D57000045580000F1
:1059C00010B5034B0446006898470023236010BDC0
:1059D0001DED0000006828B10023C25CFF2A02D13F
:1059E000023398B2704702F00F02082A02D802333D
:1059F0000233F2E70B2AFAD90D2A94BF013304339C
:105A0000F6E7000037B505460C4679B10B686BB177
:105A10000846074B9847074B019098472860019A22
:105A20002168054B03B0BDE83040184703B030BDD6
:105A3000D559000065EC000069EE0000F8B50F468E
:105A4000044630B30668144B30469847051E20DBE9
:105A50002E44737883EA17235B061AD10F4B204636
:105A600007F00F0198470B290CD90E2934BF0323E7
:105A70000623C11AA942206806D8094B984720601E
:105A80000120F8BD0423F4E74219D25C42550135E8
:105A9000F0E70020F5E700BFE1560000D55900000F
:105AA0004DF0000070B50668284B86B005463046BC
:105AB000ADF80E10ADF80C200C46984700280DDB11
:105AC00033185B7883EA14235B0607D10230204B3E
:105AD000022203A93044984706B070BDFF23ADF8F9
:105AE000163028461B4B9847041E08BF0224043476
:105AF000A4B2194B214630469847184B2860984766
:105B0000064668B9164B174900934FF4C372032039
:105B1000154CA0472A681548154933468847FEE7C3
:105B200028680B4EA31F0DF10E0118440222B04746
:105B30002868231F03A918440222B0472868023CA2
:105B400002220DF116012044B047C5E7E1560000DE
:105B50004B570000D55900004DF000000D1A000011
:105B6000BA7202006671020021EB00003E6702007B
:105B7000151A000070B50668284B86B005463046F9
:105B8000ADF80C20ADF80E100C46984700280DDB40
:105B900033185B7883EA14235B0607D10230204B6D
:105BA000022203A93044984706B070BDFF23ADF828
:105BB000163028461B4B9847041E08BF02240434A5
:105BC000A4B2194B214630469847184B2860984795
:105BD000064668B9164B1749009340F2B5120320E8
:105BE000154CA0472A681548154933468847FEE7F3
:105BF00028680B4EA31F0DF10E0118440222B04776
:105C00002868231F03A918440222B0472868023CD1
:105C100002220DF116012044B047C5E7E15600000D
:105C20004B570000D55900004DF000000D1A000040
:105C3000CC7202006671020021EB00003E67020098
:105C4000151A000070B50668294B86B00546304627
:105C5000ADF80E108DF80D200C46984700280EDB8D
:105C600033185B7883EA14235B0608D10230214B9A
:105C700001220DF10D013044984706B070BDFF239D
:105C8000ADF8163028461C4B9847041E08BF022466
:105C90000334A4B2194B214630469847184B28606C
:105CA0009847064668B9174B174900934FF4F272AC
:105CB0000320164CA0472A681548164933468847E2
:105CC000FEE728680B4E631F0DF10E0118440222F7
:105CD000B0472868E31E0DF10D0118440122B047BA
:105CE0002868023C02220DF116012044B047C4E7A7
:105CF000E15600004B570000D55900004DF0000060
:105D00000D1A0000E07202006671020021EB000033
:105D10003E670200151A000070B50668284B86B071
:105D2000054630460292ADF80E100C469847002802
:105D30000DDB33185B7883EA14235B0607D102304E
:105D4000204B042202A93044984706B070BDFF23BF
:105D5000ADF8163028461C4B9847041E08BF022495
:105D60000634A4B2194B214630469847184B286098
:105D70009847064668B9174B1749009340F213221B
:105D80000320164CA0472A68154816493346884711
:105D9000FEE728680B4EA4F108030DF10E0118442C
:105DA0000222B0472868A31F02A918440422B04762
:105DB0002868023C02220DF116012044B047C4E7D6
:105DC000E15600004B570000D55900004DF000008F
:105DD0000D1A0000F27202006671020021EB000051
:105DE0003E670200151A00002DE9F0410E461746E5
:105DF0000546C0B1D0F80080B8F1000F13D00B4BAE
:105E000040469847041E0EDBA11C094B384602226F
:105E1000414498472B6823445878C0F3060000EAB1
:105E20001620BDE8F0814FF0FF30FAE7E1560000A0
:105E30004B5700002DE9F0410E4617460546C0B10C
:105E4000D0F80080B8F1000F13D00B4B40469847B4
:105E5000041E0EDBA11C094B384601224144984721
:105E60002B6823445878C0F3060000EA1620BDE8EA
:105E7000F0814FF0FF30FAE7E15600004B57000089
:105E80002DE9F0410E4617460546C0B1D0F8008016
:105E9000B8F1000F13D00B4B40469847041E0EDBA1
:105EA000A11C094B38460422414498472B682344DF
:105EB0005878C0F3060000EA1620BDE8F0814FF0E4
:105EC000FF30FAE7E15600004B570000427912F02C
:105ED000010305D0036892074CBF586818687047E3
:105EE00018467047437913F002031ABF0368186815
:105EF0001846704738B5044628B34379DA0708D501
:105F0000114B9847054620B1104B9847104B284637
:105F1000984763799B0709D50E4B2046984705465D
:105F200020B10A4B98470A4B28469847237913B16A
:105F30002068074B984700232360A38823F4FF635E
:105F400023F00703A38038BDCD5E0000C1590000D7
:105F50001DED0000E55E000070B50C46264B0546C1
:105F600098472368B3B163792079244E13F0010F69
:105F700003F00202224B17D16AB101388000984722
:105F8000286022792168013A92000431B0472379D0
:105F9000013B2B7170BD80009847286022792168F1
:105FA0009200B0472379F4E7CAB1023880009847DD
:105FB000286022792168023A92000831B04723799B
:105FC000023BDBB22B710F4E2846B04705462046F8
:105FD000B0470D4B01462846BDE8704018470138D0
:105FE00080009847286022792168013A92000431A4
:105FF000B0472379013BE4E7F55E000069EE00005D
:1060000065EC000021590000055A000043799A0709
:1060100073B5054604D51D4B02B0BDE87040184766
:106020001B4B042098471B4B04469847064668B90B
:10603000194B1A49009340F2CD220320184DA8476E
:1060400018481949224633468847FEE75CB9174B82
:1060500000931249104B124D40F2CF220220A84764
:10606000204602B070BD124B204698472146114B86
:10607000284698476B7943F002036B71DB0742BFF8
:106080002B68D3E90021C3E90012E9E7E55E0000CF
:1060900065EC00000D1A0000047302006671020036
:1060A00021EB00003E670200151A00002F7202006B
:1060B0005D570000455800002DE9F74F0F46904608
:1060C000054618B3006808B300261B4BDFF86CB018
:1060D000ADF806604FEA112A4FF0FF342A790FFA23
:1060E00086F9914503DBE043C0F3C0300EE0F1B226
:1060F000284698470DF106023946D84782450E4B8F
:1061000007D1BDF80630A8F80030012003B0BDE883
:10611000F08F6A79910706D5002804DBB9F1000FEA
:1061200001D15207EDD58442BEBFBDF80620A8F8C4
:10613000002004460136D1E7C1560000E95D0000A9
:106140002DE9F74F0F469046054610B3006800B39F
:1061500000261B4BDFF86CB0ADF804604FEA112A43
:106160004FF0FF342A790FFA86F9914503DBE043BB
:10617000C0F3C0300DE0F1B22846984701AA394675
:10618000D84782450E4B07D1BDF80430A8F800303F
:10619000012003B0BDE8F08F6A79910706D5002889
:1061A00004DBB9F1000F01D15207EDD58442BEBF27
:1061B000BDF80420A8F8002004460136D2E700BF4D
:1061C000C1560000E95D00002DE9F74F0F469046EB
:1061D000054618B3006808B300261B4BDFF86CB007
:1061E0008DF807604FEA112A4FF0FF342A790FFA31
:1061F00086F9914503DBE043C0F3C0300EE0F1B215
:10620000284698470DF107023946D84782450E4B7C
:1062100007D19DF8073088F80030012003B0BDE8B1
:10622000F08F6A79910706D5002804DBB9F1000FD9
:1062300001D15207EDD58442BEBF9DF8072088F8F2
:10624000002004460136D1E7C1560000355E00004B
:106250002DE9F74F0F4690460546F8B10068E8B1C2
:10626000194BDFF868B04FEA112A00264FF0FF34CF
:106270002A790FFA86F9914503DBE043C0F3C03079
:106280000CE0F1B22846984701AA3946D847824522
:106290000D4B06D1019BC8F80030012003B0BDE8CA
:1062A000F08F6A79910706D5002804DBB9F1000F59
:1062B00001D15207EED58442BEBF019AC8F8002032
:1062C00004460136D4E700BFC1560000815E0000DD
:1062D000F0B5C1F34513C2F1FF06C0F34514734393
:1062E00004FB023301F01F0400F01F07744348F25F
:1062F000810507FB02446B436C43C3F3C553C4F3EE
:10630000C45444EA4314C1F3C4237343C0F3C42008
:1063100000FB023205FB02F3DB0D44EAC320F0BDB3
:106320000B46052A2DE9F04100F01F0CC0F3451E75
:10633000C0F3C42803F01F06C3F34515C3F3C424F8
:1063400002D80846BDE8F08104EB08031F2B05EBDB
:106350000E0428BF1F2306EB0C053F2C28BF3F244B
:106360001F2D28BF1F25FF2A03F01F0304F03F0441
:1063700005F01F0508D14FF0000065F3040064F339
:106380004A1063F3CF20DDE765F3040064F34A109D
:1063900063F3CF20BDE8F041004B1847D162000005
:1063A0000B46052A2DE9F04100F01F0CC0F3451EF5
:1063B000C0F3C42803F01F06C3F34515C3F3C42478
:1063C00002D80846BDE8F081A4EB0803A5EB0E0453
:1063D000A6EB0C0523EAE37324EAE47425EAE575E9
:1063E000FF2A03F01F0304F03F0405F01F0508D146
:1063F0004FF0000065F3040064F34A1063F3CF200C
:10640000E0E765F3040064F34A1063F3CF20BDE8CE
:10641000F041014B184700BFD16200002DE9F04F59
:106420008DB0054605939DF85C309DF858709DF839
:1064300060B00493042B0E46144640F2A380002F54
:1064400000F0A080A44B9847A44B82469847A44BE9
:10645000D0F808908046324629460AA89847002876
:1064600000F09080BDF82820B8F81000BDF82C305E
:10647000B8F81260BDF82A50111A181AADF82C009D
:10648000BDF82E00801BAD1BADF82E00059809B29B
:106490002DB2ADF82810ADF82A50002845D1DAF811
:1064A0001400A6B200285AD1BBF1000F40F0278299
:1064B000894B9847B8F81430B8F81020BDF92A1065
:1064C0000133A3EB0208BDF82C30BDF928200133BD
:1064D0009B1A1BB20693BDF92E30089301330FFAB5
:1064E00088F85B1A1BB208FB0122012F0793824632
:1064F0000B4609EB420540F03281049BFA2B40F237
:106500009E80436A002B00F09580764B0AA898473E
:10651000F02840F28F80DAF82450ADF800400AAB42
:10652000424649465046A8472CE09AF80800C00762
:10653000B5D4581C801A059E0FFA80FE0598C6F146
:10654000010C01380CEB0006B645A8DD10F8016F10
:10655000802E4FF0FF3698BF00260670F2E75E4BA4
:106560009847B8F81420B8F81030BDF92A50013215
:10657000D21A012F064612B221D1AA46BDF92E30F9
:106580009A4502DD0DB0BDE8F08FBDF928700FFA15
:106590008AF8BDF92C309F4202DD0AF1010AEDE7CD
:1065A000049B0293ADF80440CDF800803BB27569BE
:1065B000059249463046A8470137059AE9E7BDF8F4
:1065C0002C70BDF9283005990137FF1AA1EB030A99
:1065D0003BB20593BDF92E309D42D3DCBDF9288036
:1065E0000FFA85FBBDF92C30984503DD059B01357D
:1065F0009A44EFE71AF808300499ADF8044013FB09
:1066000001F31B0A0293CDF800B00FFA88F3776903
:10661000069249463046B84708F10108069AE1E774
:106620002846069A3146B84745440134079BA342A1
:10663000F6DCA7E72C4F4FEA48080024F6E7036A88
:1066400013B3284B0AA89847F0281DD9274B069A60
:106650005A4514DCBDF92A60244F4FEA4808BDF9B9
:106660002E309E428EDC049B00932946DAF82040AF
:10667000069B3A465046A04745440136EFE723F8CB
:10668000026B0BF1010BE2E7049A194B20464FF025
:1066900000019847049EC4F3C42272430592C4F3D8
:1066A000451204F01F0402FB06FB04FB06FA4FEA46
:1066B0004802F64300F01F03C0F3451C0492C0F3E8
:1066C000C4204FF00008F6B2079A42457FF75AAF50
:1066D0002F464FF0000E3AE0155200000DDC00008E
:1066E000B9E000009DE0000035E50000A48A00202C
:1066F000D16200003A461FFA81F91488A14507F1DA
:10670000020715D05078059B37F8021CC00800FB23
:1067100006301378C4F3451403F01F0304FB06B4DA
:1067200003FB06A3C0F30420C4F3052CC3F3042326
:10673000147863F30404147014886CF34A141480FE
:10674000C4F3072460F3C70454700EF1010E069AD7
:106750007245CFDC049A08F101081544B4E739F812
:1067600012104FEA48020992049AFA2A40F2C480B1
:10677000069BDFF89882043B0493079B5B457FF7F9
:1067800001AFDDF814A0A946002413E0B9F8001009
:106790003046C047A9F8000009E01AF0030F0DD0F9
:1067A0001AF8012B1AB1FF2AF0D1A9F800600134C0
:1067B00009F10209069BA3425746EEDC05EB4409AA
:1067C000049BA3420EDA013F05EB4409069BA3425A
:1067D0004CDC099B1D44DDE90532134405930BF1A4
:1067E000010BCAE73B684BB101330CD1A9F800603B
:1067F000A9F80260A9F80460A9F806600437043417
:1068000009F10809DCE73A781AB1FF2A19D1A9F889
:1068100000607A781AB1FF2A1AD1A9F80260BA7812
:106820001AB1FF2A1BD1A9F80460FA78002AE5D032
:10683000FF2AE1D0B9F806103046C047A9F8060093
:10684000DCE7B9F800103046C047A9F80000E0E7DF
:10685000B9F802103046C047A9F80200DFE7B9F8DE
:1068600004103046C047A9F80400DEE717F8012FEE
:106870001AB1FF2A05D1A9F80060013409F1020913
:10688000A4E7B9F800103046C047A9F80000F4E7C3
:10689000059A12F80840D4B15C45B7F8009012D0C0
:1068A000FF2C17BF049ADDF810A014FB02F24FEA88
:1068B000122A07933988554B524630469847A346CB
:1068C000079B80B201E04945F3D13880494608F181
:1068D00001080237069A4245DADC099A1544DDE9D7
:1068E0000524224405920133089A93423FF74AAEA9
:1068F0002F464FF00008EDE70846DA46F4E7BBF113
:10690000010FB8F91000B8F914600CD0BBF1020FF8
:106910002DD03F4B00933F493F4B404C4FF4047206
:106920000220A0472EE6DFF8F8B00136361A36B25C
:1069300006FB05F0012F09EB400A4FEA460627D176
:106940004FF00008049A314B414620469847BDF964
:106950002E309D423FF716AEBDF928700AEB47096D
:10696000BDF92C309F4205DDB2440135EFE7DFF879
:10697000B4B0DAE7B9F800101FFA88F38B4203D0FD
:10698000049A20468846D84729F8020B0137E7E7E2
:10699000C2F1010203EB0208059B5F1A39F81010DF
:1069A0000FFA88F808464FF0000CBDF92E309D42D2
:1069B0003FF7E8ADBDF928900AEB4903BDF92C205B
:1069C000914503DDB24447440135EEE717F809204D
:1069D000BAB1624503D1B3F800E08E4510D0F92A70
:1069E00094BF0499049A05939CBF12FB01F2120A0A
:1069F00019882046D847059B17F809C0198880B226
:106A0000188009F101090233D8E700BFD162000004
:106A100059730200237302007E73020021EB000011
:106A200021630000A16300002DE9F04F8FB089467B
:106A300006939DF860300A939DF864309DF868A035
:106A40000B92042B059340F2D7800A9B002B00F099
:106A5000D3800A46B64B01460CA89847002800F0A0
:106A6000CB80B44B9847B44B054698478346836820
:106A7000BDF832E00893BBF81230BDF836C0BDF85F
:106A80003040008AAEEB03020FFA82F8ACEB03034E
:106A9000BDF83420ADF83630211A069BADF83280AF
:106AA00009B2101AADF83010ADF83400002B5ED1E9
:106AB0006B69002B72D1C4F101042244B9F804704F
:106AC000BBF81460BBF91030BBF9120012B2079288
:106AD000B9F90020B9F9029001360137F61ABF1A48
:106AE000A9EB000936B23FB2A8EB090906FB08F48E
:106AF00007FB09F9BAF1000F40F0EA81CEF101007D
:106B0000D51A84440B9B0FFA8CF04D1B09904D4411
:106B100008980C4403EB4505864B00EB440498476A
:106B20007B0008930A9B012B80464FEA460B40F0FE
:106B3000E080036A002B00F0AF80804B0CA89847E0
:106B4000F02840F2A980BDF93270BDF936309F427D
:106B500052DC059B00932A46079BD8F8206021460B
:106B60004046B047089B5C441D440137EDE72B7A53
:106B7000D8079DD40698069E531C1B1B1BB20138D8
:106B8000C6F101073E18B34292DD10F8016F802E66
:106B90004FF0FF3698BF00260670F3E7654B984725
:106BA000B9F80450B9F90010BBF81420BBF912C0B1
:106BB000B9F90270BBF91040BDF93260BDF930304F
:106BC000BDF9348001356D1A0132A7EB0C07121B99
:106BD0002DB2641AF71B0B9905FB074401EB440423
:106BE0000A99012912B2C3F1000A4FEA450B23D1D9
:106BF000BDF936309E4202DD0FB0BDE8F08FBDF921
:106C0000308037B2BDF93430984502DD5C4401363E
:106C1000EEE7059B029334F81830ADF80430009786
:106C20004569089907920FFA88F3069008F1010860
:106C3000A847DDE90602E5E708F10108A8EB03082B
:106C4000069B53440FFA88F89A46BDF936309E42A7
:106C5000D2DCBDF9309037B2BDF93430994503DD4F
:106C6000C2445C440136F0E71AF8093005990792EE
:106C700013FB01F31B0A029334F81930ADF804300A
:106C800000974569089906900FFA89F3A84709F11A
:106C90000109DDE90602DFE7059BFA2B25D9079BF1
:106CA000DFF89C805F000026099BB342A4DD2946E3
:106CB00020463A46C047089B5C441D440136F3E732
:106CC00034F8161035F81600059AC04724F8160057
:106CD0000136079BB342F3DC089B5C441D4401373B
:106CE000099BBB4288DD0026F3E7DFF858800027C8
:106CF000F6E7059BFA2B40F2E980079BDFF844801A
:106D0000CDF814A0043B0A93099B059A93427FF7A0
:106D100073AF069BAA46A146002625E0B9F80010ED
:106D2000BAF800000B93C0470B9BA9F8000016E0CF
:106D3000B9E00000155200000DDC00009DE00000ED
:106D400069EE0000D16200009A0711D013F8012B00
:106D50002AB1FF2AE2D1BAF80020A9F800200136B2
:106D60000AF1020A09F10209079AB2421F46EBDC56
:106D700005EB460A04EB46090A9BB34212DC013FCD
:106D800005EB460A04EB4609079BB34262DCDDE9EA
:106D9000063213440693089B1D44059B01335C4453
:106DA0000593B1E73B688BB1013316D1BAF80030D7
:106DB000A9F80030BAF80230A9F80230BAF8043065
:106DC000A9F80430BAF80630A9F8063004370436BA
:106DD0000AF1080A09F10809CEE73A782AB1FF2A30
:106DE00020D1BAF80030A9F800307A782AB1FF2A09
:106DF00020D1BAF80230A9F80230BA782AB1FF2AB5
:106E000020D1BAF80430A9F80430FA78002ADDD08D
:106E1000FF2AD7D0B9F80610BAF80600C047A9F87B
:106E20000600D3E7B9F80010BAF80000C047A9F887
:106E30000000DAE7B9F80210BAF80200C047A9F872
:106E40000200DAE7B9F80410BAF80400C047A9F85C
:106E50000400DAE717F8012F2AB1FF2A09D1BAF89E
:106E60000030A9F8003001360AF1020A09F10209DE
:106E70008AE7B9F80010BAF80000C047A9F8000086
:106E8000F1E7069B9A5D72B1F92A98BF059B34F829
:106E9000161035F816008EBF059A13FB02F2120A7F
:106EA000B84724F816000136079BB342E9DCDDE958
:106EB000063213440693089B5C441D440AF1010A00
:106EC000099B53457FF798AE0026EDE7364FF7E76D
:106ED000BAF1010F0CD0BAF1020F2BD0334B009353
:106EE0003349344B344C40F253320220A04783E6FE
:106EF000DFF8C8B0089800EB44040B9800EB490990
:106F00000A9801284FEA46064FEA470720D19B1A04
:106F100009EB4305BDF9363098453FF76DAEBDF935
:106F20003090BDF93430994507DD34443D4408F1D3
:106F30000108EFE7DFF888B0DCE734F8191035F81E
:106F40001900059AD84724F8190009F10109E8E762
:106F5000069BA9EB41095D1ABDF9363098453FF70C
:106F60004BAEBDF930A0BDF934309A4506DD079B24
:106F700034441D44B94408F10108EDE715F80A202E
:106F800072B1F92A94BF059B059A34F81A1039F8A2
:106F90001A009CBF13FB02F2120AD84724F81A0009
:106FA0000AF1010ADFE700BFD16200005973020055
:106FB000237302008B73020021EB000021630000A9
:106FC000A163000030B5A1B0044603920BA80C4A9F
:106FD000029190470B4A02991288ADF82E20204664
:106FE0000BAA094DA84704A8084A9047002200921E
:106FF0002046039B0299064C04AAA04721B030BD4D
:10700000CD9D00001C740200199E0000717A0000E2
:10701000A17A0000013900F1080311F8012F00F8EE
:10702000012B9842F9D170472DE9F04F2DED028BDD
:10703000B9B01C469DF810310C939DF8143107939C
:1070400082469C4B22A88946154698479A4B9847FA
:107050009A4B9847BDF88830018A428A04905B1A9F
:10706000ADF88830BDF88A309B1AADF88A30BDF88B
:107070008C305B1AADF88C30BDF88E309B1AADF8B1
:107080008E308F4B98470B90F8B96388EBB9238902
:10709000B3F5807F19D10C9BBBB9079B002B40F047
:1070A0009980A37A002B40F09780A27B02922278ED
:1070B000019201220092834C2A4651464846A0473D
:1070C00039B0BDEC028BBDE8F08F079B0233DBB219
:1070D0000593049BBAF80480B3F91210BAF90020A2
:1070E000B3F91030BAF90270BDF98860BDF98A00B1
:1070F00008F10108A8EB02087F1AD21AC71BB21ABE
:107100000FFA88F808FB0722059F02FB0752089236
:10711000BDF88C200132921B13FA86F396B212B29C
:107120009BB21192721EADF890301344ADF89430BA
:10713000BDF88E3001331B1A1BB211FA80F1179380
:10714000638809B2ADF89210ADF89610002B40F0AC
:1071500064822389B3F5807218BF012215920B9ABD
:10716000002A40F05C82B3F5807F40F058820C9B8F
:10717000002B40F05482A37A002B40F05082079BF2
:10718000002B00F04C82504D22A8A847B0F5F07FAC
:1071900024D822A8A84707464C4E7800B04708EEEE
:1071A000100A3846B047059B119A13FB08FA22EAE9
:1071B000E2724FF00008064643460492179A424591
:1071C0004DDD18EE102A06EB030C02EB430E0021F6
:1071D000089A14E003237BE7022379E74FF4F07762
:1071E000DAE790780CF8010B30B192F801B0107822
:1071F00000EB0B202EF81100059801310244119884
:107200008842EEDC049ABDF888101344089A524470
:107210000892BDF88C200132521A03FA82F2BA4267
:1072200008D2BDF89620013212B2ADF8962008F1CE
:107230000108C3E7A37B029323780193022318EE8E
:10724000102A00931F4D334624A94846A847BDF88D
:107250009620013212B2ADF892200023E5E7BDF985
:107260009630BDF992209A420FD0013BADF896308E
:10727000A37B0293237801930223009318EE102A34
:10728000104C334624A94846A0473046104CA0472E
:1072900018EE100AA04713E74FF4F0730A93C8E101
:1072A0000522DEE110931693199313E24FF0020BBF
:1072B00024E200BF15700000155200000DDC000034
:1072C0001D9A0000296A00009DE00000EDF000001A
:1072D000A1ED0000049BBDF98820B3F910301344E0
:1072E000BAF900209B1A1B9307EB080308EE903AAB
:1072F000069318EE103A03EB48031D93089B0D9379
:107300000023099A0E931A9B13441BB21E93119BE0
:107310000E9A934243DC1F9B98440B9B33B3049813
:10732000BDF88A20408ABDF88C30BDF888109D4D8C
:107330000244099802440498008A01335B1A01440C
:107340001BB218EE900A12B209B2A847002840F00A
:107350002381BDF88C10BDF888300131C91A18EEB0
:10736000900A914B09B298474FF0020B089B1C9A68
:1073700013440893BDF88C30BDF8882001339B1A64
:107380000A9A08FA83F3934280F01681BDF896308A
:107390000133ADF89630099B01330993C9E1159B80
:1073A000002B00F0D7800E9A1B9B1E992698134441
:1073B000BDF9A0201BB29B1ABDF9A2208A1ABDF804
:1073C000A610B1F5807FDDE92F6519D1DDE931E146
:1073D00001FB03FC51430EFB12CC0EFB031106EB29
:1073E000EC1605EBE113BDF99C200F93B2EB262FB1
:1073F0004FEA262318931BDC069A00231370B0E093
:10740000BDF8CE104B434A43BDF9A41011B91E4438
:10741000AB18E8E7DDE931E103FB01FC514302FB76
:107420001ECC03FB0E1106EBEC3605EBE133DAE77D
:107430003312002BE0DB0F9B0F991B121293BDF947
:107440009E30B3EB212FD7DD129B002BD4DB9DF8B0
:10745000CC5015F00401139166D0311202FB0312D7
:1074600015F0020F4FEA420351D110F812208DF8A7
:10747000AC20C1184A788DF8AD20022213929DF8F5
:10748000CC20D20704D5BDF8AC20B2F5FC6FB3D048
:107490009DF8AB209AB10F9AADF8D2203693189A86
:1074A000139BADF8D4208DF8DC30129A3F4BADF829
:1074B000D06026A8ADF8D620984700289CD0069A20
:1074C0009DF8AE301370BDF8AC30A27AD2B11699E7
:1074D0001498149DC3F3451202FB0012109803F098
:1074E0001F01D20801FB0501C1F3042102F4FC6273
:1074F0000A431999DB0A03FB0513C3F3072342EA86
:10750000C3239BB21D9A0E9922F8113029E013442F
:10751000C218C15C8DF8AC1051788DF8AD1092781E
:107520008DF8AE200322A9E7BDF96010BDF948200F
:10753000BDF8A8301E4D2CA8CDE92012A8471D4B40
:10754000ADF8AC00DDE920122CA89847139B8DF80C
:10755000AE0094E7079B7BB10D9B069A9B78137056
:107560006BB90E9B059A01330E930D9B13440D933B
:10757000069B01330693CAE6069AFF2313700D9B00
:107580005A781B7803EB02230C9A9BB2002A9CD0FA
:10759000B3F5FC6F99D12FE7022808BF4FF0020B1B
:1075A000E4E600BF8D99000051F2000011C4000014
:1075B000B5BF0000A5C00000A37B029323786B4DEC
:1075C000CDE900B318EE102A3B4624A94846A84747
:1075D000BDF8963001331BB2ADF89230ADF896305D
:1075E000079BA3B90C9B93B9638883B92389B3F52F
:1075F000807F14BF4FF0020B4FF0010B0B9B4BB180
:107600000A995B4B384698474FF00008C3E64FF0A5
:10761000020BF3E7DDF82C80BDE601231593554EF0
:1076200022A8B047B0F5F07F3FF636AE22A8B047AB
:107630000A900A9B504E5800B04708EE100A0A986C
:10764000B0474E4B0746482126A89847159B63B381
:10765000079B002B7FF424AE0C9B002B0CBF042255
:1076600006226388ADF8A4302389ADF8A630BAF8B5
:107670000630BAF80210269501335B1AADF89E3039
:10768000A388ADF8A030E388ADF8A230A389ADF8A7
:10769000A830E37BADF89C80C3F300038DF8AB30DA
:1076A00026A8374B8DF8AA209847A37ADA43D2B29E
:1076B0001492002B3FF4F6AD627BD2085A43199224
:1076C000A289C2F345125A431692227B02F01F028E
:1076D00053431093079B002B7FF4E8AD0C9B002BCA
:1076E0007FF4E4AD6388002B7FF4E0AD2389B3F52C
:1076F000807F14BF4FF0020B4FF0010B0B9B1BB1AF
:107700000A991B4B38469847049BBDF98A20B3F968
:1077100012301344BAF902209B1A1A93059B13FBEB
:1077200008F31C93002309939846119B23EAE37303
:107730001F93179B099A93423FF7CCADBDF9963042
:10774000BDF992209A420ED0013BADF89630A37B52
:1077500002932378054CCDE900B318EE102A3B467E
:1077600024A94846A047384690E500BF296A000092
:10777000ADF200009DE00000EDF0000051F20000CD
:1077800091C1000010B5084B044610219847002312
:10779000A381FF2323704FF480732381E37B43F0A5
:1077A0000103E37310BD00BF51F200000438C0B202
:1077B0000A289DBF024B1B1898780020704700BF15
:1077C0001C740200032805D0063804288CBF002052
:1077D00001207047012070470E289DBF47F6A47313
:1077E00023FA00F000F00100002070472DE9F04F6F
:1077F0002DED028B04468DB088461F4610464AB9CF
:10780000764B0093764B4D227649774D0220A84760
:10781000764A17E01B78052B69D9B989744B9847CC
:107820000546002800F0BC80037B826903F01F033B
:107830008AB1704B0093F7226F4B6A496A4E02205F
:10784000B047AA696D4B414620460DB0BDEC028B96
:10785000BDE8F04F18471846694A9047039018460C
:10786000684B98472B690490002B45D0664B08A8BD
:10787000214698477B88388913B9B0F5807F26D098
:10788000E288618826880132521AA1880131891B59
:107890003E1DCDE900061BB212B209B25B4E08A82C
:1078A000B0472288BDF82030BDF822101344ADF84F
:1078B000203063881944ADF82210BDF824100A4422
:1078C000ADF82420BDF826201344ADF82630504BE7
:1078D00008AA41460AA8984748B1049B0193039B14
:1078E000009320462A694B4C3B460AA9A0470DB09D
:1078F000BDEC028BBDE8F08F454B2246414606A801
:1079000098470028F3D0BDF81C60BDF81830013648
:10791000F61A33B2059303EB43003F4B98473A4BBB
:1079200006A9814608A898473C4B012108A898471A
:10793000BDF91830B4F90020BDF91AA0B4F902104D
:107940009B1A1BB208EE103AAAEB010BBDF91E30D0
:107950009A4503DD324B48469847C8E72C4B08AAA6
:1079600041460AA89847002835D0059B2D4ECDF8F2
:10797000009018EE101A0FFA8BF22846B047012833
:1079800013D02846284B184D9847284B00930220C7
:10799000194B14494FF49A72A847214B484698470F
:1079A000144B009358220E4B2EE7049B0193039B2C
:1079B0000093184E3B464A460AA908A8B047BDF8AE
:1079C00022300133ADF82230BDF826300133ADF856
:1079D00026300BF1010B0AF1010AB7E7CB73020065
:1079E000297402009773020021EB0000E373020088
:1079F000D1C60000EB73020035740200C56F0000B1
:107A0000C5770000D9770000157000008DC2000016
:107A1000B9E0000029700000EDF0000093E00000E4
:107A2000A1ED000059D2000079D20000FC730200E1
:107A300038B10078A0F120035F2B04D9C0094000C1
:107A400070470320704701207047A0F13003DBB27C
:107A5000092B0AD9602884BF2038C0B2A0F14103A5
:107A6000052B9ABF3738C3B2002318467047000071
:107A700010B5094B04461C219847FF232372074B7E
:107A800063604FF6FF73E38123824FF4F8132360A2
:107A90000023A37510BD00BF51F2000004000020B8
:107AA0002DE9F04F2DED048BD1B08A460A930023C7
:107AB0002193137A5E9C0590052B934640F2DB8060
:107AC000536808EE103A0A9B1B78002B00F0D38015
:107AD0000A469C4B014631A89847002800F0CB800D
:107AE0009BF817309F0700F1CB80059B059A9B8878
:107AF000128801339B1A1BB218EE102AB2F90860E3
:107B0000059ABBF90A50B2F900200B92059AB2F916
:107B10000200BBF912202492BBF914208718B9B2D5
:107B20003FB235440697002C00F0BC80002A40F09C
:107B3000BB80002880F2B980A268121A002AB8BF60
:107B40005242C5F50070B2EB400FC4BF4FF0FF3298
:107B500022602268002AC0F2A780049262680A4468
:107B600012B206921BB2049F0A98BBF90C2009EED0
:107B7000103A9BF817300093384419EE103A18EE7B
:107B8000101A714FB847049BC3180793069ABAF9A5
:107B900002109BF8173032448A420A9AC0F287805A
:107BA00004995E0702EB010040F1AB80079A009355
:107BB000511ABBF90C30654C18EE102A89B2A04757
:107BC000059B059A9B88128801339B1A1BB2181AD1
:107BD0000B9B00EBD07003EB600003B20B939BF8A0
:107BE00008302093BBF80E301093BBF8103011937F
:107BF000DDE91032934288BFCDE910239BF818309D
:107C000099071CD0524B35A89847BBF80030ADF807
:107C1000D430DBF80430B3F908300A22053393FB83
:107C2000F2F3ADF8D6309BF808309BF819208DF8A8
:107C3000DC309DF8DD3062F301038DF8DD30454B1B
:107C40003BA89847BBF80230ADF8EE30209B0B9C68
:107C5000FA2B88BFFF230993ABB22293BDF81830EB
:107C60001E9300231D93049A0A9B13441C930A9BA2
:107C70009B5C002B5ED151B0BDEC048BBDE8F08F56
:107C8000029347F618430193BBF90A300093DBF8DF
:107C90000420BBF90C300A992F4D3BA8A847BDF929
:107CA000EC3029E704945DE7002204925AE7079933
:107CB000009302EB010819EE103ABBF90C2018EE04
:107CC000101A4046B847079B1844069B2B441BB22A
:107CD000069374B113F5806F0BDB2368002B08DA71
:107CE000079B2360059B069AB3F90230D21AC4E9B8
:107CF0000123079B049398F80030002BBBD007901A
:107D000044E71C077FF56BAF079A04990093511A5B
:107D1000BBF90C300D4C18EE102A89B2A047059B18
:107D2000059A9B88128801339B1A1BB2181A0B9B69
:107D3000184452E7249B1C4423B20C930023309335
:107D40000893C2E0B9E00000FD0101005501010007
:107D50000D880000CD9D0000D5030100109A4FF65C
:107D6000FF739A4224D0119A9A4221D0049AA34BCD
:107D70000A981B681144984786B2A14C1C98236846
:107D800030A998471C9A2368054630980021104472
:107D900098479BF8173013F00103024600F0258145
:107DA000232D0FD1089929B9BDF8C0201D92C7E72E
:107DB0000026E2E7089B012B45D0022B40F01881FA
:107DC0000023BDE7089B012B40F00F81202D7CD1C3
:107DD000309B1D9A9B1A072B32D11C9B1D999A1818
:107DE00058589388ADF8E430864A3890C0F3074578
:107DF000C0F30764C0F30726C0B290470146F0B253
:107E0000904700EB0111E8B290470546E0B2904779
:107E100000EB05149DF8E400904705469DF8E50049
:107E2000904700EB0510C0F3C400C4F3850440EA9A
:107E30004410C1F3C40140EAC123219302237FE728
:107E4000BBF80030F9E70023BBF8004008936E4B05
:107E500018EE100A29469847109A1F904FF6FF73A4
:107E60009A4220D0119A9A421DD0109BB3421AD840
:107E7000B24218D90C9BADF8E030069BADF8E23069
:107E8000BBF80C300C9A013B13440344ADF8E430CA
:107E9000229B069A013B1344ADF8E6303BAA5B4BAC
:107EA000514638A898479BF819301B93209B042B08
:107EB00000F285841F9B43B1BBF80C300C9A1A4426
:107EC00013461F9A1A4413B20C93079B049A3099D5
:107ED0009B1A8B423FF642AF9BF818309D071FD587
:107EE0000B9BADF8CC30DBF80430494CB3F90830CB
:107EF00003EBD372BDF9D63003EBD3735B1003EB06
:107F000062031E9A13441BB20C9AADF8CE30ADF842
:107F1000E020ADF8E230524635AB38A933A8A0478F
:107F20009BF81830DC071ED50B9BADF8CC30BDF9A3
:107F3000D630DBF80420364C1189528903EBD37319
:107F40005B1001330B449B1A1E9A13441BB20C9A0C
:107F5000ADF8CE30ADF8E020ADF8E230524635ABAA
:107F600038A933A8A0470A9B079A2A4C9E189BF869
:107F70001730009318EE101A19EE103ABBF90C20C6
:107F80003046A047079BC518059BB3F900409BF8F6
:107F900017300146580740F1FD8318EE102A009370
:107FA0003046BBF90C301C4EB047059B059A9B88A8
:107FB000128801339B1A1BB2181A00EBD07004EB25
:107FC000600004B2229A069B13441BB206931E9BC8
:107FD00013449BB21E93079B069A0493BAF906308A
:107FE0009342FFF648AE07953DE6089B022B02D070
:107FF000BBF800402BE7219C29E700BF5800002078
:108000004C0000204B7A0000A1D30000199E000014
:1080100029880000FD01010055010100BDF8E420A0
:10802000BDF8E21052EA01033FF444AF0C98BDF9E9
:10803000E63003440D930D9F3944BAF9007018EEF1
:10804000100A18EE103AB942B0F90A60B3F90830D4
:10805000BDF9E800FFF62EAFBAF904100D9F8F426C
:108060003FF728AF06999B1B0B449B1A1B1A1A4417
:108070001693BAF902309A42FFF61CAFBAF90630ED
:10808000169A9A423FF716AF18EE100AA94B2946E6
:108090009847074628B9A84B009340F2B712A74B60
:1080A0009FE318EE103A1A7BBDF93460BDF9588091
:1080B0009DF8EA30920700F0FA8104F01F022A923C
:1080C000C4F345122692032BC4F3C422259200F078
:1080D000E680013B072B00F2D780DFE813F0DB00DE
:1080E0000800D500E000D500D500D500D000C023A1
:1080F0001393934B02241493BDF8E230179304FBBF
:1081000003F1BAF90030179DBDF8E420B342C6BFB1
:108110009B1B03EB430300231293BAF904300320A3
:10812000B5FBF0F030449842C5BF9B1B0133179B51
:1081300003EB43031993BAF902304345CCBFA3EBD9
:10814000080300230E93BAF9063002EB08009842A8
:10815000C2BFA3EB080301332393129B0E98D8BF31
:108160002392634300FB013307EBE30103F00703B2
:108170000F93179B734F1A915343B3F5F07FA8BF2A
:108180004FF4F07318461893B847189B05465800EB
:10819000B8476D4B08EE900A98476C4B9847B0F87B
:1081A0001490B0F910C0129BD0F808E0032209F136
:1081B000010993FBF2F1B0F912300E98A9EB0C090A
:1081C0000FFA89F9A8EB030309FB036309FB00100D
:1081D000A3EB0C0303440EEB43030D981593BDF87A
:1081E000343011FA80F1013BADF8CC10199991FBB4
:1081F000F2F21A44ADF8D020169B0E9A13441BB22B
:10820000ADF8CE30ADF8D230514B9847129A199B49
:1082100027909B1A1693179B1344199A9B1A634332
:10822000169A28936FF0020392FBF3F34B445B0022
:10823000299300231F46C4F108032D930E9B239A14
:10824000934231DBBDF9D230BDF9CE209A420FD036
:10825000013BADF8D2301B9B0293099B0193022393
:10826000009318EE902A3B4C2B4633A95046A0476A
:108270002846394CA04718EE900AA0471AE6FF237B
:1082800013930824354B36E7354B009340F27A229E
:10829000344BA6E2802313930124334B2BE7F023C6
:1082A00013930424314B26E70F9A139BDDF848E023
:1082B00023FA02FC3E460022199B73455CDC279B97
:1082C000CBB13B462B449846BDF8D030BDF9CC101D
:1082D000BDF9D220264F01335B1A1BB24046B84786
:1082E00048B9BDF8D010BDF8CC300131C91A09B277
:1082F000204B40469847169B189AF3189A4240F331
:10830000C180BDF8D23001331BB2289AADF8D2300B
:108310000F9B13441A9A02EBE30203F007031A922D
:108320000F93299A159B134415930E9B01330E93BB
:10833000374683E791D30000A1740200267602003D
:1083400012750200EDF00000155200000DDC000077
:108350001D9A0000296A0000A1ED000026750200A8
:10836000CE74020035760200107502001675020008
:108370008D99000051F200000F9BE3180D931A9B9A
:108380000D991B78C1F1080103EA0C03CB4007D01B
:108390000999FF2960D1082C1ABF1499CB5CDBB274
:1083A00002F5A07169440132032A01F8843C48D1E6
:1083B000159A9DF8BC305178259A9DF8BE90C3F16E
:1083C000FF00C90813FB02F200FB0122120A1792F8
:1083D000159A10782A9A00F01F00C9F1FF0819FBBE
:1083E00002F108FB00122B92159A9DF8BD8032F81D
:1083F000020B1592C0F345121146C8F1FF0243EA81
:1084000009032C92269A58EA030318FB02F018BFBE
:108410004FF0FF330A4608BF00232C99AB552B9B26
:1084200001FB0200C0F30520C3F30421179B41EABE
:10843000401141EAC32118EE903A002223F81610A9
:1084400001360F9B2D998B4214DA0D9B0F932CFA5A
:1084500004FC0EF1010E2FE7082C17BF149909999F
:10846000CB5C09990BBF4B4313FB01F3C3F3072309
:108470001B0A95E71A9BDDF84CC001331A930023C1
:108480000F93E6E71B9B0293099B01930223A74EE0
:10849000009318EE902A2B4633A95046B047BDF8FA
:1084A000D23001331BB2ADF8CE3000262DE7032BBE
:1084B00009EE904A00F0C080013B072B00F2B0802B
:1084C000DFE803F0B404AEBAAEAEAEA7C02213929A
:1084D000974A022504230E92099AF92A12D8954A3E
:1084E000099892F80011814240F0AC80D2F8042142
:1084F000AA4240F0A7808F4B099A83F80021C3F865
:1085000004510E93BAF90030BDF8E290BDF8E420B2
:10851000B342CCBF9B1B00230F93BAF9043009EB85
:1085200006009842C4BF9B1B0133BAF90260C8BF62
:108530001293BAF90630D8BFCDF8489002EB080084
:108540004645CCBFA6EB080600269842C2BFA3EB67
:108550000803013317930F9BD8BF179205FB09F14E
:1085600003FB05F406FB014407EBD403149302FB61
:1085700009F3B3F5F07FA8BF4FF4F07315931846D5
:108580006D4B98470D9A0F99BDF8343011FA82F26D
:10859000ADF8CC20129A013B1344ADF8D030169BB5
:1085A00033441BB2ADF8CE30ADF8D230634B08EE99
:1085B000900A9847C5F108030D930F9B19909944B1
:1085C000129BA9EB030905FB09F304F007041A93B6
:1085D0004FF00009179B9E4245DBBDF9D230BDF933
:1085E000CE209A4210D0013BADF8D2301B9B0293B3
:1085F000FF260223CDE9003619EE902A18EE903AB4
:108600004F4C33A95046A04718EE900A4D4B98475F
:1086100050E4FF22139208254B4A4FF480735AE727
:108620004A4B009340F2E512494BDAE08022139264
:108630000125484A02234EE7F02213920425464AB8
:10864000102348E70E993B480B4411F8012BFF2AF1
:1086500017BF099C099A12FB04F2120A994200F80A
:10866000012BF2D147E7139B0F99CDF88C9023FA99
:1086700004F218EE903A03EB09084746129B8B422E
:108680003ADC0F9A12999B1A16938A42C8BF0023AC
:1086900018939944199BB3B1BDF8D030BDF9CC10F3
:1086A000BDF9D2202D4F01335B1A1BB24046B847AB
:1086B00048B9BDF8D010BDF8CC300131C91A09B2A3
:1086C000274B40469847189B169A13449846239B7D
:1086D0009844159B434545D9BDF8D23001331BB2B0
:1086E000ADF8D2301A9B1C44149B03EBD4031493B3
:1086F00004F0070401366DE7149B0D981B78A0EB7E
:10870000040C134033FA0CF31CBF0E98C35C07F83B
:10871000013B0D9BA3429DBF149B139A0133641927
:108720008EBFEA40149300240131A7E7296A0000B4
:1087300012750200648E0020EDF000001D9A00000A
:108740001D640000A1ED000026750200F474020013
:108750004776020010750200167502008D99000020
:1087600051F200001B9B0293FF270223CDE9003743
:1087700019EE902A18EE903ADFF88C8033A9504613
:10878000C047BDF8D23001331BB2ADF8CE304FF048
:108790000009A5E71A077FF515AC18EE102A00931B
:1087A0003046BBF90C30124EB047059B059A9B88AA
:1087B000128801339B1A1BB2181A204401E418EEE8
:1087C000100A0C4E00232A4638A9B04700287FF42F
:1087D00025AC1F2D7FF66EAB074B0093074B40F285
:1087E000A1120749074C0220A047FFF763BB00BF57
:1087F0005501010095D300007C740200267602002A
:108800004674020021EB00001D64000010B5054B0A
:1088100004460A219847FF23237200232380012363
:10882000638010BD51F200002DE9F04F2DED048B57
:108830009B46B3F90230C7B0CDE9050108EE902A96
:10884000002B00F0E4809BF80820052A40F2DF802E
:10885000059AB0F90040B1F90000B2F90210069A89
:108860008442B2F9022002D1914200F0D08003EBA1
:10887000D373C3F34F038442D4BFC3EB0405C3EBEC
:108880000005ADF828508442ACBF1D191D18914257
:10889000D4BFC3EB0100C3EB02009142ACBF5B1835
:1088A0009B180AA9ADF82A0018EE902AAA4CADF838
:1088B0002C500846ADF82E30A047002800F0A780C5
:1088C000059BB3F90290069BB3F90280C14540F0C5
:1088D0005981A24B9BF808409847A14B9847BBF998
:1088E0000230BBF90650013B03F0010680465F10E1
:1088F00006EB630625B1BBF90450003D18BF012506
:10890000984B9847002840F0878085F00102069B2D
:108910000599B3F90030B1F900108B421846A8BF91
:1089200008468B42B8BF0B46013BADF89C30059B17
:10893000ADF898005B889E1B3B44ADF89A60ADF89B
:108940009E30002A6AD09BF8093003F00303CDE97A
:10895000014301230093BBF80020834C002326A988
:108960000AA8A0479BF8093013F00C0F4FD07F4B9B
:1089700031A89847BBF80030ADF8C63047F6FF7312
:10898000ADF8C4309BF80830BBF902508DF8D030F8
:108990009BF809306C105A076FEA050505F00105D0
:1089A00018D5059B1A88A3B2D11AADF8981005996D
:1089B00049881A44C81A0B44521B5B1BADF89A0035
:1089C000ADF89C20ADF89E3018EE901A684B31AA95
:1089D00026A898479BF809301B0718D5069B1A88CC
:1089E000A3B2D11AADF89810069949881A44C81A4A
:1089F0000B44521B5B1BADF89A00ADF89C20ADF800
:108A00009E3018EE901A5A4B31AA26A8984747B0C4
:108A1000BDEC048BBDE8F08F002278E726AA4E4B10
:108A20000AA91046984700289CD0B8F812E0BDF972
:108A30009A10B8F81020B8F91060BDF89800BDF988
:108A40009C70BDF998C0ADF8C4C0A1EB0E04ADF8A0
:108A50009A40BDF89C40ADF8C870831AA21AADF8D0
:108A60009C20BDF89E20ADF8C61001341BB2A2EBCD
:108A70000E02241AADF89830ADF89E2024B2ADF85D
:108A8000CA10DDB11E44BBF90420BBF90630134403
:108A900096FBF3F203FB126633B20793354BDFF814
:108AA000C8A020469847BDF99A900746BDF99E3068
:108AB000994505DD3846304B984753E70795EDE774
:108AC0002E4B2F4E214638469847BDF89830B8F8BF
:108AD0001220B8F810104A44194412B2234609B2C1
:108AE0003846B047024695B188B100230799184629
:108AF0000AE0BBF904208A4225DB13445B1A1BB24F
:108B0000013301321BB211B29C42F2DC02229BF80B
:108B1000093003F0030302939BF8083031A9CDE933
:108B200000230AA83B46BBF80020D047BDF8C6305A
:108B30000133ADF8C630BDF8CA300133ADF8CA30E4
:108B400009F10109B2E7BBF906C062449142BABF1C
:108B5000F8540A460022D3E7B9E00000155200009D
:108B60000DDC00001D9A00001D640000CD9D00007A
:108B7000199E0000EDF00000A1ED0000ADF2000034
:108B80008D990000059BB3F90070069BB3F9006056
:108B9000B74240F0DB80664B9BF808609847654B16
:108BA0009847BBF90230BBF90650013B03F00108BE
:108BB00007464FEA630908EB630825B1BBF9045087
:108BC000003D18BF01255C4B984720BB85F0010292
:108BD000059B05991B88B1F90210A3EB08084B44CB
:108BE000ADF89C30069BADF89880B3F902308B420B
:108BF0001846A8BF08468B42B8BF0B46013BADF8EC
:108C00009A00ADF89E3042B19BF8093003F003039F
:108C1000CDE901639DE60022DAE726AA0AA91046FB
:108C2000A04700283FF49EAE3B8ABDF89840B7F8B5
:108C300012C0BDF99800BDF89C60ADF8C400E21AFE
:108C4000ADF89820BDF99A20ADF8C620A2EB0C0132
:108C5000F31AADF89A10BDF99C10ADF89C30BDF830
:108C60009E30ADF8C8100136A3EB0C03361BADF8EF
:108C70009E3033B2184608EE103AADF8CA202F4B9A
:108C800098478046C5B1BDF99830B7F91040BBF997
:108C900004201C44BBF90630134494FBF3F203FB9D
:108CA000124424B2BDF99A90DFF89CA0BDF99E3021
:108CB000994503DD4046FEE62C46F3E718EE101A10
:108CC0001F4B204E40469847BDF898307A8A398A23
:108CD0004A44194412B218EE103A09B24046B0475D
:108CE0006DB150B1BBF90420BBF906301344A24268
:108CF000B8BF00209C42A8BF0024013424B2002346
:108D000002939BF80830BBF80020CDE9000331A99D
:108D100043460AA8D047BDF8C6300133ADF8C63087
:108D2000BDF8CA300133ADF8CA3009F10109BDE719
:108D3000155200000DDC00001D9A0000EDF000004F
:108D4000ADF200008D9900001D640000C14505DBF7
:108D50004B46C14698463B4637461E46F31B099391
:108D6000A8EB09030893F31B83EAE372A2EBE37217
:108D7000089B079283EAE37AAAEBE37A524513460B
:108D8000D8BF079BBBF90250CABF4FEA4A135B0129
:108D9000B3FBF2F3B34AD8BFB3FBFAF3D25C3F2381
:108DA00015FB0235C5F3CF13BE42D4BFC3EB060299
:108DB000C3EB0702ADF83020BE42ACBF9A19DA19F6
:108DC000ADF834200CA9C845D4BFC3EB0802C3EBEF
:108DD0000902C845ACBF43444B44ADF83220ADF85E
:108DE00036300AAAA04B0846EC11984700283FF4F9
:108DF000B9AD079B04F0010404EB25245345A4B24C
:108E0000C5F30F2540F3ED8014FA89F31BB208EE89
:108E1000103AF31BA9EB050A14FA88F4A8EB050530
:108E2000002B4FF0000324B20FFA8AFA2DB20193FF
:108E300040F3C680009533465246394610A88B4D04
:108E4000A8470123CDE9004318EE102A33463946DE
:108E50001BA8A847DFF840A2002110A8D047002196
:108E600009EE100A1BA8D0479BF8095015F0100511
:108E700009EE900A40F0CF800322BDF82040019215
:108E8000F21BBDF82430079319FA82F23B1B12B291
:108E900039460092754F1BB24A4626A8B8470222AF
:108EA0000192079A424412B2331B1BB20092314620
:108EB000424631A8B847294626A8D04729460990F6
:108EC00031A8D04782466A4B6A4E98476A4B98470A
:108ED000BDF83020038ABDF83440D11AE31AADF84A
:108EE0003010ADF83430418ABDF836300546BDF853
:108EF00032000134401A5B1AA41AADF83200ADF802
:108F000036300CA823B20793B047B0F5F07F80F05D
:108F100087800CA8B0470746584B384698472B8A9D
:108F2000BDF830201A4412B20892ADF83820BDF8CE
:108F300034201344ADF83C306A8ABDF83230134413
:108F40001BB2ADF83A30ADF83E3039464C4B0646D0
:108F50009847BDF93280B5F912304FF000099844B6
:108F6000BDF93630B5F91220134498455BDDBDF9E3
:108F70003E30BDF93A209A4213D0013BADF83E3065
:108F80009BF80930BBF800203E4C03F0030302932A
:108F90009BF808300193022300930AA933460EA8D8
:108FA000A047394B394C3046984719EE100AA04774
:108FB00019EE900AA0470998A0475046A047D1E46F
:108FC00018EE102A009433463946284C10A8A047C2
:108FD0000123CDE900535246334639461BA8A0472A
:108FE00038E714FA86F3002214FA87F421B2CDE9A7
:108FF00000821BB24A461D4C10A8A0471FFA86FAF1
:10900000BAB2511BAAEB05030122CDE900821BB2C3
:109010004A4609B2E2E74FF0FF3ACDF824A052E702
:109020004FF4F07778E706EB090308EE103A089959
:10903000079B174C18EE100A0FFA88F2A04720B9C8
:109040000799144B18EE100A9847079B99444B4414
:109050009F4223D9BDF83E300133ADF83E3008F1D0
:1090600001087DE762760200B9E00000399A00004D
:10907000155200009DE000000DDC0000EDF0000046
:10908000ADF200001D640000A1ED0000CD990000CC
:109090008D99000051F200003D9900009BF80930C5
:1090A000BBF800200D4C03F0030302939BF808303B
:1090B0000193022300930AA933460EA8A047BDF8E6
:1090C0003E3001331BB2ADF83A30ADF83E30394690
:1090D000034B304698474FF00009C0E71D6400007D
:1090E000ADF20000F9290AD8052907D910FB01F0D3
:1090F00048F281035843C0F3C750704700207047BF
:109100002DE9F047089E1C46B38AD21A738AC91A01
:109110000FB296F82830316A054612B203F001000A
:1091200099BB337C03F0020680B13EB103F0030328
:10913000022B05D10132ACBF00200120BDE8F08731
:10914000032B01D1002AF9DC0020F7E7002E40F0C4
:10915000878103F0030001280AD1002FEEDCE742EB
:10916000F2D4002F00F37E8179428C42ECDD9BE04B
:109170000028F4D1391900F17381002FE4DC784222
:10918000A042C0F29C800220D8E703F0020C002825
:1091900000F09780F16907FB01F300294FEAA32350
:1091A0005FFA8CF005DD9A4205DA003818BF01201D
:1091B000C4E79A42F9DC3B194B4300294FEAA32349
:1091C00005DD9A4206DDB0FA80F04009B6E79A4222
:1091D000F9DB0132B36912025A439212111212F0F2
:1091E000FF021FBF736AC2F1FF0803FB08F84FEAD2
:1091F000282814BFC8F1FF084FF0FF08CF1B002A32
:1092000054D0002F0FDBBC420DDDC2F1FF01C8F1CD
:10921000FF035943C1F3472108B9C943C9B2E85D07
:10922000A34B9847E8557A1CDFF88492716A96F848
:109230002830884503F0020318DC944229DD002A17
:1092400027DBB169F06901FB08F1891208FB01F124
:10925000C1F347210028BCBFC943C9B20BB1C94300
:10926000C9B2A85C924B9847A85412E0002A0ADBC6
:10927000944208DDA8EB6101C9B20BB1C943C9B280
:10928000A85CC847A854736A01329442A8EB03084B
:10929000CCDC96F8283099070AD5BC42FFF654AFCB
:1092A000002FFFF670AF3946284683E03A46BBE709
:1092B000501C3FF549AF8442FFF665AF211A2844A0
:1092C00078E0B16901FB02F300294FEAA323CCBF88
:1092D00003F1010E9E4677455FFA8CF03FF765AFCC
:1092E00007EB040C63453FF76EAF4FEA022C0132E7
:1092F00012024A4301FB0CFC4FEAA249B9EBAC4F06
:10930000CCF38723C7EBAC4A00F0AE8000295ADAD1
:109310000AF1FF38002B00F0C980F26952425A432B
:10932000BAF1000F4FEAA2220DDB54450BDD534387
:10933000C3F3472108B1C943C9B215F80A005C4B11
:10934000984705F80A00B8F1000F17DB444515DD12
:10935000B36915F80800C2F1FF025942514396F86B
:109360002830891251439F07C1F3472158BFC94391
:109370004F4B58BFC9B2984705F8080096F82830F7
:109380009E071AD54445FFF6FEAEB8F1000F7FF7F1
:10939000FAAE414688E708F10108A045A8BFA046FB
:1093A000B8F1000F3FF4D0AE7FF7EDAEA4EB0801AB
:1093B00005EB08003F4B9847E5E60AF101008442BF
:1093C0004EDB002878E7F769C3F1FF035F43BAF18A
:1093D000000F4FEAA7270DDB54450BDD7B43C3F39A
:1093E000472108B9C943C9B215F80A00304B98475C
:1093F00005F80A001AF1010215D4944213DDB3698D
:10940000C7F1FF0703FB07F1891296F8283079436B
:109410009807C1F3472148BFC943A85C244B48BF04
:10942000C9B29847A85496F828309B0708D55445E8
:10943000FFF68AAEBAF1000FFFF6A5AE514633E74C
:109440000AF1020AA245A8BFA246BAF1000F3FF4F2
:109450007BAE7FF798AEA4EB0A0105EB0A00A9E703
:1094600001206BE6002C81E6D046B8F1000F0FDB3F
:1094700044450DDDC2F387211944C1F3470108B10A
:10948000C943C9B215F80800094B984705F8080008
:1094900096F828309B077FF57EAFA9EB07018C4239
:1094A0007FF752AE0029FFF66EAEFDE6FF23DCE744
:1094B000E590000051F20000013900F1080311F8B5
:1094C000012F00F8012B9842F9D170472DE9F04F98
:1094D0008DB01D46DDF8588098F81290B8F910A0AC
:1094E0000023CDE9023306468B4B8B460AA808F1D0
:1094F000080109F0010917469847BDF92A30B9F16A
:10950000000F3AD1BB4201DD002039E0BDF92E2029
:10951000BA42F9DBBDF9281001EB0A029345A1EB31
:109520000B0407DBBDF92C2005EB0B00A2EB0A02B4
:10953000904209DD03EB0A029742BDF92E003DDBA4
:10954000A0EB0A02974239DCB9F1000F25D1A54200
:10955000DADB002C03DB714B214630469847BDF91E
:109560002C00A0EB0B0001300028CDDDA8420FDA63
:10957000291A3044694B98470DE0BB4203DD0120B6
:109580000DB0BDE8F08FBDF92E20BA42C2DAF6E781
:109590000CB9A842F3D00220F2E724EAE470A84212
:1095A000F9DCBDF92C10A1EB0B01091A01314318AC
:1095B000AB4200DD291A0029EDDBDAE7BDF82C20EB
:1095C0009BB20130C01AFF1A0132B8F91030521A9A
:1095D0003FB212B25B43BA45049200B2019300F36A
:1095E0009081A0EB0A039F42D5DBC01BD8F8143052
:1095F000BAF5807FAAEB0000D4BF4FF400624FF4AD
:109600000042984200F1010767D0019B059200FBE0
:10961000103007A9424B9847059A61E0D8F81830F6
:109620000693019B059207F1FF3B0BFB1B3007A93B
:109630003B4B9847BDF81E30A8F81A30BDF81C30D7
:10964000C8F814B0BDF81C10A8F81830BDF81830D0
:10965000059A01398B4207D1BDF81E1021B9FF21AF
:10966000ADF81C30ADF81E10BDF81C1099425BD14E
:10967000BDF81A10BDF81E201144C1F34701B9F11D
:10968000000F01D0C943C9B2AAEB03035A1EA718A1
:1096900005D4AF4203DAF05D224B9847F055049BA6
:1096A0009A1A501E041905D4AC4203DA305D1D4BE2
:1096B00098473055B9F1000F22D1AF423FF724AFA0
:1096C000002F03DB154B394630469847601C3FF5A9
:1096D0001BAFA8423FF75FAF4AE7D8F818300793AF
:1096E000019B059207FB173006A90D4B9847BDF863
:1096F0001A30A8F81A30C8F81470BDF81830A1E76D
:10970000781C20EAE070AC42D4BF211A291AA84282
:10971000BFF641AF4FE700BFB994000051F200001F
:10972000CDEB0000E590000004990133AAEB0303A0
:1097300004EB0308CB1A013B1C44B9F1000F10D015
:1097400008F1010020EAE070A542ACBF211A291AF5
:10975000A84206DA002904DB754B0492304498478E
:10976000049ABDF818B0019B049208A90BFB1B30AA
:10977000704B9847BDF822106E4B049A0BF1010A0A
:1097800039B9BDF820100139ADF82010FF21ADF82E
:109790002210BDF82010B9422EDB019809A90AFB5E
:1097A0001A009847BDF82620BDF81A10C2F1FF0331
:1097B000C1F1FF015943C1F34721B9F1000F01D1B4
:1097C000C943C9B2B8F1000F07DB454505DD16F8FE
:1097D0000800594B984706F80800002C05DBA54205
:1097E00003DD305D544B9847305508F1FF380134A4
:1097F000ADF822200BF1020ABDF82020BDF81CB004
:10980000BDF822104C4F12010023D34542D23BB188
:10981000029BADF82630039BADF82430ADF8221042
:10982000BDF82230FBB1BDF81E105943C1F34721EA
:10983000B9F1000F01D0C943C9B2B8F1000F07DB7D
:10984000454505DD16F808003B4B984706F808002B
:10985000002C05DBA54203DD305D374B98473055C2
:1098600008F1FF380134B9F1000F7FF494AE08F12C
:1098700001018D42FFF648AE002902DB2C4B304639
:109880009847002CFFF640AEA5427FF784AE291B17
:1098900030196FE6019BC1F30F1010440AFB1A3C0C
:1098A00000FB00F3C3EB0C234FEA400C93FBFCF3EB
:1098B0000344C3F30F101B0103F0F003194403909A
:1098C0000293C1F34701B9F1000F01D0C943C9B2F6
:1098D000B8F1000F06DB454504DD16F80800B8476F
:1098E00006F80800002C04DBA54202DD305DB84715
:1098F0003055029908F1FF3801340AF1010A0123B9
:1099000083E7D8F81430BAF5807FAAEB0707D4BFF5
:109910004FF400624FF40042BB423FF47FAE019B24
:10992000059207FB173006A9024B9847059A78E67F
:1099300051F20000CDEB0000E590000073B50E4C35
:10994000002354F83360DAB204EBC30576B1013377
:10995000102BF6D1094B00930220094B09490A4C00
:109960005722A0474FF0FF3002B070BD44F83300DB
:10997000696010B2F8E700BF90900020B87602004E
:10998000DE7602008376020021EB00002DE9F3472A
:109990000D4E0746884691469A460024356825B9FB
:1099A0000134E0B202B0BDE8F08700952D6853465F
:1099B0004A4641463846A8470028F3D0022808BF47
:1099C00001240836EAE700BF90900020431C18BF2E
:1099D000074B4FF000021DBF53F8301043F8302002
:1099E00003EBC003114618BF5A600846704700BF1A
:1099F000909000200022084B30B5114614465D6857
:109A00000132854204BF1968C3E90044102A03F1FA
:109A10000803F4D1084630BD909000200023054A89
:109A2000184652F8331009B10130C0B20133102B7F
:109A3000F7D17047909000202DE9F041BDF91880D2
:109A400015460E461F462C213B4B0446984745457C
:109A500005DD2B464546984633463E461F46237C49
:109A60009DF81C20658162F301032374A8EB0502B5
:109A7000BB1B83EAE37082EAE271A0EBE370A1EB27
:109A8000E271884294F82810A582D4BF00200120FA
:109A900060F30001294D84F828100020C907C4E9AB
:109AA00006002681A781A4F80E80668225602071B9
:109AB0002BD533B14FF4801191FBF3F1514389124F
:109AC000E16132B14FF4801191FBF2F253439B12EA
:109AD000A361E269237C226213F0030307D0012B08
:109AE00005D0022B23D1002AD4BF0023012394F8F0
:109AF0002810002A63F341014FEAA203B8BF5B427A
:109B000084F828106362BDE8F08132B14FF480110F
:109B100091FBF2F159438912A16133B14FF48011E5
:109B200091FBF3F353439B12E361A269D2E7002A4E
:109B3000CCBF00230123DAE751F2000001910000BD
:109B4000F8B50446C8888D881F464B880130C01A76
:109B50000B880135ED1A00B22DB2A842A8BF2846E5
:109B6000B2EB600F4FEA6003164604F10800C8BF6D
:109B70001EB2084B9847A37C268267F30003A374A8
:109B8000054B2360022323714FF000420023C4E9F8
:109B90000523F8BDB9940000CD94000070B5B0F96C
:109BA000084004FB01F3B2EB232F4FEA232501DC2D
:109BB000408870BDB0F90A3001FB03F6B2EB262FE6
:109BC00001DB8088F5E71B1B5943521B0B1212B2B5
:109BD00041880679C2EB022292FBF3F38288DBB262
:109BE000C3F1FF05C1F34511C2F34512694303FBFD
:109BF0000211827802F01F0206F01F066A4348F243
:109C0000810403FB062261436243C1F3C551C2F3E1
:109C1000C45242EA4112C1784679C908F60869433C
:109C200003FB06136343DB0D42EAC320C1E70000D8
:109C30002DE9F04F45004FEA610987B0CB07044694
:109C40005A4B28460E461746CA4658BF09F1FF3AF6
:109C50009847AB1E00934FEA490301936FF001034D
:109C60000AFB03330146B8464FF0000B02935C45F4
:109C700022DC3B8893FBF6F304FB04F83B803A4676
:109C80003B464FF0010CC44541D36B4209FB03F343
:109C90000393631E05FB037302930AF1010301930F
:109CA0000AFB055A4FF0000C64453EDC404B084669
:109CB00007B0BDE8F04F1847009B019838F8032023
:109CC00000EB080C02987243631E404421F81320F5
:109CD00003EB090E7445CCBF3CF813E04FF0000EC7
:109CE000A2EB0E0EA3EB0A02002AD4BFB8F80020A4
:109CF00030F81320013B7244E8D240462D4B0391CB
:109D00002A469847A84403990BF1010BAFE75888FE
:109D100033F802EB70451CBF90FBF6F01FFA80FE93
:109D2000A3F800E00CF1010CADE7039813881018BC
:109D30007343059000270AEB0200049096460093B7
:109D400090463846009B002BACBFC3F38F1B4FF0EF
:109D5000000B21F810B0A0EB090BBBF1000FCABF3C
:109D6000059BB8F800B033F807B0009BA3EB0B0BD2
:109D7000019B03449C42CBBF049B029BDB5B33F8FB
:109D80001C3001305B4484420093A8442F44D9DC4A
:109D9000002331F81300AEF8000001339C42AE44BA
:109DA000F7DC0CF1010C02327EE700BFEDF00000A1
:109DB000A1ED000069EE0000013900F1080311F87F
:109DC000012F00F8012B9842F9D1704710B50F4BC5
:109DD0005421044698470E4B1B8863800022FF23C2
:109DE000A280E281A4F84620E28363812373237773
:109DF0002375A28684F83630064A84F8443084F805
:109E000028300F2322632264638210BD51F20000C8
:109E100070770200040000202DE9F04F9246C288BE
:109E20004588531C2DED048B5B1B1BB2002BADB082
:109E30008346884641F36E81818800884B1C1B1A3B
:109E40001BB2002B41F36681BAF92040002C00F0D0
:109E500042859AF828300893052B40F23C85DAF8C1
:109E60002070BAF92460BAF92630012F03D116B94F
:109E7000002B40F33085BAF822709BB2A7EB030C9D
:109E8000B6B21F443944F71A33441A4404EBD4736E
:109E90005B105B4292B25E1E89B2C3F10103ADF862
:109EA000441011FA83F112FA83F3ADF84E30089B97
:109EB000ADF8462060443D44FB2BADB280B228BFD4
:109EC000FF23ADF8400010FA86F015FA86F6ADF8DB
:109ED0004C10ADF842500893ADF84800AC4BADF8CB
:109EE0004A609847AB4B9847AB4B0546424612A990
:109EF00014A89847002800F0EE84298ABDF8503055
:109F00006A8A5B1AADF85030BDF852309B1AADF832
:109F10005230BDF854305B1AADF85430BDF85630AD
:109F20009B1AADF8563059469C4B16A89847BDF879
:109F30005850BDF85A00BDF85C20BDF85E10BDF861
:109F4000447001350130ADB280B2531EADF85C30C3
:109F5000521B4B1E091A12B209B28A42A8BF0A4606
:109F6000ADF85E30BAF90030BDF84210ADF85A00D5
:109F700052109A42A8BF1A4608EE902ABDF8402017
:109F8000ADF858500137BF1ABDF84620844D013254
:109F9000521A12B23FB29742A8BF17467F109F4293
:109FA000A8BF1F4604EB070909FB09F04000A847BA
:109FB000BAF92040794B069010A91EA8984704F0E2
:109FC000010204EBD473BDF840100A92C3F34F03AF
:109FD00064F00102BDF844001A443A440139091AF8
:109FE00092B2ADF87C200A44ADF87820BDF8462046
:109FF000BDF8421001330132521A9BB2ADF87A30EB
:10A0000013443E193A46ADF87E30664F00231EA930
:10A0100025A8B847012C304618BF6410A847730024
:10A020000993069B05930023079333B208EE103A79
:10A030000746079B9E4208DC5B4B38469847012C3D
:10A0400006FB06F574D100233EE0584B31463846F6
:10A05000984725AB0093BDF91C20259D18EE103ABA
:10A0600000213846A84758B909990598504B984798
:10A07000099B059A1A44079B059201330793D8E779
:10A080003B78059A05989B0193FBF4F322F8023B79
:10A09000099B394618188242EAD08C4611F8013FD4
:10A0A0009CF800C09C4517BF9B0132F8023C93FB13
:10A0B000F4F39BB222F8023BEDE7069A069932F8D8
:10A0C00013209209CA540133AB42F6D1BDF84E3089
:10A0D000BDF84A2001339B1AC3F3C03101FA83F360
:10A0E00002EB63039AB21BB20993BDF84C300B929A
:10A0F000BDF8482001339B1AC3F3C03101FA83F342
:10A1000002EB63039AB21BB20A932A4B0C92984754
:10A1100000283BD1BAF92230002B4FD1BAF92420C4
:10A1200022B9BAF92630B3FA83F35B09079346E004
:10A1300030B22146069A204F0590B8470A9921442B
:10A1400001290CDD069B069A1B8805989B010124BA
:10A15000B3FBF1F31380AC4203D3069AB847002354
:10A1600011E0538832F8026BB3421EBF9B01B3FB70
:10A17000F1F39EB216800134EDE7069A069932F8A3
:10A180001320CA540133AB42F7D19FE70023CDE738
:10A19000155200000DDC0000B9E00000B99D000080
:10A1A000EDF00000419B0000A1ED0000ADF20000C9
:10A1B00051F200001D9A0000319C00000790BDF88C
:10A1C0004C00BDF84830B24D0130C01A00B2B14B5E
:10A1D000984718EE902A012316A908EE100A25A820
:10A1E000A847AD4B002125A89847BDF94C30ADF8E4
:10A1F00064301FFA89F201339B1AADF86030BDF963
:10A200004A30ADF86230013B134408EE900A0592E3
:10A21000ADF866304246A14B18A91AA89847002805
:10A2200039D0BDF96E30099ABDF86C609342C4BF55
:10A230001346ADF86E300A9ABDF968309342D8BF24
:10A240000C9BBDF96A20DCBF0133ADF86830BDF965
:10A250006850BDF96E300136761B36B2002E1ADD1D
:10A2600001339B1A1BB20D93BDF96230D21ABDF9AE
:10A270006030ED1A069B09FB02551D441AA9884B54
:10A280001EA89847BDF97A300027ADF87E300D9BA7
:10A290009F42C0F2A380BDF94C30059AADF86430FE
:10A2A00001339B1ABDF94E200599ADF86030531C5F
:10A2B0005B1AADF86230ADF86620784B424618A9BB
:10A2C0001AA8984700283AD0BDF96A30099ABDF813
:10A2D0006C609342D8BF0B9B0A9ADCBF0133ADF888
:10A2E0006A30BDF96830BDF96A109342D8BF0C9B43
:10A2F000BDF96E20DCBF0133ADF86830BDF96850A0
:10A300000136761B36B2002E19DD531C5B1A1BB2C8
:10A310000C93BDF966309B1ABDF96020AD1A09FB9C
:10A320000355069B1AA91D441EA85D4B9847BDF80E
:10A330007E30ADF87A3000270C9B9F427ADBBDF966
:10A340004C30059AADF8643001339B1AADF860309B
:10A35000BDF84A301344ADF86230BDF84E309B1A58
:10A36000ADF8663042464D4B18A91AA8984780B3FD
:10A37000079B43B1BBF90430BDF968209342B8BFD5
:10A380001346ADF86830BDF86C50BDF96860013512
:10A39000AD1B2DB2002D1CDDBDF86E30BDF86A205E
:10A3A00001339B1ABDF960201BB20C93B61A09F158
:10A3B000FF3309FB0366069B1AA91E441EA8384BEF
:10A3C0009847BDF97A300027ADF87E300C9B9F424C
:10A3D0006EDB069A4FEA69060020A3E02946314B5E
:10A3E000314C324618EE100A9847BDF97A20BDF973
:10A3F0007810334618EE100AA0479AF829300293D5
:10A400000128089B294C08BF0220CDE900031EA9A2
:10A4100018EE103ABAF81E204046A047BDF87A3030
:10A420000133ADF87A30BDF87E3001331BB24D44B4
:10A4300001372AE729461B4B1B4C324618EE100AFF
:10A440009847BDF97A20BDF97810334618EE100A06
:10A45000A0479AF8293002930128089B134C08BFA3
:10A460000220CDE900031EA918EE103ABAF81E200A
:10A470004046A047BDF87A30013BADF87A30BDF8D0
:10A480007E30013BADF87E304D44013754E700BFCC
:10A49000419B0000EDF000003D990000B9E0000094
:10A4A000B99D000069EE00008D9900001D64000058
:10A4B000204B18EE100A2A4631469847079B53B99D
:10A4C000BDF97A20BDF978101B4C18EE100A2B4606
:10A4D000A047012800D102209AF8293002939AF867
:10A4E0002830164CCDE900031EA918EE103ABAF830
:10A4F0001E204046A047BDF87A300133ADF87A30CF
:10A50000BDF87E3001331BB201375DE711F8017FE2
:10A5100013F801CD81F800C01F70EF1ABE42F5DCC0
:10A520004A44013081450BDD09EB0205511E2B46E3
:10A53000F3E700BF69EE00008D9900001D64000084
:10A54000BDF94830059AADF86030013B1344ADF8D1
:10A550006430BDF94A30ADF86230013B1344ADF8C8
:10A5600066304246B84B18A91AA89847002837D039
:10A57000BDF96E30099ABDF968509342C4BF1346C5
:10A58000ADF86E300A9ABDF96C309342C4BF1346E1
:10A59000ADF86C30BDF86C60BDF96E30BDF96A2065
:10A5A0000136761B36B2002E1ADD01339B1A1BB220
:10A5B0000C93BDF96230D21ABDF96030ED1A069BDA
:10A5C00009FB02551D441AA9A04B1EA89847BDF9C6
:10A5D0007A300027ADF87E300C9B9F42C0F29F85F9
:10A5E000BDF94830059AADF86030013B1344BDF920
:10A5F0004E200599ADF86430531C5B1AADF86230FB
:10A60000ADF86620904B424618A91AA89847002832
:10A6100039D0BDF96A30099ABDF968509342D8BF64
:10A620000B9B0A9ADCBF0133ADF86A30BDF96C3080
:10A63000BDF96A109342C4BF1346ADF86C30BDF843
:10A640006C60BDF96E200136761B36B2002E1ADD25
:10A65000531C5B1A1BB20993BDF966309B1ABDF9F6
:10A660006020AD1A09FB0355069B1AA91D441EA8BC
:10A67000764B9847BDF87E30ADF87A300027099BBD
:10A680009F42C0F27985BDF94830059AADF8603037
:10A69000013B1344ADF86430BDF84A301344ADF8C3
:10A6A0006230BDF84E309B1AADF866304246664BBC
:10A6B00018A91AA8984788B3079B43B1BBF9003083
:10A6C000BDF96C209342A8BF1346ADF86C30BDF8BD
:10A6D0006C50BDF968600135AD1B2DB2002D1DDD3C
:10A6E000BDF86E30BDF86A2001339B1ABDF96020B9
:10A6F0001BB20993B61A09F1FF3309FB0366069BE7
:10A700001AA91E441EA8514B9847BDF97A3000275C
:10A71000ADF87E30099B9F42C0F25C85059ABDF87A
:10A7200048301344ADF86030BDF84C309B1AADF89A
:10A730006430BDF94A30ADF86230013B1344ADF8E6
:10A7400066304246404B18A91AA8984778B3079B31
:10A7500043B1BBF90230BDF96E209342A8BF134646
:10A76000ADF86E30BDF86C50BDF86830BDF96A20A8
:10A770000135ED1ABDF86E3001339B1A1BB20993F7
:10A78000BDF9623009F1FF36D21A069B09FB026659
:10A790001E441AA92D4B1EA89847BDF97A302DB238
:10A7A0000027ADF87E30099B9F42C0F24285059A92
:10A7B000BDF8483005991344ADF86030BDF84C3011
:10A7C0009B1ABDF94E20ADF86430531C5B1AADF8EE
:10A7D0006230ADF866201C4B424618A91AA898476B
:10A7E000002835D0079B43B1BBF90630BDF96A207C
:10A7F0009342B8BF1346ADF86A30BDF86C50BDF84F
:10A800006830BDF96E20BDF86A100135ED1A531C91
:10A810005B1A1BB20993BDF9663009F1FF369B1A2A
:10A8200009FB0366069B1AA91E441EA8074B9847FE
:10A83000BDF87E30ADF87A302DB20027099B9F42DB
:10A84000C0F2428504E000BFB9E00000B99D0000FD
:10A85000059ABDF848301344ADF86030BDF84C306F
:10A860009B1AADF86430BDF84A301344ADF862303D
:10A87000BDF84E309B1AADF866304246B94B18A968
:10A880001AA89847E8B1079BDBB9BDF86C60BDF822
:10A890006830BDF86E70DFF810930136F61ABDF817
:10A8A0006A300137FF1A1AA9AF4B1EA89847BDF9A5
:10A8B0007A30079D36B23FB2BD42ADF87E30C0F26D
:10A8C0003C85AA4BAA4C18EE900A984718EE100A3D
:10A8D000A0470698A0479AF80C30052B40F2A880B4
:10A8E000A14B594616A89847BAF91030012B24DD20
:10A8F0009AF81430F92B20D9BAF90030EBB1BAF834
:10A900001230BDF85810C3F380020A44BDF85A1043
:10A91000ADF85820C3F340020A44ADF85A20BDF800
:10A920005C20C3F3C001521AADF85C20BDF85E2074
:10A9300003F00103D31AADF85E309AF80C908D4BFA
:10A94000B9F1FB0F28BF4FF0FF0998478A4B984792
:10A95000844B0590424616A918A89847002867D04E
:10A96000059BBDF860101A8A8B1AADF86030059B04
:10A97000588ABDF862301B1AADF86230BDF86430F9
:10A980009A1AADF864200133BDF866205B1A121ADA
:10A990001BB2ADF86620184608EE903A774B984700
:10A9A000774B054698470C90BDF830300D93002B3F
:10A9B00040F0EF849AF80630023B18BF0123BDF83F
:10A9C0005C600893BDF85830BDF85E400136F61A59
:10A9D000BDF85A300134E41A24B236B2B442BAF99E
:10A9E0000030A8BF344664109C42A8BF1C46089B98
:10A9F000002B00F0D184002C40F0CE849AF8063071
:10AA0000002B40F07C859AF80D205E4CCDE9019238
:10AA100001220092BAF8022016A94046A0474FF042
:10AA2000FF330B93514B0B989847514B284698474F
:10AA3000DAF82C00D0B19AF83630052B16D9524BE3
:10AA400098470128064600F2BC86DAF82C004F4BE6
:10AA500025A99847012800F056864D4B00934D4993
:10AA60004D4B4E4C40F294520220A0479AF81430BD
:10AA70000593052B40F27481BAF91030002B00F0D9
:10AA80006F81BAF91230002B00F06A81059BFB2B15
:10AA900028BFFF230593374B9847374B9847314BD7
:10AAA00006904246594614A89847002800F058815D
:10AAB000069BBDF850101A8A8B1AADF85030069BD1
:10AAC000588ABDF852301B1AADF85230BDF85430D8
:10AAD0009A1AADF854200133BDF856205B1A121AA9
:10AAE0000FFA83F9ADF85620244B48469847244B7B
:10AAF00004469847002840F04987BAF91230A3F17C
:10AB00000F056B426B411F46BBF80430BBF80020B9
:10AB1000BBF8021001339B1ABBF806200132521A0F
:10AB20001BB212B29342A8BF1346BAF900205B10C1
:10AB30009342A8BF1346002B099340F32A87099A32
:10AB4000174D002359461EA8A847164B00211EA8E2
:10AB500098470C9016A8044B59469847BAF812101B
:10AB600024E000BFB9E00000B99D0000CD990000CD
:10AB7000A1ED0000155200000DDC0000EDF000001A
:10AB80001D9A00001D640000317A000055D10000BC
:10AB900024770200EF7602007277020021EB0000BA
:10ABA000419B00003D990000F1F10000BDF82450E8
:10ABB000BAF81030BDF8582048075EBF5B195B42F9
:10ABC0009BB21344BAF81020ADF858300B0758BFA9
:10ABD0005319BDF85C0056BF5B4213469BB2C31AC3
:10ABE0008E07ADF85C3058BF5319BDF85A00C34EFC
:10ABF00056BF5B4213469BB20344ADF85A30CB07B5
:10AC00005CBF53195B42BDF85E004CBF13469BB25C
:10AC1000C31AAA1A12B2ADF85E3016A9012325A8EC
:10AC2000B047B74B002125A89847BAF91030099AC8
:10AC3000BDF95260BDF956C0BBF900109A42A8BFD9
:10AC4000099BBBF90420B8BF03F1FF330893BAF89E
:10AC50000E3008EE103A9AF815300793069BB3F9B8
:10AC600012E00EEB060308EE900A1BB2002F00F074
:10AC70009D87BBF90200089FADF86010A0EB0E00A5
:10AC800038448445A8BF8446CDF828C0ADF8642078
:10AC9000ADF86230ADF866300A9BB34280F27E8632
:10ACA000069BBBF90620B3F912300899BDF9526032
:10ACB000D21A521A9642B8BF16460A9AB242A4BF96
:10ACC0001646013633441BB2ADF86230ADF866303B
:10ACD000BDF956309E4240F3DD86BBF80230089A3B
:10ACE000884D013313FA82F3ADF86230BBF80630B9
:10ACF000013B9B1ABAF81020ADF86630BBF9003062
:10AD0000ADF86030013A1344ADF86430079B02930C
:10AD10000126059B019318EE102A002318A940462E
:10AD20000096A847BAF81030BBF90420ADF86420AB
:10AD3000F31A1344ADF86030079B0293059B18EE9D
:10AD4000102ACDE9006318A900234046A8476E4D9C
:10AD500018EE900AA8470C98A8476C4B20469847D5
:10AD6000DAF83C10002964D09AF84430052B60D9F9
:10AD7000002447F61843CDE90134BAF94E30009368
:10AD8000BAF94C30DAF84020614D18A8A847BDF850
:10AD900060309AF850201E94013BADF87C30BDF82D
:10ADA00062305C4D013BADF87E301EA91AAB5846AF
:10ADB000A847BAF84830BDF86820BAF84A101A44D3
:10ADC000BDF8783013FA82F3ADF87830BDF86A3008
:10ADD0000B44BDF87A1011FA83F1ADF87A10BDF882
:10ADE0007C1011FA82F2ADF87C20BDF87E2012FAB8
:10ADF00083F3ADF87E3025A8474B9847DAF840300A
:10AE00002693BAF84C30ADF8A030BAF84E30ADF811
:10AE10009E30BAF84630ADF894309AF84430009439
:10AE20008DF89C303D4CDAF83C3025AA41461EA8EE
:10AE3000A0479AF81C300593052B40F26B81BAF9B4
:10AE40001830002B00F06681059B354DFB2B28BF89
:10AE5000FF230593334B984759460B9012A8A847F8
:10AE6000BAF81A70BDF84890BDF84C40A9EB07033A
:10AE7000ADF84830BDF84A300793DB1BADF84A30D7
:10AE8000BDF84E303B449BB23C440893ADF84E3085
:10AE9000A4B2BAF900300C9312A9BAF91830ADF87F
:10AEA0004C4014A80D93A847BAF81860BDF850306C
:10AEB00009939B1BADF85030BDF85430BDF8565087
:10AEC00033441FFA83FBBDF852300A9335449B1B71
:10AED000ADB2ADF85230ADF854B0134BADF856509A
:10AEE0009847124B9847124B0690424614A916A851
:10AEF0009847002800F00E811CE000BF419B000035
:10AF00003D9900001D640000CD990000A1ED0000F6
:10AF1000D50301005DE30000717A0000A17A000012
:10AF2000B99D00001D9A0000155200000DDC0000C4
:10AF3000B9E00000079BBDF85810C3F10103C9F147
:10AF40000109B9441F44089B04EB09023B4412B2B7
:10AF50001BB29A42A8BF1A460C9B52109A42A8BF35
:10AF60001A46099BC3F1010333449B440A9BC3F176
:10AF700001031E4435440FFA8BFB2DB2AB450D9BEC
:10AF8000C84EA8BFAB4613444FEA6B0B9B45D9464E
:10AF9000A8BF9946069BBDF85C501B8AC81AADF83D
:10AFA00058000698EB1A448AADF85C30BDF85E3064
:10AFB000BDF85A0001351B1B6D1A001BADF85E3041
:10AFC0002BB208EE103AADF85A00012312A91EA8C0
:10AFD000B047B54C00211EA8A0470FFA89F2002304
:10AFE00014A908EE900A25A8B047002125A8A0477B
:10AFF000AE4B09EE100A18EE100A9847BAF918304D
:10B00000BDF95A600B9ABAF816709AF81DB0BDF9DE
:10B0100054109945BCBF03F1FF330793069BA8BFAB
:10B02000CDF81C90B3F912C00CEB060304461BB21A
:10B03000BDF95000002A40F03F87BDF95220079D1E
:10B04000ADF86000A2EB0C022A440892ADF864103F
:10B05000ADF86230ADF86630089BB34280F22486CA
:10B06000069BBDF95660B3F91230079AF61AB61A64
:10B07000089AB242A4BF1646013633441BB2ADF85B
:10B080006230ADF86630BDF95E309E4240F38D8689
:10B09000BDF85230079A864D013313FA82F3ADF8AA
:10B0A0006230BDF85630013B9B1AADF86630BDF9F1
:10B0B0005030BAF81820ADF86030013B1344012637
:10B0C000ADF86430059B01933A46002318A9404629
:10B0D000CDF808B00096A847BDF95420BAF818106A
:10B0E000ADF8642093195B1AADF86030059BCDF87C
:10B0F00008B0CDE900633A46002318A94046A847A6
:10B100006C4D18EE900AA84719EE100AA8476A4B32
:10B11000204698472DB0BDEC048BBDE8F08F294642
:10B12000664B674C324618EE100A9847BDF97A20F4
:10B13000BDF97810334618EE100AA0479AF8293066
:10B1400002930128089B5A4C08BF0220CDE9000356
:10B150001EA918EE103ABAF81E204046A047BDF8C6
:10B160007A300133ADF87A30BDF87E3001331BB24E
:10B170004D440137FFF72EBA2946504B504C32460A
:10B1800018EE100A9847BDF97A20BDF978103346B9
:10B1900018EE100AA0479AF8293002930128089B5C
:10B1A000434C08BF0220CDE900031EA918EE103A57
:10B1B000BAF81E204046A047BDF87A30013BADF8F2
:10B1C0007A30BDF87E30013BADF87E304D4401371A
:10B1D000FFF755BA394B18EE100A2A463146984700
:10B1E000079B53B9BDF97A20BDF97810344C18EE9D
:10B1F000100A2B46A047012800D102209AF82930D6
:10B2000002939AF828302A4CCDE900031EA918EEC3
:10B21000103ABAF81E204046A047BDF87A300133F4
:10B22000ADF87A30BDF87E3001331BB20137FFF73D
:10B230006FBA3378089A02EA0301FF291CBF12FB98
:10B2400003F3C3F3072118EE100A1E4B2A46984752
:10B25000079B53B9BDF97A20BDF97810184C18EE48
:10B26000100A2B46A047012800D102209AF8293065
:10B270000293FF23CDE900030D4CBAF81E2018EE0F
:10B28000103A1EA94046A047BDF87A300133ADF808
:10B290007A30BDF87E3001331BB24E440137FFF7E0
:10B2A00080BA00BF419B00003D990000EDF0000016
:10B2B0001D640000CD990000A1ED000069EE0000C2
:10B2C0008D990000F1F100003378089A02EA030139
:10B2D000FF291CBF12FB03F3C3F3072118EE100A6A
:10B2E000B54B2A469847079B53B9BDF97A20BDF95B
:10B2F0007810B24C18EE100A2B46A047012800D156
:10B3000002209AF829300293FF23CDE90003AC4CC8
:10B31000BAF81E2018EE103A1EA94046A047BDF804
:10B320007A30013BADF87A30BDF87E30013BADF8A4
:10B330007E304E440137FFF781BA9AF828109F4CAF
:10B3400018EE100A3246C847BDF97A20BDF97810C8
:10B35000334618EE100AA0479AF8293002930128C4
:10B3600008BF0220FF23CDE90003954CBAF81E2048
:10B3700018EE103A1EA94046A047BDF87A300133B6
:10B38000ADF87A30BDF87E3001331BB20135FFF7DE
:10B3900093BA0023FFF713BB002C40F3B0800023C7
:10B3A000224616A925A8874FB847874B002125A814
:10B3B00098470B90BAF8023008EE103A9AF8063027
:10B3C000022B40F0A980BAF80420BAF802309A4261
:10B3D00000F0A2807D4B7000984700270690BE4287
:10B3E0007B4B00F39080BDF95C20BDF95810ADF89F
:10B3F0006C20531C5B1A1BB2A3EB44030A93059BFE
:10B40000BDF962205B8AADF8681013441BB2ADF839
:10B410006A300792079AADF86E30BDF966309A42ED
:10B420007DDD9AF806300C9A1A4312F0FF035DD1C5
:10B430000A9A322A5ADDBDF8582012FA84F2ADF881
:10B440006820BDF85C20A6B2921BADF86C20BDF957
:10B450005A20ADF86A203244ADF86E209AF80D20DB
:10B46000574CCDE9019201220092BAF802201AA9A4
:10B470004046A047BDF95E10BDF96E30504CADF8A6
:10B480006E108A1B12B29A42D8BF0133ADF86A20FF
:10B49000D8BFADF86A309AF80D30CDE90193012795
:10B4A0000097BAF8022000231AA94046A047BDF829
:10B4B0005830ADF86830BDF85C30ADF86C30BDF890
:10B4C0005A303B443344ADF86A30BDF85E30013B3E
:10B4D0009B1BADF86E309AF80D300097CDE90193C3
:10B4E0001AA9BAF8022000234046A047069B002B69
:10B4F0003FF498AA1846374B9847FFF793BA4FF096
:10B50000FF330B9356E73AB2314650469847069BB5
:10B5100023F81700013762E70023069363E7059BD2
:10B52000B3F91270079B1F44BDF95A30234401330D
:10B530009F4208DDBDF95E301B1B013B9F4202DAD2
:10B54000089B002B36D118EE901A234B1B4E284631
:10B550009847059B5A8A079B1A44059B198ABDF890
:10B560006030194412B218EE903A09B22846B0473A
:10B5700006469AF806300993012B2FD1BAF802201B
:10B58000BAF804309A420DD0BDF85E10BDF85A30BA
:10B590000131FA1AC91A12B20D4B09B25046984736
:10B5A00008EE100A089B002B00F0A3800A9B322BA8
:10B5B0001CDC9EE00126DCE7F1F100008D99000023
:10B5C0001D640000419B00003D990000EDF000006B
:10B5D0009D9B0000A1ED0000ADF20000089B002B38
:10B5E00000F0A2840A9B322B40F39E84BDF95A30AE
:10B5F00023449F4204DDBDF95E301B1B9F425ADB92
:10B60000BDF95830ADF87830013B13FA84F3ADF84A
:10B610007C30BDF86A30ADF87A30BDF86E30ADF8E8
:10B620007E309AF80D309E4F0096A2B2CDE901937C
:10B6300009922B4618EE102A1EA94046B8479AF8E0
:10B640000620012A15D10999BDF858300B44ADF8F0
:10B650007830BDF85C305B1AADF87C309AF80D306C
:10B660000092CDE9019318EE102A00231EA940464E
:10B67000B847BDF95C300999ADF87C305A1C521AB4
:10B68000ADF87820059ABDF96010B2F910201B1BA7
:10B690000A4401339B1A9AF80D200096CDE90192D5
:10B6A00018EE102A002BACBFEB182B1C1EA97C4EE9
:10B6B0004046B0470DE0099B022B16D19AF80D3099
:10B6C000069A0096CDE90193764E2B461AA940467C
:10B6D000B047BDF86A30079A0133ADF86A30BDF85B
:10B6E0006E3001331BB2013293E6099B012B40F00F
:10B6F0001F849AF80D300096CDE9019318EE102AB8
:10B700002B461AA9D3E7BDF89630259DC3F34A17F7
:10B710001AA8654B98479AF836308DF868309AF831
:10B7200037308DF87230BAF83430ADF87430C5F374
:10B730008A25BBB203F1FF3905939AF83830BAF97C
:10B740000020DB071FFA89F940F1C680574C00231F
:10B75000594625A8A047564B002125A89847BBF875
:10B760000440BBF80030BBF806200134E41A24B2D0
:10B7700094FBF5F305FB1344BBF802300132D21AF7
:10B7800012B292FBF7F107FB112202EBD272A3EB8C
:10B7900062039BB204EBD47408EE100AADF8623079
:10B7A00064104B441BB2BDF96220ADF86630BBF9A2
:10B7B00006309A423ADD18EE100A3E4B9847FFF7E2
:10B7C00055B9022821D13C4B3C4C1EA89847BAF8E9
:10B7D0003430ADF878309AF836308DF8803000216A
:10B7E00047F61843DAF830201F92CDE90131BDF950
:10B7F00082300093DAF82C10BDF9843025A8A047D8
:10B80000BDF99450BDF9967093E72D4B00932D49E7
:10B810002D4B2E4C40F2AE520220A04700232C4C60
:10B820001A4641465846A047FFF720B9BBF80030FA
:10B830001FFA85F91B1B9BB209F1FF32ADF860308E
:10B8400013441BB2BDF96020ADF86430BBF904307D
:10B850009A4209DDBDF86230059A1344ADF86230B2
:10B86000BDF8663013449DE7022EDAF82C2010D183
:10B8700000230093174F134641461EAA18A8B84745
:10B88000BDF860304B44ADF86030BDF864304B44D7
:10B89000D7E70F4F1AAB414618A8B847F0E700BFEB
:10B8A0001D640000296A000085770000419B0000AC
:10B8B0003D990000CD990000717A0000D503010088
:10B8C00043770200EF7602007277020021EB00005E
:10B8D000ED770000A17A0000BBF80410BBF800402F
:10B8E000BBF80630BBF802000131091B01331B1AFB
:10B8F00009B2491B1BB201EBD171DB1B04EB6104E4
:10B9000003EBD37100EB610080B2A4B2013D81442E
:10B91000ADF860401FFA89F92C44022EADF86200A0
:10B92000ADF86440ADF8669007D103F00103184408
:10B930009944ADF86200ADF86690944B594618A84A
:10B9400098470446C8B90346BAF90020904D5946B5
:10B9500025A8A84721468F4B25A898470446022EC4
:10B96000DAF82C200CD1002300938B4D134641466E
:10B970001EAA18A8A84720461FE74FF0FF34EEE79D
:10B98000864D1AAB414618A8A847F4E70023FFF7F5
:10B99000BAB84FF0FF330C93FFF7DCB8804B814F00
:10B9A000494620469847069B5A8A198ABDF8503066
:10B9B0003244194412B24B4609B22046B847BDF88A
:10B9C0006230ADF86A30BDF86630ADF86E30BBF964
:10B9D0000030ADF86830013B2B44ADF86C30079B6C
:10B9E0000293059B0B9018EE102A019300902346BA
:10B9F0001AA96D4F4046B847BBF90230BAF910108A
:10BA0000BDF96E200B449A4215DABBF800302B4486
:10BA1000ADF86830BBF804305B1BADF86C30079BA9
:10BA20000293059B01930123009318EE102A002333
:10BA30001AA94046B847BBF90430ADF86C305A1C1F
:10BA4000521BADF86820099ABDF95010564F9B1A49
:10BA5000069AB2F9102001330A449B1A079A0292FF
:10BA6000059A01920B9A0092002BACBFE318231C9D
:10BA700018EE102A1AA94046B847BDF862300133C3
:10BA8000ADF86230BDF866300133ADF8663001368E
:10BA9000FFF702B9424B434F494620469847069B61
:10BAA0005A8A198ABDF850303244194412B24B46B2
:10BAB00009B22046B847BBF90030ADF86830013B09
:10BAC0002B44ADF86C30BDF86230ADF86A30BDF88B
:10BAD0006630ADF86E30079B0293059B0A9018EE16
:10BAE000102A0193009023461AA92F4F4046B847C9
:10BAF000BBF90630BAF91010BDF96E205B1A9A42F4
:10BB000015DDBBF800302B44ADF86830BBF80430CD
:10BB10005B1BADF86C30079B0293059B01930123DF
:10BB2000009318EE102A00231AA94046B847BBF923
:10BB30000430ADF86C305A1C521BADF86820099ADD
:10BB4000BDF95010184F9B1A069AB2F91020013314
:10BB50000A449B1A079A0292059A01920A9A009245
:10BB6000002BACBFE318231C18EE102A1AA940467C
:10BB7000B847BDF862300133ADF86230BDF86630C9
:10BB80000133ADF866300136FFF7A2B8BDE2000020
:10BB9000419B00003D990000A17A0000ED77000074
:10BBA000ADF200008D9900001D640000ADF8623018
:10BBB000ADF86630BAF91230ADF86010042BADF86C
:10BBC00064205ED1089A1144ADF864100022022B63
:10BBD0008DF83E208DF83F205AD101238DF83E305C
:10BBE0009DF83E30002B5DD19DF83F3083F001037E
:10BBF00003F00103AD4D8DF84030BDF956309E4243
:10BC00003FF7A5A89DF840309BB99DF83E30BDF99F
:10BC100062202BB1BBF9023008990B449A4208DD2F
:10BC20009DF83F300BB3BBF9063008995B1A9A4276
:10BC30001BDB9F4B9F4F494620469847069B5A8ADD
:10BC4000198ABDF850303244194412B24B4609B239
:10BC50002046B847079B0293059B18EE102ACDE9B2
:10BC6000000318A923464046A847BDF862300133B7
:10BC7000ADF86230BDF866300133ADF8663001369C
:10BC8000BBE7082B02BF0899521AADF860209DE768
:10BC9000012B04D0032BA3D101238DF83E308DF866
:10BCA0003F309DE70023A3E718EE101A804B814D2B
:10BCB00020469847069B5A8A198ABDF85830324464
:10BCC000194412B218EE103A09B22046A847BDF83E
:10BCD0006230ADF86A30BDF86630ADF86E30BDF94F
:10BCE0005030ADF86830013B13FA89F31FFA89F23E
:10BCF000ADF86C30059B0A900992019300902346A1
:10BD00003A461AA9694DCDF808B04046A847BDF992
:10BD10005230BAF91810BDF96E200B449A4215DA68
:10BD2000099ABDF85030CDF808B01344ADF868302A
:10BD3000BDF854309B1AADF86C30059B019301237C
:10BD400000933A4600231AA94046A847BDF954304B
:10BD50000999ADF86C305A1C521AADF86820069A51
:10BD6000BDF95810B2F91020504DCDF808B0A3EB32
:10BD700009030A4401339B1A059A01920A9A009218
:10BD8000002BACBFE318231C3A461AA94046A8472B
:10BD9000BDF862300133ADF86230BDF86630013372
:10BDA000ADF866300136FFF757B918EE101A404B60
:10BDB000404D20469847069B5A8A198ABDF858304C
:10BDC0003244194412B218EE103A09B22046A8477C
:10BDD000BDF95030ADF86830013B13FA89F3ADF886
:10BDE0006C30BDF86230ADF86A30BDF86630ADF841
:10BDF0006E301FFA89F2059B09900892019300901A
:10BE000023463A461AA9294DCDF808B04046A8471E
:10BE1000BDF95630BAF91810BDF96E205B1A9A4276
:10BE200015DD089ABDF85030CDF808B01344ADF8D0
:10BE30006830BDF854309B1AADF86C30059B019307
:10BE4000012300933A4600231AA94046A847BDF9AA
:10BE500054300899ADF86C305A1C521AADF868206D
:10BE6000069ABDF95810B2F91020104DCDF808B05F
:10BE7000A3EB09030A4401339B1A059A0192099A1C
:10BE80000092002BACBFE318231C3A461AA9404687
:10BE9000A847BDF862300133ADF86230BDF86630B6
:10BEA0000133ADF866300136FFF7EDB81D640000D0
:10BEB000ADF200008D990000DFF88C90DFF88CA0C7
:10BEC000ADF86000ADF86410ADF86230ADF86630E2
:10BED000BDF95E309E423FF713A918EE101A2046B6
:10BEE000C847069B174D5A8A198ABDF85830324404
:10BEF000194412B218EE103A09B22046A847059B21
:10BF0000CDF808B0CDE900033A46234618A94046CB
:10BF1000D047BDF862300133ADF86230BDF866300D
:10BF200001331BB20136D1E7099B022B3FF4C6ABAC
:10BF30000D9B002B7FF4DDAB0A9B322B3FF7C9AB87
:10BF4000FFF7D7BB8D990000ADF200001D64000023
:10BF5000F0B5C1F34513C2F1FF06C0F345147343B6
:10BF600004FB023301F01F0400F01F07744348F282
:10BF7000810507FB02446B436C43C3F3C553C4F311
:10BF8000C45444EA4314C1F3C4237343C0F3C4202C
:10BF900000FB023205FB02F3DB0D44EAC320F0BDD7
:10BFA00001390244904200D1704711F8013F00F876
:10BFB000013BF7E7F7B5866807460078154600228B
:10BFC000ADF8042000F01F02042A0C4609D0053AFF
:10BFD000092A1AD8DFE802F005051D3243582F2F31
:10BFE0002F2F2E4B00F01F0098473B68C0F3C7006F
:10BFF000C3F38A2313FB05F310FB04F100FB0311C9
:10C000000222274B314401A89847BDF8040003B031
:10C01000F0BD3B68C3F38A230733DB1005FB0363E2
:10C0200003EBE40304F007021B7AC2F107020121CB
:10C0300091400B401341ADF80430E6E73B68C3F391
:10C040008A2303339B1005FB036304F0030203EB15
:10C05000A40352001B7CC2F106020321E8E73B68FF
:10C06000C3F38A2301335B1005FB036202EB640216
:10C0700004F00101890092F84030C1F104010F225F
:10C080008A4013400B41D6E73B68C3F38A2315FB74
:10C0900003452E4496F80034CDE700BFAD7700008D
:10C0A000A1BF0000F0B50B460178856801F01F01C3
:10C0B000052985B004460AD10168C1F38A2112FB23
:10C0C000013202EB42022A44907805B0F0BD0B39F0
:10C0D000032956D8DFE801F00219324E2168C1F376
:10C0E0008A210731C91003F0070002FB0152DB105F
:10C0F000C0F10700D35C01228240134003410CBF12
:10C100004FF0FF300020C0B2DFE71F4900912168E7
:10C11000C1F38A210331891003F0030002FB0152AD
:10C120009B104000D35CC0F1060003228240134004
:10C13000034110336B4413F8100CC6E7134EEC4662
:10C1400006F1100E30687168674603C708367645F9
:10C15000BC46F7D12168C1F38A210131491003F0AF
:10C16000010002FB01525B108000D35CC0F10400AF
:10C170000F22DBE72168C1F38A2112FB0132A85CA0
:10C18000A3E7FF20A1E700BF0055AAFF7F770200C9
:10C190002DE9F84FB0F90830DFF8EC801B0243625C
:10C1A000B0F90A301B020A268362B0F90C3093FB07
:10C1B000F6F51FFA85F90446C9F100004FF6F67747
:10C1C00000B215FB0737C0470135ADB28246684261
:10C1D00000B2C0478346C9F15A0000B2C047C5F15A
:10C1E0005A05814628B2C047F21B07FB0BF302FB3E
:10C1F0000A3393FBF6F3E36207FB00F302FB09301B
:10C200001F4B90FBF6F02063A07C984794F83430E5
:10C2100060F3000384F83430A07C1A4B9847A37C69
:10C22000191F02298CBF00210121420042EA81022C
:10C2300094F8341002F0060221F006010A4384F853
:10C24000342022682262A28803F01F03C2F30A028C
:10C2500043EA8223B4F9062043EA4253A26902F476
:10C2600040721343A361E2894FF48033B3FBF2F3CE
:10C27000E386FF23A375238AA382BDE8F88F00BF5E
:10C28000C5770000D977000075EB00002DE9F04F6D
:10C2900085B00746DFF874B1BDF8388002910A26F0
:10C2A0004FF6F67A93FBF6F9484619FB0A3A14461C
:10C2B000D84709F10105039028B2D847054609F18E
:10C2C0005A0000B2D847019009F15B0000B2D8478C
:10C2D000019B0399A6EB0A0C0AFB00F00CFB030080
:10C2E0000F9B90FBF6F00AFB05F5B3F900E00CFBA1
:10C2F0000155B3F902C095FBF6F5CEF10003CCF180
:10C30000000208FB03F308FB02F243F30F2342F39E
:10C310000F2200FB03F905FB02FA6B434243991815
:10C32000C91311FA8CF109B201910299A1EB0E0126
:10C3300008FB01F141F30F21A4EB0C0400FB01FB0E
:10C3400008FB04F4A9EB0A0644F30F24ABEB0A0A3A
:10C350006943F61365434FEAEA3A444316FA8EF608
:10C360001AFA8EFAA9EB050936B20FFA8AFA0A44CC
:10C37000234421444FEAE939564519FA8EF9ABEBCB
:10C38000050B4FEAE1314FEAE2324FEAE3330FFAAD
:10C3900089F912FA8CF213FA8CF34FEAEB3B11FA9B
:10C3A0008CFC3146A8BF514649451BFA8EFE0FFA58
:10C3B0008EFEA8BF49467145A8BF71465645B8BF15
:10C3C00056464E45B8BF4E463980019912B2764561
:10C3D000B8BF764691421BB2A8BF114699420FFAE8
:10C3E0008CFCA8BF19466145A8BF614679800199B8
:10C3F000BE808A42B8BF0A469342B8BF134663451F
:10C40000B8BF6346FB8005B0BDE8F08F75EB000058
:10C410002DE9F04F90F83820D0F80080B0F938506E
:10C42000B0F93A6090F83A306F2A89B0044600F2C9
:10C430009280B0F93C90B9F1000FD4BF4FF00009E1
:10C440004FF00109C9F10009803DEDB26F2B00F2F8
:10C450009780B4F93E70002FD4BF002701277F4298
:10C46000803EF6B2A38AADF80A30A37D019394F81A
:10C470003430580740F1A98094F84430216CDFF83B
:10C4800048A209FB03110222414405A8D047A28813
:10C4900094F84430216C13FB02F307FB03110222D2
:10C4A000414406A8D04794F84420A388216C13FB8C
:10C4B00002F309FB021107FB03114144022207A802
:10C4C000D04794F8343099076BD400200746834650
:10C4D00094F834309B0740F1C780019AC5F1FF03FF
:10C4E00012FB05F103FB0B114343C1F3072115FBBD
:10C4F0000733C3F30723C6F1FF0C06FB01F203FB6E
:10C500000C2212120529A27500F2AA80052B40F216
:10C51000D4800026019B052B94BF00222A46BBF144
:10C52000050F98BFFF22052F98BF0025052898BF4B
:10C53000FF25002A40F09C80BDF81470002D40F0CB
:10C54000A480BDF81C10002E40F0AD80A182012017
:10C5500009B0BDE8F08F902A0ED9B0F93C90B0F93F
:10C56000042009F101099145ACBF4FF000094FF0DB
:10C570000109C5F17F0568E7FF254FF0000965E770
:10C58000902B0BD9B4F93E70B4F9063001379F42B5
:10C59000ACBF00270127C6F17F0662E7FF26002710
:10C5A00060E7226C94F84410A388013A0A4409FB1E
:10C5B000012913FB01F37B4308EB030118F809B0D1
:10C5C0008F5CC84418F8030082E7A38FDFF8FCB043
:10C5D000B4F93E2004F1180A13FA89F109B2238A4A
:10C5E0005046D847E38FB4F93C10ADF8140013FA65
:10C5F00087F212B2238A5046D847E28FA18F238A4E
:10C60000ADF818001FFA89F81FFA87F94A44414427
:10C6100012B209B25046D84794F83430ADF81C0035
:10C620009A077FF552AFB4F93C70B4F93E20244B21
:10C630000392B8440FFA88F8414650469847039A47
:10C640001F4B91440FFA89F23946834650460392B4
:10C650009847039A1A4B074641465046984737E792
:10C66000052B98BFFF2655E7FF23A3752A4660E7F1
:10C67000FF2A02D1BDF80A7060E7BDF81410BDF8BA
:10C680000A00104B9847074658E7FF2D02D1BDF826
:10C69000181058E7BDF81C10BDF81800094B2A46C1
:10C6A000984701464FE7FF2E01D1A7824FE7054B80
:10C6B000324638469847A08249E7002048E700BF45
:10C6C000A5C0000051BF0000A1BF0000B5BF000021
:10C6D0002DE9F74FDFF89081B8F8004005460E4687
:10C6E0005CB9524B00935249524B534D44220220A5
:10C6F000A847204603B0BDE8F08F504B50481F6854
:10C7000000233A46116A01338142A8BF01F1FF318B
:10C710009BB2A8BF11629C4202F12402F2D1DFF861
:10C720004CB14FF0000A4FF02409B8F800101FFA7E
:10C730008AF2914239D807F124023C4601239942FA
:10C7400056D86368DFF8F080002B5AD03D4B204666
:10C7500098473D4B0093374B772235490120C0471E
:10C760003A4B98474FF000092946394BC4F81490CA
:10C7700007463246204698470546002846D1354BA5
:10C780002B49009383222B4B334E0220C0472D4B65
:10C790002046984720462021B04720462421B04714
:10C7A0004FF0004323622C46A3E71FFA8AF409FBEB
:10C7B00004742A4B6068984780B96268AA4214D111
:10C7C0002189B2B2914210D1236A62691344B3F550
:10C7D0007A7FA8BF4FF47A7323628AE7012804D1D5
:10C7E00060682946D8470028EED00AF1010A9CE784
:10C7F000176A206A01338742B8BF14469BB22432BD
:10C800009DE7174B00937A220A4BA6E76369C4F8A9
:10C810002090002B7FF46DAF124B3846984708B13B
:10C82000606166E70123636163E700BFDB770200B5
:10C83000A67702008E78020021EB0000089000200D
:10C840000200008079D200000278020075DC00004E
:10C85000A9D100006478020051F20000317A000092
:10C860003378020089DC00006C8F0020E96F010042
:10C87000144B2DE9F7431F68134E144DDFF8508019
:10C8800004464FF0000932881FFA89F39A4202D811
:10C8900003B0BDE8F0831FFA89F3242202FB037082
:10C8A0004368A34200D04CB913B10190C04701982E
:10C8B00001902021A84701982421A84709F10109E6
:10C8C000E1E700BF089000206C8F002051F20000CB
:10C8D00079D200002DE9F7431F4C236805462BB1A0
:10C8E0001E4B0020984720681D4B984724271D4B5E
:10C8F00007FB05F098471C4B20609847064660B937
:10C900001A4B1B490093A82203201A4DA8472268FE
:10C9100019481A4933468847FEE72368DFF86080E4
:10C9200023B9A8F8003003B0BDE8F083DFF85490D5
:10C93000A8F800500025B8F80020ABB29A42F2D90E
:10C940002068AEB27E4320213044C84720682421AD
:10C950003044C8470135EEE70890002071C8000058
:10C960001DED000065EC00000D1A0000A17802002A
:10C97000A677020021EB00003E670200151A0000B6
:10C980006C8F002051F2000070B52C4B86B0084629
:10C990000E46154698470446D8B93378C3F30403C6
:10C9A000043BDBB20A2B11D873886A883168C3F361
:10C9B0004A1363F34F126A802B68214A23F01F1336
:10C9C00023F47C430A4013432B600124204606B025
:10C9D00070BD012825D11B4B0222314604A898477F
:10C9E000B8B9194E03AB0422294604A8B047174B27
:10C9F000064604A8984716B9039B042B09D0144B8C
:10CA00000093144B40F221121349144C0220A0470A
:10CA100005E02B781C3303F01F030A2BD6D9002422
:10CA2000D4E7022804D12B6803F478720C4BCAE7D0
:10CA30000C4B00934FF49A72064BE5E7317A0000F5
:10CA40001FFC1F00CDE6000045E6000015E60000D3
:10CA5000EE7802005C7A0200B778020021EB000059
:10CA60000B0420001279020070B5CC690D4684B128
:10CA70002068084E18B1084B98472068B047606896
:10CA800000B1B047A06800B1B0472046B0470023CE
:10CA9000EB6170BD1DED000015E600002DE9F04FC3
:10CAA000087B8DB0984600F01E03042BBDF958A0FA
:10CAB000179E0D46144603D000F01F03062B3ED1EF
:10CAC00095F80A90B9F1010F36D1AF4BD5F81CB0EB
:10CAD00000F01F009847E968AC4BC1F38A2118FBAE
:10CAE00001414143C91007460431DBF80000984773
:10CAF00048B1A74B0093A74B40F22E22A649A74C62
:10CB00000220A04718E0C7F3C70717FB0AF70890F1
:10CB100008ABDBF80000A24D3A463146A847089B17
:10CB20009F4200F0DB809F4B00939B49994B9B4DAC
:10CB300040F235220220A8474FF00009CEE0A3F1D1
:10CB40000B02032A00F2CE804FF47F43ADF8183079
:10CB5000A3F5AD03A3F528530793934B08AA03F15C
:10CB6000100E1746186859689446ACE8030008335D
:10CB700073456246F6D1298933464FEA112C0022CB
:10CB800010B2824503F1030314DC287B7E4B00F0D6
:10CB90001F00984701238340013B9BB204932B7BEA
:10CBA00003F01F030B3B8146032B5FD8DFE803F044
:10CBB000082E425503F8031C03F802CC0132DFE7CC
:10CBC000EB68C3F3473213F4E05F4FEAE4010CBFB4
:10CBD0000FFA82FB02F1010BE4430BFB081104F096
:10CBE000070406AFEB6903935846704B05919847CD
:10CBF000AB7A05998046002B3CD16B689A680A4451
:10CC0000C9F108000021023640B25FE0EB68A110D4
:10CC1000C3F3083213F4406F6FEA04040CBF0FFA39
:10CC200082FB02F1010B04F003040BFB081164000A
:10CC300007AFD7E7EB685905C3F3C9224FEA640190
:10CC40006FEA040454BF0FFA82FB02F1010B04F0F7
:10CC500001040BFB0811A400C4E7EA68C2F38A21AF
:10CC60008B4618FB014100242746BBE700242146E0
:10CC7000A346F9E7039B04311868444B984703988F
:10CC80005A460068DFF818B100234146D8474246AB
:10CC9000B6E7049B92F800E003FA04FC0EEA0C03EA
:10CCA00095F80CC023410CF01F0CBCF10E0FA4EB47
:10CCB000090401EB410C14BFFB5CDBB264B2002C35
:10CCC00006F80C30BCBF0446013201310BB29A4564
:10CCD000DFDC374B404698474FF0010948460DB01E
:10CCE000BDE8F08F073B032B00F2B080264B00F02D
:10CCF0001F00984701278740013FBBB203932B7B5E
:10CD000003F01F03073B8146032B70D8DFE803F0D5
:10CD100002275265EB68C3F3473213F4E05F08BFA4
:10CD200017B24FEAE40318BF571C07FB0833E4436C
:10CD300003F1080104F007041C4B04913846D5F8B0
:10CD40001CB09847AB7A04998046002B53D16B688E
:10CD50009B680B44C9F1080500206DB272E0EB68D6
:10CD6000C3F3083213F4406F08BF17B24FEAA403AD
:10CD700018BF571CE44307FB083304F0030403F116
:10CD800010016400D8E700BFAD7700007BE600002B
:10CD900038790200797A0200B778020021EB0000AE
:10CDA00045E600005B790200A17A0200EDF0000088
:10CDB000A1ED0000EB68C3F3C9225B0558BF17B2B1
:10CDC0004FEA640348BF571CE44307FB083304F0F1
:10CDD000010403F14001A400AEE7EF68C7F38A2322
:10CDE00018FB03481F4608F580610024A4E70021D2
:10CDF0000C460F46A0E7184BDBF80000174D043136
:10CE000098470023DBF800003A464146A8474346CE
:10CE1000A0E703991A78A1400A402241DBF80410E8
:10CE200031F812103170090A7170DBF80810A4EBA8
:10CE3000090464B2002C8A5CB270BCBF2C4601337A
:10CE40000130033602B29245E3DC42E7044B009323
:10CE50004FF4FE72034B51E67BE6000045E600000E
:10CE60007E790200B17A02002DE9FF470646887AF2
:10CE700001280C4678D148688B4B98478B498C4BDE
:10CE80009847002840F0A98061688A4B022202A8D6
:10CE9000984738B1884B0093884B4FF4A672884965
:10CEA000022022E0E369DFF83C92DFF83C8213BB0A
:10CEB0000C20C847E061C047054668B97F4B8049F0
:10CEC000009340F2531203207E4EB047E2697E4841
:10CED0007E492B468847FEE7E06948B97C4B0093C2
:10CEE0007749764B40F255120320764CA04774E008
:10CEF000784B0C2198470820E769C8473860C0473D
:10CF0000054668B96D4B6E49009340F25D120320EF
:10CF10006C4CA0473A686C486C492B468847FEE742
:10CF20003B684BB96A4B0093644B40F25F12644913
:10CF3000644D0320A8474CE002AA03F1080112F84F
:10CF4000010B03F8010B8B42F9D1237B03F01F0087
:10CF5000021F022A11D8A37A002B40F08880636850
:10CF60009B682361012005E00028EED14A689268A1
:10CF7000002AEAD104B0BDE8F087C21F032A00F2FC
:10CF8000D480554BDFF85CA1DFF85C919847E369EA
:10CF9000804643BB0C20D047E061C847054668B9CE
:10CFA000464B474900934FF4C6720320454EB047A5
:10CFB000E269454845492B468847FEE7E56975B96A
:10CFC000434B00933E493D4B3E4F4FF4C772032005
:10CFD000B847424B2146304698470020CAE73D4BB0
:10CFE0000C2128469847022000FA08F0E569D0474E
:10CFF0006860C847074668B9304B3149009340F232
:10D00000971203202F4CA0476A682F482F493B46B0
:10D010008847FEE7012707FA08F73846D047A86097
:10D02000C847804668B9254B2549009340F29912BC
:10D030000320244CA047AA68234824494346884734
:10D04000FEE76B680BB1AB682BB9214B009340F244
:10D050009B121A4B6BE7A37A012B49D12868204B0E
:10D06000DFF88880042198470026BE4201D10023C2
:10D0700077E70023042202A92868C0479DF8091019
:10D080009DF808306A688908DB0843EA41139DF877
:10D090000A10C90843EAC12322F81630AB689DF88C
:10D0A0000B209A550136E0E799E70000B8790200B5
:10D0B000E96F0100CDE60000BC790200D37A0200DE
:10D0C000B778020021EB00003E670200151A00004D
:10D0D000E779020051F20000AD77000069CA000054
:10D0E0007BE6000065EC00000D1A000045E600003C
:10D0F000636899680020B84201F10401B7D011F8C3
:10D10000036C11F8043C6A68B608DB0843EA46136E
:10D1100011F8026CF60843EAC62322F81030AB6817
:10D1200011F8012C1A540130E5E7A0F10B03032B91
:10D130009DD9054B214630469847044B009340F259
:10D14000D312034BABE600BF69CA0000107A02009D
:10D15000D37A02002DE9F8430B78DFF84480DFF83A
:10D1600044906FF347130B7007460C4B0C480E4668
:10D1700098470024054615B92046BDE8F8832C6879
:10D1800034B1324639462846A04701280446F3D038
:10D1900029464046C8470546EDE700BFD5E80000F0
:10D1A000F08F0020E1E800002DE9F047224B0281DA
:10D1B000044608460F46984700230128A072E36101
:10D1C0001DD11E4B384698471D4B013098471D4BCB
:10D1D0006060394698471C481C4BDFF86C90DFF8BC
:10D1E00074A098470026054604F10C084DB91EB9F5
:10D1F000174B2021204698473046BDE8F0876760EE
:10D20000E9E72B689BB16A688AB1424639462846ED
:10D210009847012806460AD10023A36123612560AF
:10D220006B6821462846984701280646E4D02946DF
:10D230004846D0470546D9E7317A0000817301009E
:10D2400065EC0000BD720100F08F0020D5E8000001
:10D2500051F20000E1E8000073B50568AC684CB11C
:10D26000069ECDE9003613460A4601462846A047E9
:10D2700002B070BD2046FBE710B50446006858B107
:10D28000C3680BB121469847A37A012B04D1034B05
:10D29000606898470023636010BD00BF1DED00006B
:10D2A00073B50E4B0E4898470E4B044698470546FB
:10D2B00060B90D4B0D490093C92203200C4EB047B5
:10D2C0000C480D4922462B468847FEE71CB10B4B04
:10D2D000102120469847204602B070BD45E8000066
:10D2E000F08F00200D1A0000F07A0200B7780200DB
:10D2F00021EB00003E670200151A000051F2000009
:10D3000037B5154B154810219847154B98470446DB
:10D31000B8B9144A009202204722134B1349144D06
:10D32000A847144A2046904798B90F4B0F490093DD
:10D3300048220320A84710481049002200238847AC
:10D34000FEE70F4B03600F4B43600F4B83600F4BA7
:10D35000C36003B030BD00BF31E80000F08F002093
:10D36000A1D20000397A0200067B0200B7780200E1
:10D3700021EB00000D1A00003E670200151A0000A4
:10D3800089C9000069CE00009DCA000069CA00007A
:10D390004368184710B40468A4465DF8044B60471E
:10D3A0001FB51346044C0A4601A9A04708B1BDF8B1
:10D3B000040004B010BD00BF95D3000003780A78C4
:10D3C000934209BF4B78981A4078C01A7047038877
:10D3D0000A88934209BF4B88981A4088C01A704740
:10D3E000531E30B5072B1FD8DFE803F02304181AAB
:10D3F0001E1E1E1C0323CD0801F007010A44072A44
:10D40000445D18D92844C2F11002417801EB04218F
:10D4100089B241FA02F203EA020030BD0723EAE7CB
:10D420000F23E8E7FF23E6E701239340013BDBB24C
:10D43000E1E71346DFE7C2F10802144103EA040002
:10D44000EBE70000032B30B504D1072A9CBF0B4B40
:10D450009A5C042301F007054FF0FF34C1F3CF01BC
:10D46000C5F10805ED1A04FA03F363F0FF03445C09
:10D47000AB402340AA401A43425430BD537B0200C4
:10D480002DE9F74F394CDFF8E8A0D4F80090277960
:10D490004318804600934FF0020B009B434502D196
:10D4A00003B0BDE8F08F6379A3B9A66801933A464B
:10D4B00031464846D047054636B1227B019B824221
:10D4C00002BF6373012363713E442573A66008F8AD
:10D4D000015BE2E7012B31D1A6681A463146484686
:10D4E000D047637B0133DBB2711C01286373A160F9
:10D4F00018D10B2B257BEAD106224846D0470736A8
:10D500006073A66010B184F805B0E0E70190314681
:10D510003A464846D0473E44019B20730546A660E4
:10D520006371D4E73A4648460191D0470199207388
:10D5300039440546A1604FF00003F1E7022B12D1F8
:10D54000667B257B013EF6B26673002EBFD1A168D3
:10D5500001913A464846D04701992073394405461F
:10D56000A1606671B3E70025B1E700BF708F0020AE
:10D57000E1D3000000880B88C01A7047F0B50C4654
:10D5800085B021B10569AB69994246D1EC69204665
:10D5900005B0F0BDAA6800FB03F6911992598F8877
:10D5A000A21ABA42039203F1010338D88B7C13B953
:10D5B000CB88134410E0012B03D1CB689B5CCA8855
:10D5C000F7E7022B14D11B480A8A009089681A4F8A
:10D5D00003A8B84720B90023C5E906431C46D6E78F
:10D5E000AB6833449A68DB88801A03EB5003F3E797
:10D5F000032BF0D10F4B0A8A009389680E4F022348
:10D6000003A8B8470028E6D0AA6832449368C01A35
:10D610004008D368D2881B5CCBE7002314206A8AB9
:10D6200099B2C2F309028A42B4D8AC610024EC6119
:10D63000ADE700BF75D50000C50401002DE9F04F2E
:10D640002DED028B0929684B05698BB008BF20219D
:10D650009847074628B900200BB0BDEC028BBDE807
:10D66000F08F2B7DD5F804909B0709EBC00809D1FA
:10D67000B8F1000FEFD059F830302868C3F3130326
:10D680001844E9E798F8044098F8053014FB03F4CF
:10D69000002CE0D0EB7CC3F38303013B032B05D8C4
:10D6A000DFE803F0025053530734E4084F4E504B69
:10D6B00030699847A0424BD359F837202B68ED7C4E
:10D6C00098F80470C2F3130213443269336008EE11
:10D6D000102A98F805200792C5F38302032A4FF019
:10D6E000000B1146327108BF042186F805B0C6F858
:10D6F00008B086F80CB086F80DB038463D4E03925F
:10D700000491B04704463846B0473B4B064639467D
:10D7100020469847B946A04607EB040AD04531D1C8
:10D72000049B17FB03F306939A464FF00108079BEF
:10D73000434532DC2046314CA0473046A0472B4BB6
:10D74000186989E70334A408B0E701346408ADE739
:10D7500021462B4B306998472A4B30619847044645
:10D7600060B9294B2949009372220320284DA8470C
:10D7700032692848284923468847FEE73369002B49
:10D780009AD168E7039B18F8012B244D594618EEEF
:10D79000100AA847049B9B44C0E7174B49463046F4
:10D7A0009847631E0593F319B34608935146089BA7
:10D7B0009B4506D1069B08F101089A440FFA88F8A8
:10D7C000B5E705981BF8012B10F8013F05905A406A
:10D7D0000270039B114D099118EE100AA847049B93
:10D7E00009991944E3E700BF7DD50000708F002040
:10D7F00085ED0000EDF0000081D40000A1ED0000F7
:10D800004DF000000D1A00005B7B02001B7B020044
:10D8100021EB00003E670200151A000045D400000D
:10D82000092A2DE9FF47DFF83CA107690C4611469C
:10D8300008BF2021804699460CBF01260026D0470C
:10D840000546002800F08680FB683BBB0023796812
:10D850003A8A01EBC50153434A88C2F30B101B11EE
:10D8600002460EB102B25200083313441B09238052
:10D870004B79A3800B79638091F90620E28091F9BE
:10D8800007202281FA7CC2F38302A272002E63D0A9
:10D890005B006380304604B0BDE8F08749464046EF
:10D8A000D0470028D2D0D8F81020D2F80C80D27CF3
:10D8B00053063AD498F80B2012F003021BD1D8F883
:10D8C0000090D8F80820DFF8A0A005EB0023ADF801
:10D8D0000C30224B009322F07F420223494603A8DA
:10D8E000D04703460028B2D0A0EB09035B08D8F864
:10D8F0000420D356ABE7012AA8D1D8F80090D8F875
:10D900000820174B009305EB002003900423DFF859
:10D9100058A022F07F42494603A8D047034600287A
:10D9200095D0A0EB09031B09E1E7D8F80420D8F84B
:10D930000810525D095C002A88D0002986D0D8F8EA
:10D94000003098F80D00013A0B4400FB023313F944
:10D95000013C7CE706469DE701269BE7BDD300001E
:10D96000CFD300007DD50000C504010010B5044CE4
:10D97000206918B1034B98470023236110BD00BFF5
:10D98000708F00201DED000010B50D4B2C210446BA
:10D9900098470C4B0022C4E900322389E26023F44B
:10D9A0007F6323F00F0343F4027343F001032381E9
:10D9B0004FF4FC63C4E908222385626110BD00BFF7
:10D9C00051F20000E0011001F8B504460D4617467B
:10D9D0001E462421034B9847C4E90057C4E9025668
:10D9E000F8BD00BF51F200002DE9F3413B4B3C4E26
:10D9F00005463C489847044698B9B04720B10024F2
:10DA0000204602B0BDE8F081374B384900937C22B4
:10DA10000320374CA0473748374900220023884766
:10DA2000FEE7364B4FF4B87198472946344B354DD5
:10DA30002C2220469847344B4C2104F13000984763
:10DA40000023C4F86C312B6803B92C6023460322F1
:10DA50001E212E48DFF8CC802F682C60C047E06282
:10DA6000B047064660B9204B204900938D22032021
:10DA70001F4DA847E26A1F481F4933468847FEE703
:10DA8000E36A002BBBD0B4F86831214E6FF3090371
:10DA90000021A4F86831C4F86C110846B047002191
:10DAA000E0630846B047002120640846B047194E9D
:10DAB00060640021206CB047606C0021B047206C8E
:10DAC000154E0021B047606C0021B047E06B134B4E
:10DAD0009847E06A124B2F60984791E745E80000AD
:10DAE0000D1A0000A88F00204FB802001CB80200D9
:10DAF00021EB00003E670200151A000051F2000001
:10DB000069EE0000848F002031E8000021520000FF
:10DB100011330000C130000089200000B12900004D
:10DB200079FE000009FE0000014B1868704700BF35
:10DB3000848F002010B9074B186838B1037A9B070F
:10DB400054BFB0F90000B0F9020070474FF4F07014
:10DB5000704700BF848F002010B9074B186838B198
:10DB6000037A9B0754BFB0F90200B0F90000704778
:10DB70004FF48870704700BF848F002010B9044BA9
:10DB8000186818B10089C0F3890070478220704777
:10DB9000848F002008B5014610B90F4B196899B160
:10DBA0000E4B0846984702460D4B084698470A23F5
:10DBB0005A43B2FBF0F01D2809D9312809D946286B
:10DBC00034BF0220032008BD4FF4F072ECE70020C0
:10DBD000F9E70120F7E700BF848F002035DB000064
:10DBE0007DDB0000436800229A61DA617047000023
:10DBF0000146034809B9034B1847034B184700BFB8
:10DC0000A88F0020D5E80000E1E8000040687047D8
:10DC10004368186818B15868003818BF0120704769
:10DC200008B5074B0246984740B11388518852689F
:10DC3000D06813FB01F31B1A5842584108BD00BFBE
:10DC400011DC00000146034809B9034B1847034B98
:10DC5000184700BFB48F0020D5E80000E1E80000BD
:10DC6000034B00221A705A6810445860704700BF76
:10DC7000888F0020034B5868012119701A78002AF8
:10DC8000FBD07047888F002010B5024B04469847A0
:10DC9000001B10BD75DC0000D1E908239A421CBFAF
:10DCA0009B0293FBF2F3D1E9060208BF4FF48063B5
:10DCB000121A534300EBA32000B2704710B5074C73
:10DCC000074801232370074B9847074B014618B9B3
:10DCD0006068BDE8104018470421F9E7908F0020E4
:10DCE000D88F0020D5E80000A5FD00002DE9F04701
:10DCF0004F48504F4E4C504D90B0B847A0B94F4D83
:10DD00004F4BA868DFF82881DFF82C91DFF848A195
:10DD1000984706464648B84704467CB9494B984759
:10DD2000A86010B0BDE8F08790F83C306FF3410375
:10DD300080F83C3001462046A847DFE700232B70DF
:10DD400094F83C309A076FD443F0020384F83C30D7
:10DD5000636A002B05DCF34203D4A3680BB12046B1
:10DD60009847636A3344002B63622EDB226A9A422F
:10DD7000D4BF626263622046214650F8103F53B31D
:10DD80009847636813B101B220689847D4E9083214
:10DD90009A421ADB94F83C30A28EE16A13F0010338
:10DDA00022D1DAB900293CD1402221466846D04729
:10DDB0002146254B40469847244B20469847244B04
:10DDC0009847039B0BB1684698472B7863B340464E
:10DDD000B8470446A1E71F4B9847D2E74FF6FF70BC
:10DDE000824204D0013AA286A28E002ADAD0226BA7
:10DDF000524262620029E8D013B9A26A52426262BA
:10DE000083F0010294F83C3062F30003D4E9060287
:10DE100084F83C30DB0758BFA16B2162C4E90620BF
:10DE2000D3E7002BE3D0BFE721464046C847D0E701
:10DE3000D88F0020D5E80000E1E80000908F002096
:10DE400089DC000075DC000099E900001DED000090
:10DE5000BDDC000099DC000069EE000038B540210F
:10DE600009480A4B0A4C0B4D98470B4B9847002327
:10DE7000A06004221E210948A847094B606098470A
:10DE80000023237038BD00BFD88F002031E8000088
:10DE9000908F002009FE000075DC0000EDDC000022
:10DEA000BDDC000010B50B4B0446402198474FF4F1
:10DEB000FA73236200216423C4E90613064B23612D
:10DEC0000123A38694F8363043F0010384F83630FA
:10DED00010BD00BF51F2000099DC00002DE9F84FA1
:10DEE000144BDFF85490DFF85CA0DFF85CB0064616
:10DEF00011480D4698474FF00008044614B94046B3
:10DF0000BDE8F88F21464846D0472368B34207460C
:10DF10000DD16368AB4200D04DB921464846D84781
:10DF2000064B20469847064B98474FF001083C4661
:10DF3000E4E700BFD5E80000D88F00201DED000009
:10DF4000BDDC0000E1E8000099E9000073B541681C
:10DF5000054611B100681D4B98471D481D4B984759
:10DF600020B11D4B98471D4B013898601C4B184839
:10DF700098471C4B04469847064660B91A4B1B4904
:10DF800000936A2203201A4DA8471A481A492246CC
:10DF900033468847FEE7B4B12B6AAB634022174B88
:10DFA00029462046984794F83630DB0706D5636843
:10DFB00023B1206810B1B4F918109847104B02B083
:10DFC000BDE87040184702B070BD00BFDDDE000044
:10DFD000D88F0020FDEA000075DC0000908F002043
:10DFE00045E800000D1A000094B8020064B8020071
:10DFF00021EB00003E670200151A000069EE0000E8
:10E00000BDDC0000F8B5094B094E0A4F044608482C
:10E010000D46984700B9F8BD0368A34202D1436892
:10E02000AB42F8D001463046B847F3E7D5E80000E8
:10E03000D88F0020E1E800008A1A002AB8BF5242B7
:10E040004FF47A735A43B2FBF0F0012838BF012035
:10E050004FF6FF73984228BF184680B2704730B51C
:10E06000B0F90430B0F9005040885B1B03EBD37368
:10E07000121A5C10C3F34F03491BD21AC91A12FBC0
:10E0800002F2644311FB01218C42B4BF0020012045
:10E0900030BD438801391944C1807047B0F9003060
:10E0A000B0F90420B0F90210D21AB0F90630581AAB
:10E0B000013002FB00007047B1F9003070B5B2F9D1
:10E0C0000050B1F90240B1F90460B1F906109D4267
:10E0D000B8BF1D46B2F902300580A342B8BF23463F
:10E0E000B2F90440B2F906204380B442A8BF3446D6
:10E0F0008A42A8BF0A46A5428480C28004DC9342BB
:10E10000CCBF0020012070BD0020FCE7B2F9003038
:10E1100010B5B1F90040A342A8BF23460380B1F96E
:10E120000240B2F90230A342A8BF23464380B1F9AE
:10E130000440B2F90430A342B8BF23468380B2F949
:10E140000630B1F906209342B8BF1346C38010BD14
:10E150002DE9F04FB1F90090B0F90040A14587B02A
:10E160008846C0F28880B0F904300193994500F3E5
:10E170008280B1F902A0B0F902B0DA457BDBB0F9D8
:10E1800006309A4577DC002A03DC012007B0BDE8A1
:10E19000F08FBDF804000290A7B20130C01B9EB200
:10E1A000ADF81040C0F3C0341FFA8BFC04FA80F0C5
:10E1B000741CA4EB0C04C4F3C03505FA84F54010BC
:10E1C0006D10A842A8BF28469042A8BF10461CFA6E
:10E1D00080F417FA80F7002285B2BFB224B204A8F7
:10E1E0000393ADF81470ADF812B0ADF81640FFF718
:10E1F000AFFF039B024640B13D44ADF814501F4BA6
:10E200005246494604A89847C0E7761BB6B2414635
:10E2100004A8ADF81260ADF81630FFF799FF02467A
:10E2200030B12F44751BADF81470ADF81250E6E70D
:10E23000029B5F1BBFB2019BADF81070414604A862
:10E24000ADF81430FFF784FF024630B17F1B761B18
:10E25000ADF81070ADF81260D1E7414604A8ADF8F2
:10E2600012B0ADF81640FFF773FF00288DD07F1B6A
:10E27000ADF81070C3E7002088E700BF5FE0000042
:10E28000B0F90020B1F904309A4214DCB0F904204E
:10E29000B1F900309A420EDBB0F90220B1F9063034
:10E2A0009A4208DCB0F90600B1F902309842B4BFD6
:10E2B0000020012070470020704700002DE9FF4139
:10E2C000B0F90070B1F90030BB4205460C4624DCC1
:10E2D000B0F90210B4F9023099421EDBB0F9041013
:10E2E000B4F90430994218DCB0F90630B4F90610DC
:10E2F0008B42CCBF0020012062B16B88164E019288
:10E3000003A92046ADF80C70ADF80E30B047019A65
:10E3100028B9002004B0BDE8F0810020ECE7B5F991
:10E320000480ADF80C8003A920460192B047002874
:10E33000EFD0EB88019AADF80C7003A92046ADF838
:10E340000E30B0470028E4D0019AADF80C8003A944
:10E350002046B047DEE700BF51E10000F0B5448839
:10E360000588142A3FD8DFE812F015003B0045006D
:10E370005A00610069007C00830085008C009300D6
:10E38000A600AD00B300C600CD00D200D700DC006F
:10E39000DF00E20082880F880132521BC2F3C036D0
:10E3A00006FA82F68A880132D21BC2F3C03707FA16
:10E3B00082F25210C2EB66021A80C2880132121B2E
:10E3C000C2F3C03000FA82F0CA8849880132521A7A
:10E3D000C2F3C03101FA82F25210C2EB600201E0D6
:10E3E00000221A805A801A8815445A881D801444C5
:10E3F0005C80F0BD82880132521BC2F3C03000FA4B
:10E4000082F08A8809880132521AC2F3C03101FAB7
:10E4100082F25210C2EB60021A800022E2E70A8800
:10E420008988521A81880A44521BF5E700221A8013
:10E430004A88C988521AC1880A4447E082880F88EE
:10E440000132521BC2F3C03606FA82F68A880132C4
:10E45000D21BC2F3C03707FA82F25210C2EB660237
:10E46000E5E78E880A88921B86883244521BDEE7D5
:10E470000022A1E78E880A88921B86883244521BAC
:10E480009AE700221A804A88C988013A521AA9E7F5
:10E4900082880E880132521BC2F3C03000FA82F02B
:10E4A0008A880132921BC2F3C03606FA82F25210F9
:10E4B000C2EB6002E6E70A888E888088921B0244DD
:10E4C000521BDFE700221A80C2880132121B89E743
:10E4D00082880132521BC2F3C03606FA82F68A885D
:10E4E00009880132521AC2F3C03101FA82F2521085
:10E4F000C2EB6602E7E70A888988521A81880A44D3
:10E50000521BE0E70A888988013A521A84E70A8890
:10E510008E88013A921B4FE70A888E88013A921B37
:10E5200085E7828801327FE782880132A7E7828807
:10E5300001329BE7830710B58CB21CBF20F8021B89
:10E5400002F1FF3204EB0443102A014600F12000DF
:10E5500004D801EB42028A420AD110BD40E90833D7
:10E5600040E9063340E9043340E90233103AEBE76F
:10E5700021F8024BEFE730B5C1F1FF04C0F34515B8
:10E5800065433F23C1EB411213FB015100F01F0310
:10E5900048F2810504FB0323C0F3C42069436B43A5
:10E5A00004FB0020C1F3C5516843C3F3C45343EADD
:10E5B0004113C00D43EAC02030BDC1F1FF0110B5C9
:10E5C000C0F3451200F01F0348F281044A434B4355
:10E5D000C0F3C420624363434843D20D6043DB0D64
:10E5E00043EA4213C00D43EAC02010BD431C184645
:10E5F00013F8012B2AB13A2AF9D05C2AF7D02F2A36
:10E60000F5D070470148024B44211847C08F0020C5
:10E6100031E8000038B50446406860B1036963B171
:10E6200021689847064B0546206898470023C4E9AF
:10E630000033284638BD0B25FBE70925F9E700BF65
:10E640001DED00007FB505461C460BB1002323607D
:10E65000686870B1866976B10023039303AB0093B9
:10E6600013460A462968B0470CB1039B236004B0E7
:10E6700070BD0B20FBE70920F9E7436810B40A4698
:10E680003BB11C6A4CB10168184623465DF8044B47
:10E6900018470B205DF8044B70470920FAE700008B
:10E6A00070B5074B074D084E04460648984700B919
:10E6B00070BD0378A342FBD001462846B047F6E779
:10E6C000D5E80000C08F0020E1E8000000232DE91C
:10E6D000F341C0E90033044617460E46002943D0F3
:10E6E0000878234B9847606028B9206003252846A6
:10E6F00002B0BDE8F08183682BB1984718B9C4E92E
:10E7000000000125F3E7636858881A4B98471A4BB5
:10E7100020609847054660B9184B194900936F224D
:10E720000320184EB0472268174818492B468847DF
:10E73000FEE7216811B961600A25D8E7D4F80480A2
:10E74000D8F80C5095B1124B304698473B460246DC
:10E750004046A84705460028C9D00E4B2068984778
:10E760000023C4E90033C2E70B25C0E70925BEE753
:10E77000A1E6000065EC00000D1A0000EDB80200F3
:10E78000ACB8020021EB00003E670200151A000041
:10E79000EDE500001DED000010B5094B044698475B
:10E7A00008B9084804E0235C2E2B02D10130204434
:10E7B00010BD2F2BF5D05C2BF3D00138F0E700BF54
:10E7C00081730100F4DD01000139031D11F8012FEF
:10E7D00000F8012B9842F9D17047000007B501926B
:10E7E00029B1006808442AB1044B01A9984703B035
:10E7F0005DF804FB024B04219847F8E7C9E70000E5
:10E8000051F2000007B5019231B103680433C81812
:10E810002AB1054B01A9984703B05DF804FB034BEF
:10E8200004219847F8E700BFC9E7000051F2000053
:10E830000023C0E901338B071CBF21F00301043121
:10E840000160704770B5044600680D4B083098476A
:10E85000054690B10146002220460A4EB04729469F
:10E860006268094B20469847616811B12A462046E4
:10E87000B047A368656003B9A560284670BD00BFB6
:10E8800065EC0000DDE7000005E8000070B5044617
:10E8900000680D4B08309847054690B101460022AC
:10E8A00020460A4EB0472946A268094B20469847A1
:10E8B000A16811B12A462046B0476368A56003B934
:10E8C0006560284670BD00BF65EC000005E80000EB
:10E8D000DDE7000000B14068704700B18068704714
:10E8E00007B50023019328B103680433194401A834
:10E8F000024B9847019803B05DF804FBC9E700009C
:10E9000007B50023019320B1036801A81944034B04
:10E910009847019803B05DF804FB00BFC9E7000009
:10E920002DE9F0410E46044640B349B3436899428D
:10E9300003D1BDE8F041134B18470068124B083073
:10E9400098470546B8B1114BDFF84880314620465C
:10E9500098472A46074601462046C0473A46294678
:10E960000B4F2046B8472A4631462046B847324624
:10E9700029462046C0472846BDE8F0810546FAE70B
:10E980000D46F8E745E8000065EC000001E90000ED
:10E99000DDE7000005E8000070B50D460446F8B15B
:10E9A000436899420CD12946174B204698470146A7
:10E9B000606008B9A06070BD0022144B20460CE0D6
:10E9C000836899420ED1124B98470146A06008B95E
:10E9D0006060F0E70F4B00222046BDE8704018470A
:10E9E0000029E0D029460A4B20469847294606468A
:10E9F000054B20469847314602460546054B2046C2
:10EA0000984732462946D8E7E1E80000DDE70000F4
:10EA100001E9000005E800002DE9F0410C461E4622
:10EA20001146164BDFF85C80154F1546984796B196
:10EA3000002229462046C047294662682046B8473A
:10EA4000616811B12A462046C047A368656003B9D2
:10EA5000A560BDE8F081A26829462046C047294646
:10EA600032462046B847A16811B12A462046B84729
:10EA70006368A560002BECD16560EAE799E90000C6
:10EA800005E80000DDE7000091422DE9F843044667
:10EA90000D46174622D01AB3144B11469847064626
:10EAA000AE421BD0124BDFF84C80DFF84C90294669
:10EAB000204698472A4631462046C04732462946D6
:10EAC0002046C8472A4639462046C8473A4629467E
:10EAD0002046C04707B9A56006B96560BDE8F88360
:10EAE00008B18668DCE70646DAE700BF01E9000006
:10EAF00099E9000005E80000DDE7000030B1436857
:10EB000033B98068B0FA80F040097047012070473F
:10EB100000207047014B1860704700BF2091002013
:10EB20002DE9F0431F46431EDBB2042BC5B004465B
:10EB30000D46164617D84DAB0DF11009DFF83080A1
:10EB400003934C9A4FF480714846C047074BD3F863
:10EB50000080B8F1000F06D0CDF800903B46324659
:10EB600029462046C04745B0BDE8F08320910020EB
:10EB700059FA00004FF4B47390FBF3F202FB130058
:10EB800000B20028BCBFC01800B259280E4B02DCEE
:10EB900033F91000704780B2A0F15A02592A03D805
:10EBA000C0F1B40080B2F3E7A0F1B40292B2592AE6
:10EBB00085BFC0F5B47080B233F8120033F810008E
:10EBC000404200B2704700BF08B9020030B50002F1
:10EBD0000023D41804FB04F5A84228BF234652089A
:10EBE000F7D11A091B01DBB20A804B8030BD00004F
:10EBF000074A0346106853B153F8042B03EB520342
:10EC0000191D00F58042914234BF1846002070471C
:10EC1000249100208B0718BF21F00301026818BF60
:10EC2000043110B50C1DB4EB520FC2F35E030BD0D0
:10EC30008B4204D0043B42185B1A5B0053600368AC
:10EC400061F35F03036010BD1946F8E7034A044B04
:10EC5000136047F6F8721A60704700BF24910020D5
:10EC60003091002073B50546E8B1820718BF20F047
:10EC70000305124E18BF043500242046B047044651
:10EC800098B10378DB07F8D40368B5EB530FF4D8D9
:10EC90000B4B29469847037843F0010304F8043BE3
:10ECA000204602B070BD074CFAE7074B00930749B6
:10ECB000074B084DD1220220A847F1E7F1EB0000F5
:10ECC00015EC000028910020EDB90200BEB9020049
:10ECD000D2BA020021EB000038B50E4B0E4D1C6875
:10ECE00004B938BD2046A8472378DA070FD5044673
:10ECF000F6E70378DB07FAD423680168C3F35E0202
:10ED0000043202EB510262F35F032360A84700283C
:10ED1000EFD1E6E724910020F1EB0000164A131D25
:10ED2000984270B5044610D078B110F8043C6FF3E7
:10ED3000000300F8043C138901339BB20F2B1381AD
:10ED400014D80E4D0438A84700B970BD0378DB070E
:10ED5000FBD454F8043C0168C3F35E02043202EBB6
:10ED6000510262F35F0344F8043CECE70023138193
:10ED7000BDE87040024B184724910020F1EB0000E1
:10ED8000D9EC000040B1054B984204D050F8040C77
:10ED9000C0F35E0070470020704700BF289100203C
:10EDA000164B1A68904213B50BD09A6890420AD15C
:10EDB000012203EBC2039A796FF300029A7102B049
:10EDC00010BD0022F5E70E4A002352F8334084427A
:10EDD00002EBC30104D18B796FF300038B71EEE773
:10EDE0000133102BF1D1074B00930749074B084C17
:10EDF00040F232220320A047E1E700BF38000020A4
:10EE00001090002006BA0200BEB90200DFBA02006C
:10EE100021EB0000114B9A796FF300022DE9F041CC
:10EE20009A719A7B0E4CDFF83C806FF3000200254C
:10EE30009A7327462E46206840B1C04707EBC503AA
:10EE400026609A7966F300029A71A6800135102D2A
:10EE500004F10804EFD1BDE8F08100BF38000020C4
:10EE6000109000201DED000070B500F0030501F0CA
:10EE70000306B54204460B4640F09880002D40F052
:10EE8000A88005462B46202A1C4601F1200503F1E7
:10EE9000200300F2B080042A0E4640F29F8051F811
:10EEA000043B44F8043B043AF5E713F8201C04F84B
:10EEB000201C13F81F1C04F81F1C13F81E1C04F858
:10EEC0001E1C13F81D1C04F81D1C13F81C1C04F850
:10EED0001C1C13F81B1C04F81B1C13F81A1C04F848
:10EEE0001A1C13F8191C04F8191C13F8181C04F840
:10EEF000181C13F8171C04F8171C13F8161C04F838
:10EF0000161C13F8151C04F8151C13F8141C04F82F
:10EF1000141C13F8131C04F8131C13F8121C04F827
:10EF2000121C13F8111C04F8111C13F8101C04F81F
:10EF3000101C13F80F1C04F80F1C13F80E1C04F817
:10EF40000E1C13F80D1C04F80D1C13F80C1C04F80F
:10EF50000C1C13F80B1C04F80B1C13F80A1C04F807
:10EF60000A1C13F8091C04F8091C13F8081C04F8FF
:10EF7000081C13F8071C04F8071C13F8061C04F8F7
:10EF8000061C13F8051C04F8051C13F8041C04F8EF
:10EF9000041C13F8031C04F8031C13F8021C04F8E7
:10EFA000021C13F8011C04F8011C203A202A1D46FB
:10EFB000214603F1200304F120043FF676AF6B1ED7
:10EFC0000A44914200D170BD13F8014F01F8014B82
:10EFD000F7E7C5F1040505441E4612B9731E224425
:10EFE00030E013F8011B04F8011BAC42194602F192
:10EFF000FF32F1D146E755F8201C43F8201C55F8A4
:10F000001C1C43F81C1C55F8181C43F8181C55F818
:10F01000141C43F8141C55F8101C43F8101C55F828
:10F020000C1C43F80C1C55F8081C43F8081C55F838
:10F03000041C43F8041C203A294624E713F8011F56
:10F0400004F8011B9442F9D1BDE700008B07F7B526
:10F050000D4618BF21F00305044618BF043528B13A
:10F0600010F8043C13F0010F08BF0024164B204693
:10F0700098478542074604D005D2144B2946201FE5
:10F08000984726460DE0124B28469847064658B941
:10F09000104B00931049114B114C40F23F120220CB
:10F0A000A047304603B0F0BD002CFAD0002FF8D0B6
:10F0B000BD422A460B4B28BF3A46214698470A4B89
:10F0C00020469847EDE700BF85ED000015EC0000F5
:10F0D00065EC0000EDB90200BEB90200F3BA02000F
:10F0E00021EB000069EE00001DED0000F7B590B1C6
:10F0F000102812D8364A937913F0010303D0937B7A
:10F10000DE070AD4012302EBC300817941F001013B
:10F11000817152F8330003B0F0BD2E4C00234FF044
:10F12000FF32271D04EBC306B5792946ED0713D43A
:10F1300037F8335085420FD305D141F0010154F81F
:10F140003300B171E7E7561C01D15AB204E004EB79
:10F15000C2018988A942F8D80133102BE2D1551C8D
:10F1600008D004EBC20154F832008B7943F001035C
:10F170008B71D0E7002504EBC50399790A46C907CE
:10F1800017D442F0010298809A710146124B54F84C
:10F190003500984744F8350040B9104B00931049AA
:10F1A000104B114E4FF404720320B04754F8350051
:10F1B000B1E70135102DDED10C4B00930320094B34
:10F1C0000749094C40F21622A0470020A3E700BFE0
:10F1D00038000020109000204DF0000032BA0200EC
:10F1E000BEB9020002BB020021EB000094BA02008B
:10F1F00010F0030310B409D0C3F1040303442AB18F
:10F2000000F8011B984202F1FF32F8D101EB012412
:10F2100004EB014404EB01640346202A184603F181
:10F22000200305D8042A0DD8084B5DF8044B184775
:10F2300043E9084443E9064443E9044443E90244FA
:10F24000203AEAE740F8044B043AEBE7F96E010094
:10F2500010F003030A460DD103460021202A184668
:10F2600003F1200315D80023042A08D940F8043BF1
:10F27000043AF9E7C3F104030344002112B90A4B2D
:10F280000021184700F8011B834202F1FF32F5D13B
:10F29000E2E743E9081143E9061143E9041143E9B0
:10F2A0000211203ADAE700BFF96E010010F0030303
:10F2B0000A460FD103464FF0FF31202A184603F1CA
:10F2C000200316D84FF0FF33042A08D940F8043B36
:10F2D000043AF9E7C3F104030344FF2112B90A4BCE
:10F2E000FF21184700F8011B834202F1FF32F5D1DC
:10F2F000E0E743E9081143E9061143E9041143E952
:10F300000211203AD9E700BFF96E01009A4238BFD6
:10F310008854704770472DE9F74F1746DDE91162B1
:10F3200012F0020A8046DDE90C54DDE90F0C9DF86D
:10F3300038E01FD102F001094EB1B9F1000F06D03B
:10F34000BEF1000F02D112F00C0F00D0013E4FF0C1
:10F35000300B02E005F804B00134A44501D9202C9B
:10F36000F8D14FF0300BB9F1000F03D0A64201D90C
:10F37000202C37D112F0100F19D012F4806F36D133
:10F38000ACB3644501D0B44231D1B4F1010C2DD0FD
:10F3900010286AD1023C900631D41F2C0FD8782057
:10F3A000285501341F2C0AD8302028550134202C30
:10F3B00005D0BEF1000F26D02D202855013492072C
:10F3C0003BD03A4625441444A2423AD1BAF1000F48
:10F3D00004D0D51BB54205EB07043DD3204603B04E
:10F3E000BDE8F08F05F804B00134BCE7644610288E
:10F3F000D1D00228D6D11F2CE1D86220D0E71F2C13
:10F40000DDD85820CCE7500701D52B20D5E71007D1
:10F41000D5D52020D1E72020CDE90013C047DDE974
:10F42000001309F101094E450BEB0902F3D8321B19
:10F43000B44288BF00223A44C4E7A146A7EB040BBC
:10F44000F1E702F1010915F8010DCDE90013C047FC
:10F45000DDE900134A46B7E72246202001930091D8
:10F460000135C047DDE90013B4E70228644699D1AD
:10F47000C3E700002DE9F04391B0189D1A9E1D9F2F
:10F480000DB927F010077C0500D515B317F0200F34
:10F4900014BF4FF0410E4FF0610EAC460DF1200845
:10F4A0000025AEF10A0EBCFBF6F906FB19C95FFA9E
:10F4B00089F4B9F1090F94BF30347444E4B2B4450F
:10F4C00008F8014BBCFBF6F405F1010501D3202D32
:10F4D00010D11C9C05941B9C0697CDE903649DF8F4
:10F4E0006440CDE9015408AC0094034CA04711B02E
:10F4F000BDE8F083A446D6E717F300002DE9F04FEE
:10F500002DED048B93B0DDE920649A4656EA04039E
:10F5100002BF289B23F010032893289B5B05DDE99D
:10F5200024B908EE100A08EE901A09EE102A02D546
:10F5300056EA04033FD0289B13F0200F14BF412349
:10F5400061230A3B0DF128080025099321461B4F32
:10F550005A464B463046B847D2B2092A8ABF099B61
:10F560003032D2185E45D2B274EB090408F8012B90
:10F5700005F1010501D3202D1AD1289B0693279B65
:10F580000593269B0E4CCDE903B39DF88830CDE959
:10F5900001530AAB009319EE102A18EE901A18EED8
:10F5A000100A5346A04713B0BDEC048BBDE8F08FA2
:10F5B00006460C46CAE70025DFE700BF15690100D3
:10F5C00017F300002DE9F04F17461E46AC4AAD4B2D
:10F5D0008946011E91B014BF93469B46002538789A
:10F5E00058B94D452CBF09F1FF322A464B46002041
:10F5F000D847284611B0BDE8F08F252807F101074C
:10F6000006D06C1C4B462A460A91D8472546D2E0C4
:10F61000002306E02D2A16D0302A0CD143F0010336
:10F620000746384610F8012B2B2A0FD0F2D8202A93
:10F630000FD0232A10D0A2F13004092C2CD84FF07F
:10F6400000080A2410E043F00203E9E743F0040352
:10F65000E6E743F00803E3E743F01003E0E704FBC9
:10F660000822A2F130080746384610F8012BA2F113
:10F67000300CBCF1090FF2D93A782E2A5AD1787899
:10F68000A0F13004092C07F1010243F4806348D84B
:10F6900000244FF00A0E14E02A2A0AD156F8048BEF
:10F6A000B8F1000FBCBF43F00203C8F100080746E1
:10F6B000E2E74FF00008DFE70EFB0400A0F13004A2
:10F6C0003A46174617F8010BA0F1300CBCF1090FB0
:10F6D000F2D917463A4612F8010B6C2833D02BD8D2
:10F6E000682837D06A283FD017F801EBBEF1780FB1
:10F6F00011D8BEF1630F3AD8BEF1620F00F0A280BC
:10F70000BEF1630F00F0FC80BEF1250F03D0BEF107
:10F71000580F00F093806C1C4B462A460A917046A5
:10F7200073E72A2805D156F8044B023724EAE4741B
:10F73000D0E717460024CDE7742801D07A28D3D12A
:10F7400043F480730BE078786C28F9D143F440736C
:10F750000237C9E77878682803D043F0800317465A
:10F76000C2E743F0C003F3E743F40073F7E7AEF1F9
:10F77000640C45485FFA8CFC012202FA0CF202404C
:10F780001BD1BEF1730F00F0FB80BEF1700FC2D130
:10F7900043F0210305930823CDE903431023CDE96A
:10F7A000012356F8043B00932A46384C0A914B46F5
:10F7B0005846A04705460A9911E7BEF1780F3FD099
:10F7C000BEF16F0F00F04481BEF1690F23F010030A
:10F7D0004FF00A0202D0BEF1640F34D1580548BF81
:10F7E00023F00103BEF1690F03F4007C02D0BEF1E7
:10F7F000640F4FD1BCF1000F28D0073626F0070662
:10F80000B24676685AF8080B0694CDE907830023C0
:10F810000593F30F002E02930492034602DA43424B
:10F8200066EB4606CDE90036194C0A914B462A464E
:10F830005846A0470A9905465646D0E643F02003AD
:10F84000102200E0022223F00C03C7E7D80506F1DE
:10F85000040A01D5306802E058060CD53078CDE9AD
:10F860000224CDE9048300284FEAD0730193B8BF86
:10F87000404200902DE01806ECD5B6F90000EEE706
:10F880000DF3000015F300002108120075F40000CC
:10F89000FDF40000BCF1000F0FD0CDE90783002379
:10F8A000CDE9042306F1070A2AF0070A0694029319
:10F8B000FAE80223CDE90023B6E7D80506F1040AE9
:10F8C0000ED5CDE90483CDE90224CDF804C0336818
:10F8D0000093604C0A914B462A465846A047A9E738
:10F8E000580607D53078CDE904830023CDE90224FA
:10F8F0000193BEE7306813F0800F18BF80B2F2E7C3
:10F9000013F0020426D04FF0010A6B1C0A930B91EE
:10F9100016F8040B4B462A46D8470B9974B30A9A3B
:10F92000544621E00A914B462020D8470A9905EB1E
:10F930000A020AF1010AC245F4D3B8F1000F08F136
:10F94000FF3308BF002308F1010A1D4408BF4FF030
:10F95000020ADAE7A246EAE70B914B462020551C43
:10F96000D8470B9901342A464445F5D30A9AA8EBA7
:10F970000A03D04538BF00231A440A920A9D2EE696
:10F980003246002C52F8046B0A9214BF20464FF006
:10F99000FF303044324692F800C0BCF1000F01D075
:10F9A000904211D1A2EB060A13F480620B9202D0AE
:10F9B000A24528BFA24613F002030C931CD1AAEB68
:10F9C00005032A460E9309E00132E4E7531C0D9328
:10F9D0000F914B462020D8470D9A0F990E9BD318B4
:10F9E0004345F3D3A8EB0A03D04538BF00230AF1FF
:10F9F00001021D4403EB020AAB1B0D9305E01C46FC
:10FA00000E914B462A46D8470E990D9B9D1916F824
:10FA1000010B28B10B9B002BF2D0631E002CEED102
:10FA20000C9B9BB12A46AAEB050406E00B914B46C2
:10FA30002020561CD8470B993246A3189845F5D874
:10FA4000A8EB0A03D04538BF00231D440A9EC6E533
:10FA50000822F8E675F4000010B4024CA4465DF8E4
:10FA6000044B6047C5F5000008B50548054B182153
:10FA70009847054B00221A7001225A7008BD00BF3A
:10FA80009C8F002031E8000050D10020F7B5364BA4
:10FA9000364898470546E0B1344E354C2B7D03F08F
:10FAA0000703032B29462ED8324B30489847324B58
:10FAB00004469847054608BB304B31490093DB228A
:10FAC0000320304EB0473048304922462B46884705
:10FAD000FEE72F4B25489847274B04469847054695
:10FAE00060B9264B26490093D3220320254EB04708
:10FAF0002548264922462B468847FEE7ECB90024D4
:10FB0000204603B0F0BD3046A04705460028C5D1C9
:10FB1000204B16489847184B044698470028EDD1CB
:10FB2000164B17490093E5220320164EB04716489E
:10FB3000164922462B468847FEE74FF4FA732360A6
:10FB4000237D154D032262F30203002723754FF036
:10FB5000FF3301262361A760104B2E709847E760A2
:10FB60006060AE70CCE700BFD5E800009C8F00203D
:10FB7000E1E8000021E900000D1A000042BB02008C
:10FB800012BB020021EB00003E670200151A0000C4
:10FB900045E800008DE8000050D1002075DC000031
:10FBA00070B501460446074B0748084D98470126A3
:10FBB000074B2E7020469847064B1B68A34208BF90
:10FBC000EE7070BD99E900009C8F002050D100209C
:10FBD0001DED00000C90002038B5124B0446406823
:10FBE0009847236898421BD30F4B104D984700232A
:10FBF000EB70AB70A368606043B92369002B0CDC29
:10FC0000236943B90A4B2046984704E020469847A9
:10FC1000EB78002BF1D0012038BD013B2361EFE7E9
:10FC20000020F9E789DC000075DC000050D10020DD
:10FC3000A1FB00002DE9F84FDFF85CB19BF8044010
:10FC4000012034B99BF801208BF804001AB98BF815
:10FC50000420BDE8F88FDFF84481DFF838A1DFF831
:10FC60004091C047CBF80800002250468BF8032093
:10FC70008BF80220C847434D434F2860296889B15B
:10FC8000424B5046984706462868027D12F007010D
:10FC900008D0A04250D0052939D1B8479BF802209E
:10FCA000002A62D03A4CDBF80800A047DBF80C20B1
:10FCB0001044CBF80C00DBF81400A047B0F5FA7F35
:10FCC00016D3DBF80C2064214A434FF4FA71B2FBDF
:10FCD000F1F2D2B2642A9ABFC2F16402D2B2002217
:10FCE0008BF810200022CBF80C20C047CBF8140072
:10FCF0004FF0FF322748CBF81820C847254E234F36
:10FD00000546E5B9DBF818008BF80450A1E734B1DB
:10FD1000217D02F0070201F007018A42BED9B847EF
:10FD20000028BBD09BF80220002ABBD19BF80320FF
:10FD3000002AB7D12C6897E700242E609EE72A7D21
:10FD400053070DD06868A0472A68904238BF101A40
:10FD5000DBF8182028BF0020824288BFCBF81800AB
:10FD600029463046B8470546CBE79BF80320002AD2
:10FD700098D19BF800100029DFD08BF800201446A2
:10FD800072E700BF0C900020D9FB0000E1E8000002
:10FD900089DC00009C8F002050D1002075DC000021
:10FDA000D5E80000F8B5037D03F007038B42044655
:10FDB0000D4618D00F48104B0E4E104F9847024674
:10FDC00032B1137D03F007039D420DDBA24203D045
:10FDD00008480B4B214698470A4B01221A70237D95
:10FDE00065F302032375F8BD11463046B847024655
:10FDF000E6E700BF9C8F0020D5E80000E1E80000A6
:10FE000089EA000050D100202DE9FF411E46124B27
:10FE100003920F4680469847104B04469847039933
:10FE2000054668B90E4B0F4900934FF483720320C7
:10FE30000D4EB0470D480E4922462B468847FEE737
:10FE400034B10C4BC4F80880276020469847E66020
:10FE5000204604B0BDE8F0818DFA00000D1A0000C4
:10FE600057BB020012BB020021EB00003E670200FC
:10FE7000151A0000A5FD000010B5044B0446984774
:10FE80002368C31A013B636010BD00BF75DC00002E
:10FE900090F900200378002A0FDA03F0E002C02A6C
:10FEA0000DD003F0F002E02A0BD003F0F800A0F12F
:10FEB000F0035842584180007047012070470220EB
:10FEC00070470320704773B50023019301B901A95E
:10FED0000A688556835C002D02F1010403DB184695
:10FEE0000C6002B070BD03F0E005C02D10D10C60B5
:10FEF000005D00F0C004802C01D00020F1E79B01E0
:10FF000003F4F86300F03F00184402320A60E8E7A7
:10FF100003F0F005E02D17D10C60045D04F0C0057E
:10FF2000802DEAD1951C0D60455D05F0C00080284C
:10FF3000E3D1180380B205F03F05A401284404F47E
:10FF40007C6420440332E1E703F0F805F02D0C60F7
:10FF5000D3D1045D04F0C005802DCED1951C0D6079
:10FF6000455D05F0C006802EC7D1D61C0E60805DB1
:10FF700000F0C006802EC0D19B042403AD0100F028
:10FF80003F0003F4E01304F47C3405F47C651C4367
:10FF9000054428190432B9E70B68F7B5013B0D4F4A
:10FFA0000B6006460C46042520683B6830449847A1
:10FFB000236848B92BB1013D013B15F0FF052360D3
:10FFC000F2D1002003B0F0BD019301A97B68304657
:10FFD0009847F7E7480000202DE9F0410024DFF8BA
:10FFE000288007460D462646AE4202D12046BDE88F
:10FFF000F0813819D8F800309847012838BF01201F
:020000021000EC
:1000000054FA80F40136EFE748000020F7B50024E9
:10001000074F019406460D46019BAB4202D3204692
:1000200003B0F0BD7B6801A9304698470134F3E77F
:100030004800002073B50024074E01940546019B3B
:10004000EB5C13B9204602B070BD736801A9284665
:1000500098470134F3E700BF480000207F2882B0B2
:1000600011D9B0F5006F10D2830963F03F0300F09F
:100070003F008DF8043060F07F0000238DF805000C
:10008000ADF80630019802B07047B0F5803F14D249
:10009000030B63F01F038DF80430C0F3851363F086
:1000A0007F0300F03F008DF8053060F07F000023F3
:1000B0008DF806008DF80730E4E7B0F5881FE1D22F
:1000C000830C63F00F038DF80430C0F3053363F045
:1000D0007F038DF80530C0F3851300F03F0063F017
:1000E0007F0360F07F008DF806308DF80700C9E7C8
:1000F000030612D5C0F30722030603EB0243C0F345
:10010000074203EB022303EB10600423C2B202B9DF
:10011000000A013B13F0FF03F8D17047232916D1E1
:1001200002785AB9012303700278012A04D12029E8
:1001300004BF02230370134618467047012A4FF08C
:100140000003F0D0022AEFD103700123ECE7002373
:10015000EAE700002DE9F04F884685B017461E46B5
:100160000546002400283ED0002A3ED003948DF896
:100170000B40002935D09DF83890DFF87CA009F0BD
:100180000109DAF8043003A9284698478346039802
:10019000DAF804200021284490470246B9F1000F04
:1001A00011D1134B59463846984703B2002B14DC43
:1001B000039B9845E5D8002C01DDA61B34B22046F0
:1001C00005B0BDE8F08F01900A4B59460DF10B00C8
:1001D0009847019A0028E4D0EAE73444204404B266
:1001E000E6E70C46EBE70446E9E71446E7E700BF1D
:1001F000A1D300001D010100480000202DE9F04FAF
:100200008FB099469DF8603002910492039307469F
:1002100098B1002900F0D280039B13F012030FD095
:10022000002000E001303B5C0A2B00F0C9800D2B60
:1002300000F0C680002BF5D180B20FB0BDE8F08F82
:10024000039A8DF82B3012F00202059247F61842FD
:1002500018BF91460B930B9B009307EB030BFB5CC2
:10026000002B00F08E80B9F1000F40F38A80059AD0
:1002700047F61843002A08BF4B460793514B002509
:100280005B68CDE90C550CA9584698470C9B0D931B
:10029000039B019503F0010380464FF0FF3A2E4681
:1002A0002A462C4608931BF8043043B9BAF1FF3FA5
:1002B00052D0009B002B6ED11FFA8AF455E0414BBF
:1002C0000DA95B6858469847019B01330693089B2C
:1002D000024673B109903C4B41460DF12B00984703
:1002E000099A30B1DDE90C430C93069B01939046CB
:1002F000D9E7364B0298099241469847064400B226
:100300000028C8BF049B099AB6B2C4BFF618B6B29B
:10031000BAF1FF3F36B205D1049B0799F31A8B421D
:10032000C8BFA246B8F10A0F10D0B8F10D0F0DD01A
:1003300027480023D9B2415C21B9BAF1FF3F08BF79
:100340003546CFE7884503F10103F3D1002CADD149
:10035000BAF1FF3FADD13546019B23B1B8F10D0F86
:1003600002D10A2A00D10C9CA4B2A9EB05050B9B73
:100370000FFA85F994B95BB9124B0BA95B68384643
:1003800098470B9B23B90F4B0BA95B6838469847DE
:10039000BDF82C0051E700252C46E6E71C443B78CD
:1003A0000B940A2BEDD00D2BEBD03B5D0A2B02D02A
:1003B0000D2B7FF450AF01340B94E2E702983CE739
:1003C000013039E7480000201D010100A1D30000E1
:1003D00066BB02002DE9F04F89B0002598469DF8D4
:1003E0005030BDF948B0BDF94CA004930446164600
:1003F00005804580039129B322B3049B13F0020FBB
:1004000047F6184318BF9A46B2F908300693138985
:1004100005935B440793039B03EB05095B5DA3B95D
:1004200055B119F8013C0A2B01D00D2B04D1059BC5
:1004300062885B4413446380B4F90230002B31D1ED
:10044000069B638009B0BDE8F08F049B0093424691
:1004500053463146154F4846B847B4F90230079A1B
:100460001344B3F5004F014605440BD3104B114C18
:1004700012931149114B71220220A44609B0BDE824
:10048000F04F60476380049B009348464346DFF883
:1004900030903246C847B4F900309842B8BF184689
:1004A0002080B8E7A3EB0B03CBE700BFFD01010001
:1004B0009DBB020021EB00006EBB0200DDBB020011
:1004C000550101002DE9F047089D80460F4614466E
:1004D00099460CB9264612E04FEA540A09FB0A76FF
:1004E00031464046A847002808DDE44304F00104F3
:1004F000AAEB040A06EB09075446EAE7FCD13046AA
:10050000BDE8F087014B1860704700BF6CD1002038
:10051000014B1B68D86870476CD10020014B1B68E9
:100520001B6818476CD10020C0F3031310B500F00E
:10053000F001C4B2C0F30712194300F00F0343EAFD
:10054000041322F00F02890842EA1020C3F3C40307
:1005500043EA4113C0F3C40043EAC02010BD0000C9
:1005600001392DE9F0470446272934D8DFE811F096
:1005700028003900BB00820044004F004703B70049
:100580000F01560239006F0320029503B700B70030
:100590007100B7005101B700F701150285032A0168
:1005A0003B01EF016601D301EB001B033703D700CA
:1005B000980084028E01B901F002C701BE02E50273
:1005C000994B00219847994B002120469847984B1A
:1005D0001968984B98472046974BBDE8F047FF2194
:1005E0001847914B00219847904B0021204698478F
:1005F0008F4B19680431ECE78B4B002198478B4BEC
:100600000021204698478A4B19681031E1E7884E4F
:10061000DFF81492DFF81482864D0021C8470021CC
:100620002046C047316804310746A8473168183171
:100630003846A84701212046C84701212046C04727
:10064000316804310746A847316838460831A84761
:10065000C1E70021DFF8D091DFF8D081744E754DED
:10066000C84700212046C04731680746A84731687F
:100670006831DDE7DFF8B0816D4E6C4F6D4D0021C4
:10068000C04700212046B84731682431A8470121DE
:100690002046C04701212046B84731682831D6E7B7
:1006A000DFF88481624E614F624D0021C047002116
:1006B0002046B84731682431A84701212046C04769
:1006C00001212046B84731682831A8470221204639
:1006D000C04702212046B84731689C31B7E7524BEA
:1006E0000021984777E7DFF84091514EDFF83C81D1
:1006F000504D0021C84700212046C04731680431D1
:100700000746A847316838462031A84701212046CE
:10071000C84701212046C04731681C3197E7DFF800
:100720000881434E414F434D0021C04700212046E0
:10073000B84731682031A84720460121C047012130
:100740002046B847E8E73A4EDFF8DC80374F394DAE
:100750000021C04700212046B84731682431814636
:10076000A847316848469431A84701212046C04730
:1007700001212046B84731682831A8470221204688
:10078000C04702212046B847316890315FE7284FC3
:10079000DFF89480254E274D0021C04700212046D8
:1007A000B04739684C31A84740212046C047402116
:1007B0002046B047396810310646A84739683046A8
:1007C000503144E7184B1A4F1A4E00219847174BE7
:1007D000002120469847396804310546B0473968FA
:1007E0007C3128467BE0DFF84080114E0F4F114DE1
:1007F0004021C04740212046B84731681831A847FA
:1008000041212046C04741212046B8473168103178
:100810001DE7054B00219847044B002120469847CF
:10082000034B19686C31D4E675270000B926000027
:1008300070D1002045580000BD2F0000DFF8A882CD
:10084000A64EA74FA74D0021C04700212046B8471C
:1008500031680431A84740212046C0474021204646
:10086000B84731681431A84701212046C04701210B
:100870002046B84731688031A84702212046C0474A
:1008800002212046B84731688431E0E6964D934F07
:10089000DFF84C82934E0021A84700212046C04734
:1008A0003968B04740212046A84741212046A84743
:1008B00041212046C0473968A831B047432120462E
:1008C000A84743212046C0473968AC31B047422190
:1008D0002046A84742212046C0473968A431B04786
:1008E00079E6814D0021A84740212046A8477C4B4E
:1008F000402120469847794B1968B03169E60021BC
:10090000DFF8E481754E764F764DC04700212046D2
:10091000B8473168A7E7714EDFF8CC91DFF8C081A6
:10092000704D0021C84700212046C047316804317E
:100930000746A847316838468831A8470321204632
:10094000C84703212046C04731688C317FE6664B9B
:1009500000219847624B0021204698473BE6624FB2
:100960005E4EDFF87C915F4D0021B84700212046A4
:10097000C847316804318046A84731684046743121
:10098000A84740212046B84701212046B847012109
:100990002046C8473168803159E6534B00219847BB
:1009A0004F4B0021204698474C4B1968783110E690
:1009B0004A4EDFF834814A4F4A4D0021C04700219A
:1009C0002046B847316804318146A8473168484617
:1009D0000831A847316848461831A84740212046C9
:1009E000C04740212046B847316804318146A847B6
:1009F000316848465431A84741212046C04741212B
:100A00002046B84731688031A84742212046C04778
:100A100042212046B8473168583118E62F4EDFF89A
:100A2000C890DFF8BC802F4D0021C8470021204628
:100A3000C047316804310746A8473168384640311D
:100A4000A847316838461831A84701212046C847D1
:100A500001212046C047316818310746A847316850
:100A600038464431A84702212046C8470221204683
:100A7000C04731684831EAE5DFF86C80174E184FFF
:100A8000184D0021C04700212046B8473168043185
:100A9000A84701212046C04701212046B8473168B8
:100AA000A031A84702212046C04702212046B8476E
:100AB0003168A031A84703212046C04703212046C2
:100AC000B8473168A031A84704212046C047042117
:100AD0002046B8473168A031B9E500BF70D1002089
:100AE000B92600004558000075270000DFF8008295
:100AF0007C4E7D4F7D4D0021C04700212046B847E8
:100B00003168A84742212046C04742212046B847C5
:100B100031688031A84741212046C0474121204605
:100B2000B8473168B031A84740212046C04740212E
:100B30002046B8473168A83189E56D4B00219847B8
:100B4000694B002120469847664B1968A43140E55F
:100B5000DFF89C81634E644F644D0021C047002143
:100B60002046B847316804318146A8473168484675
:100B70001831A84720460421C04704212046B84721
:100B80003168B831A84720460321C04703212046D9
:100B9000B8473168B431A84720460121C047012138
:100BA0002046B847F6E64F4EDFF84491DFF838812B
:100BB0004E4D0021C84700212046C047316804310E
:100BC0000746A847316838461831A8470321204610
:100BD000C84703212046C0473168983137E5444B68
:100BE000404F424E002198473F4B002120469847F6
:100BF000396804310546B04739680831F1E5DFF856
:100C0000F080384E384F394D0021C0470021204632
:100C1000B84731680431A84703212046C047032163
:100C20002046B84731682C31A84701212046C047EB
:100C300001212046B84731683031A84702212046BB
:100C4000C04702212046B84731683431FFE4DFF85D
:100C5000A080244E244F254D0021C047002120466E
:100C6000B84731683831A84701212046C0470121E3
:100C70002046B84731683C31E9E41D4B194F1B4E03
:100C800000219847184B00212046984739680431C5
:100C90000546B04739687031A3E5124EDFF8508041
:100CA000114F124D0021C04700212046B84731683E
:100CB00004318146A847316848465C31A847012184
:100CC0002046C04701212046B84731686031A84717
:100CD00002212046C04702212046B84731686431CE
:100CE000B5E400BF70D10020B926000045580000CF
:100CF00075270000034B1B790BB1034B1847034BBF
:100D0000FCE700BF70D10020C15900005D57000012
:100D10002DE9F0413A4D3B4B28683B4E3B4C9C3013
:100D2000984728683A4BFF222C219C309847286826
:100D3000384B29211A88384B9C309847286847F649
:100D4000FF7201219C30B04700202F68A0473B284C
:100D500007F19C0747DD0020A0476FF0270300F153
:100D6000140292FBF3F212B238461021B047002071
:100D70002F68A0473B2807F19C0737DD0020A047DC
:100D80006FF0270300F1140292FBF3F212B238461F
:100D90001121B04700202F68A0473B2807F19C078E
:100DA00027DD0020A0476FF0270300F1140292FB1B
:100DB000F3F212B212213846B04700202D68A04746
:100DC0003B2805F19C0517DD0020A0476FF02703A5
:100DD00000F1140292FBF3F212B2284633461321BB
:100DE000BDE8F04118474FF0FF32BDE74FF0FF324A
:100DF000CDE74FF0FF32DDE74FF0FF32EDE700BF08
:100E000070D10020F50C0100A55A00007DDB000028
:100E1000455C0000F2BB0200755B00002DE9F0416B
:100E20006B4D6C4B28686C4E6C4C70309847286842
:100E300047F6FF7201217030B04700202F68A047AD
:100E400000EB80008000EF2807F1700740F3B280CC
:100E50000020A0471423502200FB0322A02392FB72
:100E6000F3F212B238461221B04700202F68A04793
:100E700000EB80008000EF2807F1700740F39C80B2
:100E80000020A0471423502200FB0322A02392FB42
:100E9000F3F212B238461321B04700202F68A04762
:100EA00000EB80008000EF2807F1700740F3868098
:100EB0000020A0471423502200FB0322A02392FB12
:100EC000F3F212B238461021B04700202F68A04735
:100ED000C0EB00104000EF2807F1700770DD002024
:100EE000A0471E23502200FB0322A02392FBF3F213
:100EF00012B238461421B04700202F68A04700EBFB
:100F0000800000EB8000EF2807F170075ADD002019
:100F1000A0471923502200FB0322A02392FBF3F2E7
:100F200012B23846C021B04728682D4FAA899921AE
:100F30007030B8472868AA89C9217030B847286836
:100F4000284B00F1700840F688009847CA210246F5
:100F50004046B84700202F68A04700EB80004000C3
:100F6000EF2807F170072FDD0020A0470A23502249
:100F700000FB0322A02392FBF3F212B29021384629
:100F8000B04700202D68A047C0EBC000EF2805F156
:100F900070051BDD0020A0470723502200FB032221
:100FA000A02392FBF3F212B228463346C321BDE8D8
:100FB000F0411847012255E701226BE7012281E742
:100FC000012296E70122ACE70122D7E70122EBE7F5
:100FD00070D10020F50C0100A55A00007DDB000057
:100FE000755B0000290501002DE9F041324C334BBF
:100FF0002068334F334E344D6C3098472068FF22C1
:101000002C216C30B8472068A28929216C30B04768
:101010002068022230216C30A84720687F223C21C2
:101020006C30B8472068294B00F16C074C21A0892F
:101030009847392102463846B0472068244F47F682
:10104000FF7201216C30A8472368002003F16C086F
:10105000B847C0EB0010EF282ADD0020B8470F2367
:10106000502200FB0322A02392FBF3F212B2502184
:101070004046A8472068A28959216C30B04700201B
:101080002468B84700EB8000EF2804F16C0411DD00
:101090000020B8470523502200FB0322A02392FB27
:1010A000F3F212B220462B465321BDE8F041184717
:1010B0000122DCE70122F5E770D10020F50C0100E8
:1010C000455C0000755B0000A55A000077E5000054
:1010D0007DDB0000C0F38522C0F3C40343EA421362
:1010E000C0F3C44043EAC020704700002DE9F04738
:1010F000434CDFF834912068424E434FDFF82C8197
:101100002430C847206847F6FF7201212430B047D9
:101110002068FF2224302C21B847236A256813F069
:10112000020F14BF39483A48C047243502462921E6
:101130002846384DA847236803F1240A236A9A07F2
:1011400058D53548C047024679215046A8472068FF
:10115000A28949212430A8472068E28940F2494108
:101160002430A847206800224C212430B84720684A
:101170007F224FF413712430B847206803224021A6
:101180002430B04720689622B0212430B047206830
:101190004C22B7212430B04720682830C847206847
:1011A000FF222C212830B847206847F6FF72012122
:1011B0002830B0472068A28929212830A847206814
:1011C000164B00F1280640F68800984742F22901A4
:1011D00002463046A847236A20689B0700F128068C
:1011E0000BD50F48C047024630462B467921BDE853
:1011F000F04718470B4B1A88A6E70A4B1A88F3E703
:1012000070D10020A55A0000455C0000D9D7D40059
:101210004D494500755B00004F4031002905010034
:101220004F404100F2BB0200F50C0100D510010057
:101230002DE9F0417D4C7E4F20687E4D9030B847BF
:1012400020687D4BFF222C2190309847236A20682C
:101250009A0756BF794BA2891A8890302921A8474E
:10126000236A26689B0706F1900640F1CC807448FB
:10127000744B9847024630467921A8472068724E41
:10128000724D47F6FF7201219030B047236800206D
:1012900003F19008A847C0EBC000EF2840F3B680E8
:1012A0000020A8470723502200FB0322A02392FB23
:1012B000F3F212B240461221B0472368002003F136
:1012C0009008A847C0EBC000EF2840F3A1800020A1
:1012D000A8470723502200FB0322A02392FBF3F22E
:1012E00012B240461321B0472368002003F1900852
:1012F000A847C0EBC000EF2840F38C800020A8472F
:101300000723502200FB0322A02392FBF3F212B228
:1013100040461021B0472368002003F19008A847F9
:10132000C0EBC000EF2877DD0020A847072350223C
:1013300000FB0322A02392FBF3F212B211214046DC
:10134000B04720689430B84700202768A84700EBD2
:1013500080004000EF2807F194075FDD0020A847D8
:101360000A23502200FB0322A02392FBF3F212B2C5
:1013700038461721B04700202768A84700EB8000B7
:101380004000EF2807F194074ADD0020A8470A2310
:10139000502200FB0322A02392FBF3F212B2384644
:1013A0001821B04700202768A84700EB80004000C4
:1013B000EF2807F1940735DD0020A8470A235022C3
:1013C00000FB0322A02392FBF3F212B21521384650
:1013D000B04700202468A84700EB80004000EF28B9
:1013E00004F1940420DD0020A8470A23502200FBCA
:1013F0000322A02392FBF3F212B2204633461621B9
:10140000BDE8F04118470D4B1A8834E7012251E737
:10141000012266E701227BE701228FE70122A7E78D
:101420000122BCE70122D1E70122E6E770D10020CA
:10143000F50C0100755B0000455C0000F2BB02008A
:101440004F403100D5100100A55A00007DDB00009F
:101450002DE9F047B64CDFF8F4822068DFF8F0920F
:10146000B44F5C30C047206800F15C0540F688004E
:10147000C847992102462846B847206800F15C0514
:1014800040F68800C847C92102462846B847206868
:10149000A289A94DCA215C30B84700202668A84718
:1014A00000EB8000EF2806F15C0640F38D81002000
:1014B000A8470523502200FB0322A02392FBF3F24E
:1014C00012B2304690219D4EB0472368002003F1B0
:1014D0005C0AA8473B2840F379810020A8472823CD
:1014E00000F1140292FBF3F212B25046C321B0474E
:1014F0002368002003F15C0AA8471D2840F3688197
:101500000020A847142300F10A0292FBF3F212B262
:101510005046C221B0472368002003F15C0AA84767
:1015200000EB80008000EF2840F354810020A847A2
:101530001423502200FB0322A02392FBF3F212B2E9
:1015400050461221B0472368002003F15C0AA847E7
:1015500000EB80008000EF2840F33E810020A84788
:101560001423502200FB0322A02392FBF3F212B2B9
:1015700050461321B0472368002003F15C0AA847B6
:1015800000EB80008000EF2840F328810020A8476E
:101590001423502200FB0322A02392FBF3F212B289
:1015A00050461021B0472368002003F15C0AA84789
:1015B00000EB80008000EF2840F312810020A84754
:1015C0001423502200FB0322A02392FBF3F212B259
:1015D00050461421B0472368002003F15C0AA84755
:1015E000C0EB0010EF2840F3FD800020A8470F2338
:1015F000502200FB0322A02392FBF3F212B25046CA
:10160000C021B047206847F6FF7201215C30B04727
:1016100020686030C047206800F1600A40F688000A
:10162000C847992102465046B847206800F1600A31
:1016300040F68800C847C92102465046B84720688E
:10164000A289CA216030B8472368002003F16009ED
:10165000A8471D2840F3C8800020A847142300F1A4
:101660000A0292FBF3F212B248469021B047236877
:10167000002003F16009A8471D2840F3B78000202F
:10168000A847142300F10A0292FBF3F212B2484673
:10169000C321B0472368002003F16009A84700EB8D
:1016A000800000EB8000EF2840F3A2800020A847D4
:1016B0001923502200FB0322A02392FBF3F212B263
:1016C000C0214846B04720686430C047236803F112
:1016D0006408236A9A0740F18D801948194B98478E
:1016E000024640469921B8472368002003F1640868
:1016F000A8471D2840F381800020A847142300F14B
:101700000A0292FBF3F212B240469021B0472068E1
:101710000D4BFF222C2164309847236803F16408A5
:10172000236A9B076BD50648064B9847024611E093
:1017300070D10020755B00007DDB0000A55A000021
:101740005B4B4600D5100100455C0000F50C010024
:101750002905010029214046B847206847F6FF7255
:1017600001216430B04700202768A847C0EB001073
:101770004000EF2807F1640744DD0020A8471E233E
:10178000502200FB0322A02392FBF3F212B20321AA
:101790003846B04700202468A84700EB800040008E
:1017A000EF2804F164042FDD0020A8470A2350220B
:1017B00000FB0322A02392FBF3F212B22046334631
:1017C0001421BDE8F047184701227AE601228CE691
:1017D00001229DE60122B3E60122C9E60122DFE6ED
:1017E0000122F5E601220AE701223DE701224EE748
:1017F000012265E7054B1A8873E7012284E7034B52
:101800001A88A7E70122C2E70122D7E7F2BB02004C
:101810002DE9F047684D694F2868DFF8BC914030EA
:10182000B8472B6A2C6813F0020F04F1400400F053
:10183000B180634B40F6AA209847024648F28901DE
:101840002046DFF898815F4CC04728684430B8478D
:1018500000202E68A047EF2806F1440640F39D8043
:101860000020A047A02300F1500292FBF3F212B235
:1018700030469021544EB0472B68002003F1440AB3
:10188000A04700EB80004000EF2840F38880002054
:10189000A0470A23502200FB0322A02392FBF3F26D
:1018A00012B250469221B0472B68002003F1440A3F
:1018B000A04700EB80004000EF2872DD0020A04729
:1018C0000A23502200FB0322A02392FBF3F212B260
:1018D00050469321B0472B6803F1440A2B6A9B07BB
:1018E0004CBF3A483A48C847992102465046C0473B
:1018F00028684830B84700202F68A04700EB400018
:10190000EF2807F148074EDD0020A04703235022AF
:1019100000FB0322A02392FBF3F212B2384690217F
:10192000B04700202F68A0473B2807F148073CDD5F
:101930000020A047282300F1140292FBF3F212B218
:1019400038460321B04700202F68A047772807F1C9
:1019500048072CDD0020A047502300F1280292FB0D
:10196000F3F212B214213846B04700202D68A04788
:10197000EF2805F148051CDD0020A047A02300F159
:10198000500292FBF3F212B2284633460121BDE821
:10199000F04718470F48C8474FE7012268E7012280
:1019A0007FE7012294E70122B8E70122C8E701227C
:1019B000D8E70122E8E700BF70D10020F50C010054
:1019C000290501007DDB0000A55A0000E3DDD600FB
:1019D000978A8000BDADA100D5100100755B0000A5
:1019E0002DE9F04F2DED028BA14CA24F2068A24DA6
:1019F000DFF8B0A283B0B8472068FF222C21A847A7
:101A0000236A266813F0020F14BF9C489C48AB461B
:101A10009C4DA847B94602469B4F30462921B847FE
:101A2000236A266898074CBF98489948A84748F207
:101A3000890102463046B847236A266899074CBF99
:101A400092489348A847792102463046B8476269D0
:101A50002068904E48F28E01D047626920687E214E
:101A6000D04720680430C8472368002003F10408E9
:101A7000B0471D2840F368850020B047142300F1CB
:101A80000A0292FBF3F212B240460121DFF81882FB
:101A9000C0472068FF2204302C21D847236803F177
:101AA000040B236A9A0754BF7B486FF07F40A84716
:101AB000292102465846B847236803F1040B236ADC
:101AC0009B074CBF75487648A847392102465846BF
:101AD000B8472068A28940F239210430B84720680D
:101AE000E28940F239410430B8472368002003F10D
:101AF000040BB047772840F32A850020B0475023D5
:101B000000F1280292FBF3F212B258463021C0478E
:101B10002068012233210430C04720686269043004
:101B200048F28E01D047236803F1040B236A98071B
:101B30004CBF56486FF07F40A84748F289010246E3
:101B40005846B8472068626904307E21D047236830
:101B500003F1040A236A99074CBF4C486FF07F4099
:101B6000A847792102465046B847236803F1040A82
:101B7000236A9A074CBF45486FF07F40A84748F258
:101B8000A90102465046B847236803F1040A236AB4
:101B90009B074CBF3D486FF07F40A8479921024604
:101BA0005046B8472068DFF804A101229021043094
:101BB000C04723680020043308EE103AD0470128BC
:101BC0004FF0000000F2D384B047C0EB0010EF28C4
:101BD00000F3C0844FF0010B0020B047772840F39A
:101BE000D1840020B0475023283090FBF3F080B21E
:101BF0000BEB000212B218EE100A1221C047236844
:101C00000020043308EE103AD04701284FF00000BE
